:020000040800F2
:100000000000012095410008FD270008FF27000897
:100010000128000803280008052800080000000047
:100020000000000000000000000000000728000899
:1000300009280008000000000B2800080D2800080F
:10004000E5410008E541000811280008E5410008E5
:10005000E5410008E54100081D28000823280008A4
:10006000E5410008E541000855280008E541000881
:10007000292800082B2800082D2800083928000806
:100080004528000851280008E5410008E54100081E
:1000900000000000E541000857280008E54100087D
:1000A000E5410008E5410008E5410008E541000898
:1000B000E5410008E5410008E5410008E541000888
:1000C000E5410008E5410008E5410008E541000878
:1000D000E541000861280008E5410008E541000805
:1000E000E54100085D2800086D280008E54100088A
:1000F000E54100080000000000000000E5410008A4
:10010000E5410008E541000879280008E5410008BC
:10011000E5410008E5410008E5410008E541000827
:10012000E5410008E5410008E5410008E541000817
:08013000E5410008E54100086B
:1001380010B5054C237833B9044B13B10448AFF319
:1001480000800123237010BDBC08002000000000BF
:100158005840010808B5034B1BB103490348AFF3E6
:10016800008008BD00000000C008002058400108B9
:1001780014214160704714207047406A704700009E
:10018800790100087F01000883010008990100082F
:1001980010B5044604F1100000F05CFCC4F8F80047
:1001A8000148C4F87C0110BD88010008F8B5E6B024
:1001B80004460D4616461F460A4906A800F0CAFE20
:1001C80070996F9A05910492009733466E996D9ACB
:1001D800039102922A466C990191214600F060F839
:1001E80067B0F0BD94010008F8B5E6B004460D46C6
:1001F80016461F46094906A800F0ACFE6F996E9A8C
:100208000491039200976D996C9A0291019233467A
:100218002A46214600F087F867B0F0BD940100082F
:1002280038B500281CBF01680029184A23D1184B8B
:100238001C684FF6F0710C404CF24025AC421FBFD1
:100248001B6819404CF27024A14212D1114D296843
:1002580079B911490B68C3F30B03B3F58A6F1FBF54
:100268000968C1F30B0140F28343994204BF01219D
:10027800117028B905E0094B994204BF012111709A
:100288004068BDE8324001F09FBE00BFD80800209A
:1002980000ED00E0002004E00010005C000037489A
:1002A8002DE9F04104460D46216816464A681F4666
:1002B80090478046B8F5403F2ED122680A99936846
:1002C800204698478046B8F5403F25D12368089ACC
:1002D8000799D3F80CC02046E0478046B8F5403F60
:1002E8001AD12368069A39461F692046B8478046BE
:1002F800B8F5403F10D1236829465D69324620464B
:10030800A8478046B8F5403F06D123680B9A09995B
:100318009D692046A847804621680A68204690477C
:100328004046BDE8F0812DE9F04104460D462168BC
:1003380016464A681F4690478046B8F5403F2ED17A
:1003480022680A999368204698478046B8F5403F46
:1003580025D12368089A0799D3F80CC02046E047AE
:100368008046B8F5403F1AD12368069A39461F6976
:100378002046B8478046B8F5403F10D12368294643
:100388005D6932462046A8478046B8F5403F06D109
:1003980023680999DD6900222046A847804621681C
:1003A8000A68204690474046BDE8F0814FF4403047
:1003B80070470000F0B50C4685B0114600281A4673
:1003C8001CBF0568002D0B4B11D082B104B971B95F
:1003D8000D9860B10F9E0E9F0A9B0290049603979A
:1003E8000B980C9E009001962046A8470346184695
:1003F80005B0F0BD020003002DE9F04F0646D0B06D
:100408000868F56DD6F860E0726EB76EF36E00BAE4
:1004180000906C46486800BA60600DF14008886832
:1004280000BAA060C86800BAE060086900BA206134
:10043800486900BA6061886900BAA061C86900BAF1
:10044800E061086A00BA2062486A00BA6062886A95
:1004580000BAA062C86A00BAE062086B00BA2063FA
:10046800486B00BA6063886B00BAA063C86B00BAB7
:10047800E063402058F80C1C58F820CC58F838ACE9
:100488008CEA010158F840CC8AEA01018CEA01099A
:100498004FEAF979401E48F8049BEBD187EA02003D
:1004A80000EA0E00784010EBF5610098DFF824C4EC
:1004B80041186144C81882EABE032B404FEAF06134
:1004C80053405918636859186144CF194FEAB50366
:1004D80083EABE01014081EABE0111EBF765A1681C
:1004E8004D196544A91883EAB0023A404FEAF1650C
:1004F8005A405519E26855194FEAB70282EAB0071F
:1005080065440F4005EBBE0E97EAB00717EBFE6592
:1005180027697D194FEAB10782EA0701654401EAB4
:100528000E01EB18514011EBF36561694D194FEA63
:10053800BE0187EA010E65440EEA030E15EBB00012
:100548008EEA070E0EEBF065D4F818E075446544A2
:10055800AA1881EAB30505404FEAF26E4D40AE4451
:10056800E569AE44E64477444FEAB00080EAB30E4A
:100578000EEA020E8EEAB30E0EEBF765D4F820E011
:1005880075446544691880EAB2053D404FEAF16E4A
:100598004540AE44656AAE44E6440EEBB3034FEA09
:1005A800B70787EAB20E0EEA010E8EEAB20E0EEB1C
:1005B800F365D4F828E075446544281887EAB1053E
:1005C8001D404FEAF06E7D40AE44E56AAE44E64415
:1005D8000EEBB2024FEAB30383EAB10E0EEA000E45
:1005E8008EEAB10E0EEBF265D4F830E0754465443E
:1005F800EF1983EAB00515404FEAF76E5D40AE4447
:10060800656BAE44E6440EEBB1014FEAB20282EAF2
:10061800B00E0EEA070E8EEAB00E0EEBF165D4F8B6
:1006280038E075446544EB1882EAB7050D404FEA97
:10063800F36E5540AE44E56BAE44E6440EEBB000B5
:100648004FEAB10181EAB70E0EEA030E8EEAB70E41
:100658000EEBF065D4F840E07544654481EAB30ECA
:10066800AA180EEA000E4FEAF2658EEA010E7544EA
:10067800DDF844E04FEAB000754480EAB30E654403
:100688000EEA020E15EBB7078EEAB30E0EEBF7650E
:10069800DDF848E04FEAB202754480EA020E65448C
:1006A8000EEA070E69188EEA000E0EEBF165DDF80A
:1006B8004CE07544654405EBB3034FEAB70E1427C5
:1006C8000DF1500CDFF810528EEA010B82EA0B0B89
:1006D8000BEBF36A5CF804BBDA44AA44504483EA9F
:1006E800B10B4FEAF06A8EEA0B0BDA445CF804BBF4
:1006F800DA44AA44524480EAB30B4FEAF26A8BEA1E
:10070800B10BDA445CF804BBDA444FEAB000AA44FF
:1007180080EA020BD6448BEAB30B0BEBFE6A5CF85B
:1007280004BBDA444FEAB202AA4482EA0E0B0AEB8F
:10073800B10180EA0B0B0BEBF16A5CF804BBDA44FD
:100748007F1DAA44282F0AEBB3034FEABE0EBBD382
:100758003C2F61D3502F4DD204EB870CC7F15407BF
:100768005E4CA7FB04A504465D4FA8088EEA010A63
:1007780082EA0A0A5CF804BB0AEBF3655D447D195A
:100788002C1983EAB10A4FEAF4658EEA0A0A55443D
:100798005CF804AB5CF804BB55447D19AA1884EADC
:1007A800B30A4FEAF2658AEAB10A55445D444FEA52
:1007B800B4047D1984EA020AAE448AEAB30A0AEB51
:1007C800FE655CF804AB55444FEAB2027D1982EA33
:1007D8000E0A15EBB10184EA0A0A5CF804BB0AEBBD
:1007E800F1655D447D1915EBB303401E4FEABE0E5B
:1007F800BCD12046F46D1B19F365336EC9183166F8
:10080800716E71447166B36ED218B266F16E40189B
:10081800F06650B0BDE8F08F4EEA010B0EEA010A0F
:100828000BEA020B4BEA0A0A0AEBF36554F827A015
:10083800DFF8B0C0554443EAB10B654403EAB10A96
:100848000BEA0E0B28184BEA0A0A7F1C0AEBF06524
:1008580054F827A0554440EAB30B654400EAB30AAC
:100868000BEAB10BAA184BEA0A0A7F1C0AEBF265DD
:1008780054F827A055444FEAB00040EA020B6544FB
:1008880000EA020A0BEAB30BAE444BEA0A0A7F1CE1
:100898000AEBFE6554F827A055444FEAB20242EA33
:1008A8000E0B654402EA0E0A0BEA000B15EBB101C8
:1008B8004BEA0A0A7F1C0AEBF16554F827A0554455
:1008C8007F1C65443C2F05EBB3034FEABE0EA3D350
:1008D80040E700BF9979825AA1EBD96ECDCCCCCC38
:1008E800D6C162CADCBC1B8F00B581B00168074A5B
:1008F800914200D110B9064801B000BD7C2113F027
:100908000FFB4FF4003001B000BD00BFFC09000828
:10091800030002002DE9F0410B4A92E8F85188B033
:10092800694681E8F8510268084B9A4200D118B923
:10093800074808B0BDE8F0811422083000F04FFBEA
:1009480008B0BDE8F08100BFDC090008FC09000818
:1009580003000200152904D20268044B9A4200D110
:1009680008B903487047083000F048BBFC09000884
:100978000300020010B481B013460268074CA2427B
:1009880000D118B901B010BC0548704701B000F19A
:10099800240210BC083000F035BB00BFFC09000879
:1009A8000300020010B481B013460268074CA2424B
:1009B80000D118B901B010BC054870470A4601B00B
:1009C80000F1240110BC083000F070BBFC090008DD
:1009D800030002000123456789ABCDEFFEDCBA981E
:1009E80076543210F0E1D2C300000000000000008D
:1009F80000000000F10800081D0900085D09000852
:100A08007D090008AD09000801040008790F0008F5
:100A1800C50F0008810F0008F0B5A3B004460B48C5
:100A280002900D4616461F46094B0822402104A88D
:100A380000F0D1FA28980190009733462A462146BB
:100A480002A800F01BF823B0F0BD00BFFC090008A5
:100A5800100A000810B5040008BF002408D0054893
:100A6800054B20600822402104F1080000F0B3FA89
:100A7800204610BDFC090008100A00082DE9F041C5
:100A880004460E46216817464A681D469047804628
:100A9800B8F5003F19D1226806999368204698470F
:100AA8008046B8F5003F10D123683146DE683A46E3
:100AB8002046B0478046B8F5003F06D12368079A1C
:100AC80029461D692046A847804621680A682046AD
:100AD80090474046BDE8F08110B500F033FA4FF476
:100AE800403400280EBF034C4FF4C07113F018FABD
:100AF800204610BD0200030010B5044600F022FA9B
:100B080008B9054810BD0021A160D0F87C21116802
:100B180088474FF4403010BD0200030070B504460A
:100B28000D4600F00FFA064E40B1D0F87C0141683E
:100B38008847A84224BF65604FF44036304670BDF0
:100B4800020003002DE9FF4715000C4600D02CB128
:100B5800064600F0F7F95FEA000801D16448C3E0EF
:100B6800D8F8F80001684A689047B0F5003F17D1F7
:100B7800D8F87C118A68404690478146B9F1810FC0
:100B880080F09E80A94508F1FC0A17D2D8F8F80031
:100B98000368D3F80CC02A462146E047B0F5003F69
:100BA80040F08E80D8F8F8000368D3F810C06A4681
:100BB8005146E047B0F5003F76D10AE0002004E056
:100BC800215C0AF800100098401C00900098A84288
:100BD800F6D34FF0000C4749474A484B01AC009800
:100BE800844558D2D3E9007001ADC5E9007010788A
:100BF80000281ABF042086464FF0000E085854F803
:100C08000E5028443E4D05600127D0F800E087606B
:100C1800019D4F681AF80C007D408EEA050585F0A5
:100C2800040E65680F687D4085F0FC05754485F005
:100C3800A30568400AF80C000CF1010CCFE7D3E9D2
:100C4800004501A8C0E9004510782E4D002814BFC2
:100C58004FF0040E4FF0000E01A8744651F80EE054
:100C68000459A6440127CEF80050DEF80040CEF81B
:100C780008704D68019F40687D406C400D68684071
:100C880084F0040480F0FC00041984F057040AF886
:100C98000C400CF1010CCC45D1D3D8F8F800016810
:100CA8004A689047B0F5003F0AD1D8F8F8000368C1
:100CB800D3F80C804A465146C047B0F5003F01D0F2
:100CC800114811E0002006E05AF8201081F06A313E
:100CD8004AF82010401CB0EB990FF5D3B06840F0EB
:100CE8000100B0604FF4403004B0BDE8F08700BFA9
:100CF80002000300F0400108D8080020240F000873
:100D0800ADBE4ED70DBE75A10100030038B50C4627
:100D1800017A1546CA0702D500F014F908B908483F
:100D280032BDD0F8F80003682146DC682A46A0479F
:100D3800B0F5003F01D0034832BD4FF4403032BD1A
:100D480002000300010003002DE9F84191B00546B7
:100D58000E461746402101A813F0E2F8297AC80781
:100D680004D5284600F0EEF8040002D1DFF8A4808C
:100D78004BE0D4F8F800DFF8A0800368D3F810C07F
:100D88006A4601A9E047B0F5003F3ED1D4F8F80023
:100D980001684A689047B0F5003F36D1D4F87C1115
:100DA8008A6820469047D4F8F830024618461B68EF
:100DB800D3F80CC004F1FC01E047B0F5003F24D1A2
:100DC800D4F87C0141688847D4F8F83002461846C0
:100DD8001B68D3F80CC001A9E047B0F5003F14D157
:100DE800D4F8F8000268696893689847B0F5003F3E
:100DF8000BD1D4F8F80003681C693A463146A0477D
:100E0800B0F5003F08BF4FF44038404612B0BDE887
:100E1800F08100BF02000300010003002DE9F84142
:100E2800A5B0074688461646402115A813F078F85D
:100E380000220492402105A813F072F8387AC107FD
:100E48005ED5384600F07EF8050059D0D5F8F80090
:100E58002D4C0368D3F810C06A4605A9E047B0F5E1
:100E6800003F3CD1D5F8F80001684A689047B0F5D2
:100E7800003F34D1D5F87C118A6828469047D5F8C8
:100E8800F830024618461B68D3F80CC005F1FC017F
:100E9800E047B0F5003F22D1D5F87C01416888478A
:100EA800D5F8F830024618461B68D3F80CC005A9D7
:100EB800E047B0F5003F12D1D5F8F800026879682C
:100EC80093689847B0F5003F09D1D5F8F800036852
:100ED8001D6904AA15A9A847B0F5003F01D020460E
:100EE8000FE00A4B0A490B4A0396029101924046C9
:100EF8001C68049B009415AA796800F0E5F900E0E5
:100F0800054826B0BDE8F08101000300F84001085B
:100F1800936E030026C703000200030004B001011A
:100F280000170145E10A0008010B0008250B00081D
:100F3800B50300084D0B0008150D0008510D0008F9
:100F4800250E00080168024A914218BF0020704728
:100F58002C0F000810B5040008BF002404D0034873
:100F68002060204609688847204610BD2C0F0008DD
:100F780020225C3012F0D2BFF0B58468A3080022AA
:100F880004F0030407E000F15C0555F8226035BA67
:100F980041F82250521C9A42F5D300220BE000F18E
:100FA8005C0502EB830755F82360D500C5F11805E9
:100FB800EE40CE55521CA242F1D3F0BD30B5C46804
:100FC80003690022E31AD5188C5C0544521C082AD0
:100FD8002C77F8D330BD0360C1600261704738B523
:100FE800044615460022626023685A68904700202C
:100FF8006061A061A5604FF4003032BD81604FF49C
:10100800003070472DE9F84304462079D4F80C8065
:10101800450748BF244845D466691D46A8F1010024
:1010280000EAD60306EBC506B6EBC50F666102D229
:10103800A669761CA6611746A66906EB5576A661D1
:101048000E46E918884225D2A8EB03094A463146DC
:10105800F81812F063FF2268136839460FE0424619
:10106800384612F05BFF23681A68394620469047D5
:1010780007E0311811F00300F1D122681368204607
:101088009847484600EB0809A9F10101A942F0D3A5
:10109800002300E000202A1A3118F81812F03EFF49
:1010A8004FF40030BDE8F283040002002DE9FC4F44
:1010B800024685B0D0681369DFF86CC1DFF86C812F
:1010C800A0EB030A506840F004005060002703A812
:1010D80002900DF10C0ED8E9003403A8544DC0E974
:1010E80000342878534D00280CBF00230423994668
:1010F8005CF803305EF80940234401261D601C6833
:101108009E60DCF80430039DDCF80090DEF8046093
:101118005D406540484C654089EA0606474C664094
:101128007519474C6540D8E9006B03AC0028C4E941
:10113800006B0EBF002404200424029E5CF800000B
:10114800345920183F4C04600126046886600398CF
:10115800029E43406340384C7068634089EA00004F
:10116800364C6040034438484340280018BF0120EB
:101178005B1E9B41042F2CBFC0B2D80F02F1140391
:1011880053F8200007F00303C3F10303DB00D84042
:101198000DF807007F1C082F9DD315460C466A6979
:1011A800AB69E868D20842EA4372401E00EA0207C7
:1011B800002302409B420AD8524508D28020E055BD
:1011C8007F1C574516D2AAEB0701E01910E08020D2
:1011D800E05500E0E355E8687F1C8742FAD32A68A7
:1011E800136828469847BAF1000F03D051462046A5
:1011F80012F096FE2A68069E059F9368694628465F
:1012080098472A68D2F8009021462846C8472B6894
:10121800DA683946284690470EB1A86830604FF41E
:10122800003007B0BDE8F08FF04001085412000804
:10123800D80800205FC5109304850012FC68017A65
:10124800C0F524FF24AF33D426AF698B04B0010165
:1012580000170145F8B501240094002300240DE08F
:10126800009D065D0F5D7E40F643761CF60F86F006
:10127800010635400095641C009DEB189442EFD39D
:101288001846F2BDF8B5002301240094002A11E0A5
:10129800009C85188F1815F8016C17F8015C6E40D2
:1012A800F643761CF60F86F0010634400094009C45
:1012B800E318521EECD11846F2BD00005D1200087A
:1012C8008D120008010000002DE9F84F1D46DDF8D9
:1012D80028900B9F0D9C4FF0FF3300930E469246CB
:1012E800D9F800B0804632465146D847834664B3A1
:1012F800D9F8043032465146404698476FEA0B0207
:10130800521C42EA0B0200996FEAD2735B1C194027
:10131800C2430091521C024300996FEAD2735B1CCE
:101328001940009186F05531484087EA000181F064
:101338005531216080F05531C943491C0843009A52
:101348006FEAD070401C82430092D9F80800012847
:1013580009D17540E943491C0D4300986FEAD572DD
:10136800521C90430AE0F11C85EA9102D243521CB8
:10137800154300986FEAD5735B1C984386F0AA362C
:10138800009086EA0B0686F0AA33F243DB430C98FA
:10139800C2F3C0725B1C42EAD3720099D243521C5A
:1013A80091430091774000998843009987F0AA37C4
:1013B8000F403843BDE8F28F034613F8012B002A8B
:1013C800FBD1181A0138704781F0004102E000BFD4
:1013D80083F0004330B54FEA41044FEA430594EAED
:1013E800050F08BF90EA020F1FBF54EA000C55EA28
:1013F800020C7FEA645C7FEA655C00F0E2804FEAF9
:101408005454D4EB5555B8BF6D420CDD2C4480EADA
:10141800020281EA030382EA000083EA010180EA0A
:10142800020281EA0303362D88BF30BD11F0004F58
:101438004FEA01314FF4801C4CEA113102D040428E
:1014480061EB410113F0004F4FEA03334CEA1333C9
:1014580002D0524263EB430394EA050F00F0A780E1
:10146800A4F10104D5F1200E0DDB02FA0EFC22FADC
:1014780005F2801841F1000103FA0EF2801843FAD0
:1014880005F359410EE0A5F120050EF1200E012AC1
:1014980003FA0EFC28BF4CF0020C43FA05F3C018FF
:1014A80051EBE37101F0004507D54FF0000EDCF178
:1014B800000C7EEB00006EEB0101B1F5801F1BD321
:1014C800B1F5001F0CD349085FEA30004FEA3C0C25
:1014D80004F101044FEA445212F5800F80F09A801B
:1014E800BCF1004F08BF5FEA500C50F1000041EB1F
:1014F800045141EA050130BD5FEA4C0C404141EB23
:101508000101013C28BFB1F5801FE9D291F0000F1D
:1015180004BF01460020B1FA81F308BF2033A3F1CC
:101528000B03B3F120020CDA0C3208DD02F1140CC3
:10153800C2F10C0201FA0CF021FA02F10CE002F1FE
:101548001402D8BFC2F1200C01FA02F120FA0CFCF7
:10155800DCBF41EA0C019040E41AA2BF01EB045140
:10156800294330BD6FEA04041F3C1CDA0C340EDC3E
:1015780004F11404C4F1200220FA04F001FA02F381
:1015880040EA030021FA04F345EA030130BDC4F13F
:101598000C04C4F1200220FA02F001FA04F340EA34
:1015A8000300294630BD21FA04F0294630BD94F0E5
:1015B800000F83F4801306BF81F480110134013DCC
:1015C8004EE77FEA645C18BF7FEA655C29D094EA3D
:1015D800050F08BF90EA020F05D054EA000C04BFBB
:1015E8001946104630BD91EA030F1EBF00210020A6
:1015F80030BD5FEA545C05D14000494128BF41F045
:10160800004130BD14F580043CBF01F5801130BDA8
:1016180001F0004545F0FE4141F470014FF0000033
:1016280030BD7FEA645C1ABF194610467FEA655CE4
:101638001CBF0B46024650EA013406BF52EA033586
:1016480091EA030F41F4002130BD00BF90F0000F74
:1016580004BF0021704730B54FF4806404F13204B0
:101668004FF000054FF0000150E700BF90F0000F69
:1016780004BF0021704730B54FF4806404F1320490
:1016880010F0004548BF40424FF000013EE700BF60
:1016980042004FEAE2014FEA31014FEA02701FBFF0
:1016A80012F07F4393F07F4F81F06051704732F022
:1016B8007F4208BF704793F07F4F04BF41F4002179
:1016C800704730B54FF4607401F0004521F00041D7
:1016D8001CE700BF50EA010208BF704730B54FF061
:1016E80000050AE050EA010208BF704730B511F062
:1016F800004502D5404261EB41014FF4806404F19A
:1017080032045FEA915C3FF4D8AE4FF003025FEA1F
:10171800DC0C18BF03325FEADC0C18BF033202EBA3
:10172800DC02C2F1200300FA03FC20FA02F001FAFD
:1017380003FE40EA0E0021FA02F11444BDE600BFA0
:101748004FF0FF3C06E000BF4FF0010C02E000BF85
:101758004FF0010C4DF804CD4FEA410C7FEA6C5C68
:101768004FEA430C18BF7FEA6C5C1BD001B050EA0B
:10177800410C0CBF52EA430C91EA030F02BF90EAF6
:10178800020F0020704710F1000F91EA030F58BFB5
:10179800994208BF90422CBFD8176FEAE37040F017
:1017A800010070474FEA410C7FEA6C5C02D150EAB5
:1017B800013C07D14FEA430C7FEA6C5CD6D152EA70
:1017C800033CD3D05DF8040B704700BF8446104635
:1017D80062468C461946634600E000BF01B5FFF734
:1017E800B7FF002848BF10F1000F01BD4DF808ED04
:1017F800FFF7F4FF0CBF012000205DF808FB00BFD5
:101808004DF808EDFFF7EAFF34BF012000205DF82E
:1018180008FB00BF4DF808EDFFF7E0FF94BF01207B
:1018280000205DF808FB00BF4DF808EDFFF7CEFF7C
:1018380094BF012000205DF808FB00BF4DF808EDBB
:10184800FFF7C4FF34BF012000205DF808FB00BF8C
:101858004FEA410212F5001215D211D56FF47873D0
:10186800B3EB625212D94FEAC12343F0004343EA73
:10187800505311F0004F23FA02F018BF404270474E
:101888004FF00000704750EA013005D111F00040D8
:1018980008BF6FF0004070474FF00000704700BF6E
:1018A80080F0004002E000BF81F0004142001FBF0D
:1018B8005FEA410392EA030F7FEA226C7FEA236C16
:1018C8006AD04FEA1262D2EB1363C1BFD21841400B
:1018D80048404140B8BF5B42192B88BF704710F0A1
:1018E800004F40F4000020F07F4018BF404211F044
:1018F800004F41F4000121F07F4118BF494292EAAC
:10190800030F3FD0A2F1010241FA03FC10EB0C00D7
:10191800C3F1200301FA03F100F0004302D5494264
:1019280060EB4000B0F5000F13D3B0F1807F06D311
:1019380040084FEA310102F10102FE2A51D2B1F109
:10194800004F40EBC25008BF20F0010040EA0300FE
:101958007047490040EB0000013A28BFB0F5000F7E
:10196800EDD2B0FA80FCACF1080CB2EB0C0200FA34
:101978000CF0AABF00EBC25052421843BCBFD04083
:101988001843704792F0000F81F4000106BF80F4FD
:1019980000000132013BB5E74FEA41037FEA226CC0
:1019A80018BF7FEA236C21D092EA030F04D092F08B
:1019B800000F08BF0846704790EA010F1CBF0020BF
:1019C800704712F07F4F04D1400028BF40F000401C
:1019D800704712F100723CBF00F50000704700F03C
:1019E800004343F0FE4040F4000070477FEA226263
:1019F80016BF08467FEA23630146420206BF5FEA34
:101A0800412390EA010F40F4800070474FF0000333
:101A180004E000BF10F0004348BF40425FEA000CFA
:101A280008BF704743F0964301464FF000001CE0A2
:101A380050EA010208BF70474FF000030AE000BFF8
:101A480050EA010208BF704711F0004302D5404236
:101A580061EB41015FEA010C02BF844601460020A8
:101A680043F0B64308BFA3F18053A3F50003BCFAC3
:101A78008CF2083AA3EBC25310DB01FA02FC634470
:101A880000FA02FCC2F12002BCF1004F20FA02F277
:101A980043EB020008BF20F00100704702F120026A
:101AA80001FA02FCC2F1200250EA4C0021FA02F2CB
:101AB80043EB020008BF20EADC7070474FEA40029F
:101AC800B2F1FE4F0FD34FF09E03B3EB12620DD964
:101AD8004FEA002343F0004310F0004F23FA02F0CE
:101AE80018BF404270474FF00000704712F1610F75
:101AF80001D1420205D110F0004008BF6FF000404C
:101B080070474FF00000704753B94AB9002908BF21
:101B180000281CBF4FF0FF314FF0FF3000F070B9C4
:101B2800ADF1080C6DE904CE00F006F8DDF804E02C
:101B3800DDE9022304B070472DE9F047089E0D4601
:101B480004460F46002B4AD18A42944665D9B2FA18
:101B580082F343B102FA03FCC3F120029F4020FA4A
:101B680002F217439C404FEA1C4E1FFA8CF5B7FB54
:101B7800FEF1220C0EFB117742EA074201FB05F049
:101B880090420AD91CEB020201F1FF3780F01B8159
:101B9800904240F2188102396244121AA4B2B2FB90
:101BA800FEF00EFB102244EA024400FB05F5A542B4
:101BB8000AD91CEB040400F1FF3280F00681A5422B
:101BC80040F203816444023840EA0140641B00216A
:101BD8001EB1DC400023C6E90043BDE8F0878B4214
:101BE80008D9002E00F0EC800021C6E9000508465F
:101BF800BDE8F087B3FA83F1002949D1AB4202D39B
:101C0800824200F2F780841A65EB0302012017462E
:101C1800002EE2D0C6E90047DFE702B9FFDEB2FADC
:101C280082F3002B40F08F808A1A4FEA1C471FFA74
:101C38008CFE0121B2FBF7F507FB1520220C42EAC6
:101C480000420EFB05F0904208D91CEB020205F198
:101C5800FF3802D2904200F2CA804546121AA4B256
:101C6800B2FBF7F007FB102244EA02440EFB00FE29
:101C7800A64508D91CEB040400F1FF3202D2A645A0
:101C880000F2BA801046A4EB0E0440EA05409FE734
:101C9800C1F120078B4022FA07FC4CEA030C05FA35
:101CA80001F420FA07F3FD40234300FA01F94FEA53
:101CB8001C401FFA8CFEB5FBF0F81C0C00FB1855F5
:101CC80044EA054408FB0EF5A54202FA01F20BD9D5
:101CD8001CEB040408F1FF3A80F08780A54240F22B
:101CE8008480A8F102086444641B9DB2B4FBF0F33D
:101CF80000FB134445EA044403FB0EFEA64508D93D
:101D08001CEB040403F1FF306BD2A64569D9023BF2
:101D1800644443EA0840A0FB0283A4EB0E049C42FF
:101D2800C6461D4655D352D056B1B9EB0E0364EBE7
:101D3800050404FA07F7CB40CC401F43C6E90074FA
:101D48000021BDE8F087C3F1200102FA03FC20FA64
:101D580001F225FA01F19D402A434FEA1C471FFA78
:101D68008CFEB1FBF7F007FB1015110C41EA054199
:101D780000FB0EF58D4204FA03F408D91CEB0101AF
:101D880000F1FF382FD28D422DD902386144491B0A
:101D980092B2B1FBF7F507FB151142EA014205FBC8
:101DA8000EF1914208D91CEB020205F1FF3816D258
:101DB800914214D9023D6244521A45EA004139E77A
:101DC8003146304609E73946E7E61046FCE6C145A4
:101DD800AAD2B8EB020E63EB0C050138A4E745461E
:101DE800EAE7034695E74046D1E7D0467CE7023D5F
:101DF800624433E708460BE76444023843E700BF10
:101E0800704700BF1348144A08B54FF00043C0E9B3
:101E180000230422002342610122C2614FF4805151
:101E280007220383C0E90233C0E90933C0E90C1271
:101E38000361837680F8203080F82C30826380F844
:101E48003C30C36404F0BEFF18B1BDE8084000F0A0
:101E58002DBC08BDDC080020002401400268084BA6
:101E68009A4282B00AD14FF0B0431A6E42F400721F
:101E78001A661B6E03F400730193019B02B070474E
:101E8800002401400268054B9A4201BF4FF0B0425E
:101E9800136E23F400731366704700BF00240140DB
:101EA80030B585B000240546CDE901440394FFF719
:101EB800A9FF144805F01EFB08B100F0F7FB114814
:101EC800039401A9CDE9015405F0DAF808B100F04E
:101ED800EDFB0C4805F038FA08B100F0E7FB4FF0CD
:101EE800FF31084805F06EF8064805F0E5FA0548A0
:101EF80005F0C2F80446034805F088FA204605B004
:101F080030BD00BFDC080020014B024A1A60704750
:101F1800DC0800200024014008B50948FFF7C0FF8D
:101F280068B1084BB3F8AA304FF6FF72934216BF58
:101F380040F6E442044B5343B3FBF0F398B208BDB8
:101F4800002000B40075FF1FD8084C0013B500230B
:101F5800ADF80630FFF7E0FF04461948FFF7A0FF89
:101F6800184BB3F8C820B3F8A8108A4204FB00F055
:101F780018D040F6E443B0FBF3F364205B1A434304
:101F8800521A93FBF2F31E331BB2ADF80630BDF8BC
:101F980006305BB21B02ADF80630BDF8060000B291
:101FA80002B010BD4FF47A7240F6FF73B0FBF3F342
:101FB8005343A3F53923A3F50C6340F6C412E0E7B5
:101FC800001000B00075FF1F4FF0B04382B09A6A4E
:101FD80022F480529A629A6C42F480529A649B6C02
:101FE80003F480530193019B002002B070474FF027
:101FF800B04382B09A6C02439A649B6C034001938D
:10200800019B02B0704708B50420FFF7F0FF0120DC
:10201800FFF7EDFF0220FFF7EAFF002211460B2031
:1020280005F006FB0B2005F035FB002211460C20BD
:1020380005F0FEFA0C2005F02DFB002211460D20BC
:1020480005F0F6FA0D2005F025FB002211460E20BA
:1020580005F0EEFA0E2005F01DFB002211460F20B8
:1020680005F0E6FA0F2005F015FB002211461020B6
:1020780005F0DEFA102005F00DFB002211461120B4
:1020880005F0D6FA112005F005FB0022362011468E
:1020980005F0CEFABDE80840362005F0FBBA00008E
:1020A80008B505F03FFD10B16FF0040008BD064B00
:1020B8009A6942F040429A614CF2FA321A6105F08C
:1020C80043FD0028F2D0EFE700400058F0B585B096
:1020D80000230C4600930646A8B3FFF7E1FF054628
:1020E80070BB05F01FFD88BB1A481B4A02230193E9
:1020F800D0F8E01506F1784302EA8121B3FBF1F745
:1021080001FB1733DB0A0293D0F8E00504F17841AC
:102118000139314402EA8022B1FBF2F002FB1011CE
:10212800C3EBD1230133694601A8039305F08CFD65
:1021380020B102280CBF01256FF0010505F004FD50
:10214800284605B0F0BD6FF00505F9E76FF0040506
:10215800F6E700BF0070FF1F00FCFF03014B18608B
:1021680000207047400900202DE9F04F89B0B0F1F8
:10217800006F06460F460092C0F0C580DFF89881D0
:10218800664DD8F8E03505EA832303F10063013B87
:10219800984200F2B880002800F0B880002900F0CA
:1021A800B58040EA02035B0740F0B080FFF778FF94
:1021B8000446A0BB05F0B6FC002840F0AA80D8F879
:1021C800E01506F1784205EA8121B2FBF1F301FB43
:1021D8001322009B03F17843013B3344B3FBF1F036
:1021E80001FB1033DB0A01334FEAD22AA3EBD222D8
:1021F800012A039388BFC6F30A050AF58038C6F199
:10220800080398BF009D069388BFC5F500654FEA8F
:10221800C828B346039B9A4505D305F095FC20468C
:1022280009B0BDE8F08FA6F10803069A1A44954252
:1022380019D804950197CDF814B04FF00009059B03
:1022480009EB0301049B99453ED3009BAB442F4403
:102258005D1BB5F5006F28BF4FF400650AF1010A50
:1022680008F50068D6E753F8081F5A68B2F1FF3F2F
:1022780008BFB1F1FF3FD8D0294B186810B96FF0EB
:102288000504CAE7B8F1000F04D04FF400624146D4
:1022980011F0D8F9DFF88890D9F80030CBF30A00AC
:1022A80039461844AAB211F0CDF94FF400614046FE
:1022B800FFF70CFF08BBD9F8003001934FF4006317
:1022C800CDF814800493B8E7019B07914B4402931F
:1022D8000120D3E9002305F071FC88B90799019B17
:1022E800D1E9000259F80310029B5B689A4208BFC3
:1022F800884205D109F10809A1E76FF001048CE7CC
:102308006FF0030489E74FF0FF3488E76FF00504A6
:1023180085E76FF0040482E70070FF1F00FCFF03ED
:1023280040090020B1F1006F70B511D30B4BD3F801
:10233800E0650B4B03EA862303F10063013B9942F6
:1023480006D840B139B192B211F07CF9002070BDC5
:102358004FF0FF30FBE76FF00500F8E70070FF1F54
:1023680000FCFF03B0F1006F10B40DD3084BD3F895
:10237800E045084B03EA842303F10063013B9842DC
:1023880002D810BCFFF7A2BE4FF0FF3010BC704758
:102398000070FF1F00FCFF034FF0B04382B0DA6CFF
:1023A8000243DA64DB6C03400193019B02B070477F
:1023B8002DE9F04186B01422002101A811F07AFD20
:1023C80001203B4EFFF7E8FF0220FFF7E5FF04205E
:1023D800FFF7E2FF08210122304605F0A9FD01259B
:1023E8004FF40417022301A94FF09040CDE90137BB
:1023F800039505F077FC4FF4441301A94FF0904082
:102408000024CDE902354FF02008019505F06AFC5B
:1024180001A93046CDE90187039405F063FC01A9C1
:102428003046CDE90187039405F05CFC082301A937
:102438003046CDE90135CDE9035405F053FC4FF49E
:10244800007301A94FF09040CDE90135CDE903545F
:1024580005F048FC04230DEB03013046CDE90135B6
:10246800CDE9034405F03EFC22462146062005F04E
:10247800DFF8062005F00EF922462146072005F070
:10248800D7F8072005F006F922462146162005F060
:10249800CFF8162005F0FEF822462146162005F052
:1024A800C7F8162005F0F6F806B0BDE8F08100BFC1
:1024B8000004004808B51248124A134BC0E900232B
:1024C80000230122C0E90232C0E90433C0E906331F
:1024D800036205F0A1FE08B100F0E8F80848002101
:1024E80006F01AF808B100F0E1F80548002106F0F6
:1024F80039F818B1BDE8084000F0D8B808BD00BFE9
:10250800040A0020005800405D3E302070B596B0A7
:1025180005461422002103A811F0CCFC3822002122
:1025280008A811F0C7FC2A68304B9A425BD1802377
:10253800089308A84FF440230E9306F06FFD08B1E6
:1025480000F0B4F84FF0B0444FF4C050E36C43F0DF
:102558000103E364E36C03F001030293029B12237B
:102568000026CDE903030323CDE905634FF090402E
:10257800042303A9079305F0B5FBA36DDFF870C02A
:1025880043F48003A365A36D1A4C03F480030193FD
:10259800019B26620D23C4E900C320468023C4E9B9
:1025A8000266C4E90436C4E9066605F0D3F808B142
:1025B80000F07CF8104AEC63A562104C0E23C4E9C5
:1025C80000231021002380222046C4E90213C4E915
:1025D8000423C4E90633236205F0BCF808B100F00F
:1025E80065F8AC63A56216B070BD00BF0058004026
:1025F800440002404409002058000240A409002079
:1026080000B59BB04822002108A811F053FC1822FD
:10261800002102A811F04EFC05F0CAFF4FF0B042AD
:102628000120D2F8903023F01803C2F89030D2F885
:10263800003423F4C06343F40073C2F80034D2F8C2
:10264800003403F4C0630193019B2423089381237E
:102658000B930023CDE91003B02208A8CDE912237B
:1026680006F01EF908B172B6FEE74F23CDE9023035
:10267800CDE90400CDE90600022102A806F0AAFB74
:1026880008B172B6FEE71BB05DF804FB08B504F0AC
:1026980047FBFFF7B5FFFFF78BFEFFF7B4FCFFF72B
:1026A80009FF00F0BAFD00F0BFFDFCE772B6FEE7D7
:1026B80000B58DB02C22002101A811F0FBFB1748B2
:1026C800174B03601F2383604FF080420023C0E94B
:1026D8000433C0E9072383614FF48073436206F033
:1026E80023FE08B1FFF7E2FF0C4806F049FF08B1E6
:1026F800FFF7DCFF4FF000530022079307480892CA
:102708004FF4807301A9029206920B9306F06CFEB7
:1027180008B1FFF7CBFF0DB05DF804FB580A0020A5
:102728000028004010B5044690B03822002102A8C5
:1027380011F0C0FB2268194B9A422CD14FF4803318
:10274800029302A84FF480730F9306F067FC08B158
:10275800FFF7ACFF4FF0B0430220D3F8902042F4CB
:102768000042C3F890209A6D42F480629A659B6D8E
:10277800002203F4806311460193019B04F058FF83
:10278800022004F087FF00222A20114604F050FF9F
:102798002A2004F07FFF10B010BD00BF00280040C1
:1027A8007047000008B504F0D1FA044B0120C3F8C3
:1027B8008800BDE8084005F053BF00BF000400587A
:1027C80004F0CBBA08B504F0C8FA00F059FCFFF7DA
:1027D800EFFDFFF718FCBDE80840FFF76BBE08B532
:1027E80004F0B4FABDE808400121002005F0E8BE75
:1027F80070477047FEE7FEE7FEE7FEE7FEE7704733
:102808007047704770470000014806F0DFBE00BF00
:10281800580A0020012005F091BB022005F08EBB6C
:1028280070477047014805F00FB900BF4409002000
:10283800014805F009B900BF300B0020014805F038
:1028480003B900BFD00A0020FFF7F2BF704720206D
:1028580005F074BB70470000014807F07BBA00BF61
:10286800900B0020014806F0E3BC00BF580A002086
:10287800014807F0D6B800BFBC0A00202DE9F04394
:1028880089B080460020109E0790894615461F464D
:10289800FDF7C6FCF0B9104CCDE90090CDE9020473
:1028A80007AB0E480593142304933A46434629463A
:1028B8000068FDF77FFD2346324604F1140153F802
:1028C800044B42F8044B8B42F9D1079B337509B08E
:1028D800BDE8F0830120FAE7900A0020EC400108E7
:1028E8001FB50E4C00233C2202A8CDE902336275C5
:1028F800237500F0B9F8042303AA009412210848AC
:10290800FFF7BCFF07491422204611F0C3FAB0FABA
:1029180080F35B09637504B010BD00BFA40A0020F2
:10292800144101083E0E0020054808B5082303603D
:1029380006F092FE18B1BDE80840FFF7B7BE08BD23
:10294800BC0A00204FF0B04307B55A6E42F00102AE
:102958005A665B6E002203F0010301931146322090
:10296800019B04F065FE322003B05DF804EB04F02F
:1029780091BE00000CB407B5054A05AB10210193C0
:1029880011F06AF903B05DF804EB02B0704700BFBC
:102998002641010830B585B0044602A80D4610F05E
:1029A80087FFBDF90C30064A00931021029B204690
:1029B800FFF7E0FF2046FEF7FFFC288005B030BD9A
:1029C800264101084FF0B04210B5936823F4004344
:1029D800936010F0F5FF0E4B01241C7000F0B6F860
:1029E80010F0BEFC0B4810F0D5FC0B4B4FF4004226
:1029F8001A61002010F0D4FCFFF786FA00F012F9F3
:102A080010F0CAFD21462046BDE8104010F0E4BD94
:102A1800C80A00209D2900080040005810F0F2BDA7
:102A280008B5FFF779FA40F6B83398420CD8B0F5F4
:102A3800E16F0BD3FE23A0F5E16058434FF4966392
:102A4800B0FBF3F0C0B208BDFE20FCE70020FAE7B7
:102A58007FB5684600F0CAF80198FFF72FF800B272
:102A680007B05DF804FB0000194A38B5D2F8803584
:102A7800591C044619D104F077F9054604F080F989
:102A8800054404F077F92B0EE3712B0CA3712B0A84
:102A98006371030EE370C0F30742C0F30723257187
:102AA800C0B2A2706370207038BD190AC3718171F9
:102AB800190C1B0E41710371D2F88435C370D2F81A
:102AC8008405C0F30722C0F30743000EE9E700BFFF
:102AD8000070FF1F38B5094BD3F880350360013308
:102AE800054609D104F040F9044604F043F944408E
:102AF80004F046F944402C6038BD00BF0070FF1F49
:102B08000121022010F052BD0021022010F04EBD1C
:102B180000207047024B187808B100F0BBB8704726
:102B2800C80A002082B00190019802B000F04EB9A6
:102B38004FF0B04382B0DA6C42F00202DA64DB6C28
:102B480003F002030193019B02B070472DE9F043A3
:102B5800254C87B004F01AF904F020F904F026F99E
:102B68000123002502934FF48059032301A920462D
:102B780004934FF4005803950595FFF7D9FFFFF725
:102B8800D7FFFFF7D5FFFFF7D3FFCDF8049005F087
:102B9800A9F801A920464FF40067CDF8048005F094
:102BA800A1F801A920464FF40046019705F09AF8CC
:102BB80001A92046019605F095F82A46494620467F
:102BC80005F0B6F92A464146204605F0B1F92A46ED
:102BD8003946204605F0ACF92A463146204605F02C
:102BE800A7F907B0BDE8F0830004004810B5044613
:102BF800FFF7ACF9074BA36040F30F20FEF70AFF7D
:102C0800054B064A2360064B6060C4E90323002095
:102C180010BD00BF0000484200007A440D093E0084
:102C2800AB03050000207047014B1868704700BFD0
:102C3800CC0A00200320704708B501464FF47A7289
:102C480000238002890DFEF75FFF08BD4FF47A73F9
:102C5800A0FB0303800A40EA83507047034B98683F
:102C68009A689042FBD1C043704700BF00280040DB
:102C780008B5FFF7F3FF014B186008BDCC0A002028
:102C880008B5FFF7EBFF024B1B68C01A08BD00BF71
:102C9800CC0A0020024B187808B1FFF7DFBF704755
:102CA800C90A002010B5074B074C0122DA654FF41A
:102CB8008071204606F082FA4FF0FF33236300202C
:102CC80010BD00BF00280040580A0020024600211D
:102CD800014806F08CBC00BF580A002002460121BA
:102CE800014806F084BC00BF580A002010B58CB01B
:102CF8002C220021044601A811F0DCF8FFF7D2FFCE
:102D08000C4B0D481B681C440023089306934FF096
:102D18000053E443079301224FF4807301A90294FE
:102D28000B9306F061FB08B1FFF7C0FC00200CB064
:102D380010BD00BFCC0A0020580A002038B505464F
:102D4800FFF78CFF02210446074806F057FCC4F33E
:102D580009024FF47A71A2FB0121920AA30A2A8080
:102D680043EA805038BD00BF580A002001480021BE
:102D780006F044BC580A00200148012106F03EBC78
:102D8800580A0020F8B50F4D2E78CEB90E4C4FF0EA
:102D9800FF372763FFF78CFCFFF784FF4FF4807140
:102DA800204606F00BFA2046276306F0CBFB324696
:102DB8002046022106F01BFCFFF75AFF01232B7067
:102DC8000020F8BDC90A0020580A0020014610B5A5
:102DD8004FF47A7200238002890DFEF795FE0146B2
:102DE800FFF73CFF0446FFF739FF031B8B4200D374
:102DF80010BD00BFF7E710F0EBBE000010B5064CA1
:102E08000221204606F0FAFB0221421C2046BDE8BA
:102E1800104006F0ECBB00BF580A00201648174ABD
:102E280008B54FF4E133C0E9002300230C22C0E9C0
:102E38000233C0E90523C0E90733C0E90933036158
:102E480007F069FD08B1FFF731FC0B48002107F0D6
:102E5800DEFE08B1FFF72AFC0748002107F0F7FE5D
:102E680008B1FFF723FC044807F0B1FE18B1BDE82C
:102E78000840FFF71BBC08BD900B00200044004031
:102E880070B596B005461422002103A811F012F877
:102E98003822002108A811F00DF82A68334B9A420D
:102EA80061D10223089308A8314B0A9306F0B6F8BB
:102EB80008B1FFF7FBFB4FF0B0430C219A6D2D4C86
:102EC80042F400329A659A6D02F400320292029A34
:102ED800DA6C42F00102DA64DB6C03F0010301935F
:102EE800019B02230026CDE903130323CDE90563E3
:102EF8004FF09040072303A9079304F0F3FE1E4800
:102F080026621423C4E900031023C4E902362046CC
:102F18008023C4E90436C4E9066604F01BFC08B142
:102F2800FFF7C4FB154AEC67A562154C1323C4E9E7
:102F38000023204600238022C4E90233C4E9042385
:102F4800C4E90633236204F005FC08B1FFF7AEFBC1
:102F58002520C5F8804000220221A56204F068FB04
:102F6800252004F097FB16B070BD00BF0044004058
:102F780004000C00300B0020800002406C0002406E
:102F8800D00A002002680E4B9A4210B5044616D1AA
:102F98004FF0B0420C21936D23F4003393654FF04A
:102FA800904004F04BFFE06F04F048FCD4F8800038
:102FB80004F044FCBDE81040252004F079BB10BDA6
:102FC8000044004008B50A460146024806F026FEBD
:102FD800002008BD900B002013B5114B114C186050
:102FE8004FF40013009302AB13E90600204607F0E4
:102FF80092FD2368DA69D103FCD4DA695202FCD560
:103008009A68084842F480029A6007F0CAFD0649A7
:103018000448012207F038FD002002B010BD00BFAF
:10302800240C0020900B00202C0C002008B5074B26
:103038001860FEF7E8FFFFF7F1FE054AD2F8803086
:1030480043F00063C2F88030002008BD280C00203F
:103058000008005808B54FF0B04308489A6B42F48E
:1030680000329A639A6B22F400329A63FFF78AFF60
:103078000F2004F01DFB002008BD00BF900B0020AE
:1030880008B5074807F047FC08B1FFF70FFB0548EC
:1030980004F060FB18B1BDE80840FFF707BB08BDA6
:1030A800900B0020300B00200268044B9A4203D199
:1030B800034B00201B681847704700BF00440040BE
:1030C800280C002002680B4B9A4210B504460FD119
:1030D800094B1B682BB1D0F8902012B90748012181
:1030E800984720460549BDE81040012207F0CCBCAE
:1030F80010BD00BF00440040240C00202C0C002010
:1031080002480122102104F013BF00BF0004004848
:1031180002480022102104F00BBF00BF0004004841
:1031280010B50A4C23780BB9E37C6BB1FFF7D8FBD9
:103138000038074B18BF0120400018701B78022B7D
:1031480002BF00232370E37410BD00BF3E0E0020B1
:10315800340C002038B5114C2378F3B9E37CE3B97B
:103168000F4D2B68012B07D92B68042B04D80D4A67
:103178000421012000F024FA2B68042B0DD9FFF755
:10318800AFFB0038084B18BF0120400018701B78AF
:10319800022B02BF00232370E37438BD3E0E0020CB
:1031A800300C002080410108340C002008B5FFF7DE
:1031B800A7FF01F011FABDE80840FFF7A9BF0228F0
:1031C80001D8FFF79DBF7047022801D8FFF7A0BFBD
:1031D80070470000022808B51BD8012210210D48AD
:1031E80004F0A6FE3220FFF79DFC0A4800221021B9
:1031F80004F09EFE01221021064804F099FE3220B8
:10320800FFF790FCBDE8084002480022102104F0B6
:103218008FBE08BD00040048704708B5FFF7D2FB11
:10322800BDE8084000F06ABB4FF0FF3010F04EBA1E
:103238007047704770470000014BD870704700BF57
:103248005C000020014B1874704700BF5C00002030
:1032580020B1037813B1024810F068BC704700BF72
:10326800740D002008B50220002110F0F7F9BDE820
:103278000840014810F05ABC8C0D002000210120A4
:1032880010F0ECB910B5094C60B12060084810F096
:10329800FFFB2168064810F083FCBDE81040044895
:1032A80010F044BC42F210732360EFE77400002072
:1032B8008C0D002010B5094C206023680BB9084B11
:1032C8002360084810F0E4FB2168064810F068FC09
:1032D800BDE81040034810F029BC00BF0C000020D6
:1032E800A0860100A40D002010B5044680B190F915
:1032F80006306BB9094810F0CBFB094BE2791A701C
:10330800084B1868FFF7D6FF074B1868FFF7BAFF96
:10331800BDE810400021022010F0A0B9280D0020BF
:10332800580D00200C0000207400002038B5044619
:103338000D4607484FF40061FFF714F830B92A46E4
:1033480021460348BDE83840FEF70EBF38BD00BF30
:1033580000F003080A460149FEF7E4BF00F003083D
:1033680038B50C4810F094FB08F0D6F860B90A4C50
:103378000A480125257007F061FF2078294607F0E3
:10338800B3FC044810F0D2FBBDE83840044810F004
:10339800CDBB00BF8C0D0020000000205C00002089
:1033A8005C0D002008F054B930B585B0FFF738FB44
:1033B800044607F08FFD054680B100243C4810F014
:1033C80067FB3C4B3A481968A14238BF214610F0C8
:1033D800E7FB374810F0AAFB05B030BD01464FF4B3
:1033E800807010F03BF9684600F0D8FF23B203EB79
:1033F8004303FE2203EB4313B3FBF2F32E4A3921B6
:1034080011702E4950680978DBB28DF80C300170C4
:103418005068457050682724847050680124C4702F
:1034280050680371264B187840B11D70536861F0DD
:103438007F0119703A23137005231CE0214B2248A1
:10344800197811B901780029F6D000210170197096
:10345800536804215971BDF800305168180A887101
:103468005168CB71BDF8083051681B0A0B72BDF862
:1034780008304B720A231549154C0978012988BF71
:1034880000235370637A33B107F010FD012802D18D
:10349800204610F0FDFA0F4B0748D978002207F0B4
:1034A8002FFD063089D107F0FBFC044686E700BFF4
:1034B8008C0D00207400002004000020270D00203F
:1034C800BC0D0020530E00203D0E0020340C0020BF
:1034D800280D00205C00002008B5104B01220021B7
:1034E80002201A7010F0BAF80D4810F01FFB0D4BAF
:1034F8001B788BB10C4B1A7872B9DB7C63B90B4B18
:103508001A68042A9EBF1A6801321A600021BDE8B1
:103518000840102010F0A2B808BD00BFBC0D002064
:10352800A40D0020580D00203E0E0020300C002075
:10353800044B1B78022B03D10021082010F08EB811
:10354800704700BF0000002008B507F0EEFF80B903
:1035580007F0ACFC01280CD1BFF34F8F0549064B8F
:10356800CA6802F4E0621343CB60BFF34F8F00BF19
:10357800FDE708BD00ED00E00400FA05704770475C
:1035880070477047022808B501460FD0202810D090
:10359800012811D14FF0904004F0C4FC01280BD150
:1035A80000210220BDE8084010F058B8002108208A
:1035B800F8E7024B01221A7008BD00BFB80E0020C0
:1035C80070B505460C46164607F084FC03460028ED
:1035D80034D000241A4810F05BFA1A4B18481968BE
:1035E800A14238BF214610F0DBFABDE8704014480C
:1035F80010F09CBA4A68F05CD0540133DAB29442B5
:10360800F8D8114B0D701B78012B88BF00244C7023
:103618000E4C637A33B107F049FC012802D12046E9
:1036280010F036FA0A4B0B48D978002207F068FCEC
:103638000630CED107F034FC0446CBE70549DDE778
:103648008C0D002074000020340C0020280D002070
:103658005C00002004000020044B1B7823B9044AB6
:1036680005210120FFF7ACBF704700BF340C0020D4
:103678008541010810B5002490B03C22214601A8DC
:10368800009410F017FC2F4B2022DA7219788DF86D
:10369800001059788DF8011099788DF80210D978B2
:1036A8008DF8031019798DF8041059798DF80510E3
:1036B80099798DF80610D9798DF80710197A8DF84F
:1036C8000810597A8DF80910997A8DF80A108DF832
:1036D8000B2021460DF10B0258180131007B02F82E
:1036E800010F1C29F8D193F828208DF8282093F889
:1036F80029208DF8292093F82A208DF82A2093F87C
:103708002B208DF82B2093F82C206AB193F83F20BA
:1037180052B10DF12B0100229818013290F82C00BB
:1037280001F8010F142AF7D107484FF40061FEF79A
:1037380019FE20B9044840226946FEF715FD10B06D
:1037480010BD00BF7800002000F80308014940229E
:103758000FF078BF00F8030870B52A4D28796B7907
:103768004D2BC0B233D1C0EB001080000A2838BFFF
:103778000A204FF47A735843234BAC791860EB79DD
:103788004D2BE4B22BD1C4EB0414A40095F82C30D3
:103798001E4E63BB95F83F304BBB42F21070FFF7EB
:1037A80071FD3068FFF786FD2B7A194A1949DBB29B
:1037B80013706B7A184ADBB213700023EA1892F878
:1037C8002C20D2B2CA540133142BF7D170BD6B79B7
:1037D800482B0ABF4FF461636B795843C6E7EB790E
:1037E800482B0ABF4FF46163EB795C43CEE7FFF7E0
:1037F80049FD012C38BF01244FF47A735C433460CF
:10380800CFE700BF78000020740000200C000020E3
:10381800520E00203E0E0020340C002010B590B04F
:1038280000213C2201A8009110F044FB40223149BC
:1038380068460FF007FF9DF800203AB99DF801008F
:10384800272803D19DF80210012909D0FFF712FF9C
:103858004FF47A70FFF766F9FFF77EFF10B010BDDE
:10386800254B1A70587099709DF80310D9709DF8FF
:10387800041019719DF8051059719DF80610997179
:103888009DF80710D9719DF8081019729DF8091054
:1038980059729DF80A1099729DF80B1001F03F01BA
:1038A800D972D87AD1B288421BD89DF8282083F8DB
:1038B80028209DF8292083F829209DF82A2083F8BC
:1038C8002A209DF82B2083F82B200DF12B010022B4
:1038D8009818013211F8014F80F82C40142AF7D1BA
:1038E800BAE701F140006844194410F8340C087331
:1038F8000132D6E700F80308780000201FB500243D
:1039080003A92046039407F0F3FD03A9012007F05B
:10391800EFFD384B3848009422464FF4FA7110F006
:1039280059F8364B3648009422464FF4FA7110F095
:1039380051F8344B3448009401224FF4FA7110F0D6
:1039480049F82046FEF70AFC08B1FEF7AFFE2F4BF8
:10395800009400224FF4FA612D4810F03BF82D4AEC
:10396800002101200FF036FF2B4A002102200FF022
:1039780031FF2A4A002104200FF02CFF284A002199
:1039880008200FF027FF00F085FB2649264807F09E
:1039980065FD264807F052FC1B4810F0C7F8244B79
:1039A8000021187807F0A0F922490094224B0968F1
:1039B8002248002210F00EF8204810F0B7F8FFF760
:1039C8002DFF1F4A002110200FF004FF1D4A00217F
:1039D8004FF480700FF0FEFE1B4B1C4819681C4BFF
:1039E800009400220FF0F6FF184810F09FF804B07A
:1039F80010BD00BF89350008740D00208B35000804
:103A0800400D002085350008280D002039350008B4
:103A18005C0D00203DB00008B1330008AD3300084C
:103A28006933000800000301100000205C0000203A
:103A380000000020740000206D3200088C0D00206A
:103A48005D310008B53100080C000020A40D0020ED
:103A5800E134000810B50024A2B07C22214603A856
:103A6800029410F027FA53238DF8083040F22713F8
:103A7800ADF80A3001238DF80C30ADF80440FEF79C
:103A8800CFFF00B200EB400000EB4010FE23B0FB7C
:103A9800F3F08DF80D0001A800F090FCA0B95823B0
:103AA8008DF80E30072430228021144810F002FAD5
:103AB800224602A9114810F036FA104A2146012080
:103AC800FFF77EFD22B010BD430001338DF80E30A4
:103AD8008DF80F0000F080FD094B1A6812128DF85E
:103AE80010201A688DF811205A685B688DF8133019
:103AF80012128DF812200C24D5E700BFBD0D00204E
:103B0800E40E002030B50378592B91B0044640F0FC
:103B1800F481052959D84378443B162B55D8DFE85A
:103B280013F032015400220154002A0154005400B9
:103B380054005400940054000D01540054005400E3
:103B48009B0154005400B000540054005400170066
:103B58008578482D11D1B74A14210120FFF730FD8F
:103B680041F28830FEF7DEFF40F6B830FEF7DAFFA4
:103B780011B0BDE83040FFF7E7BC532D0ED130221D
:103B88008021AD4810F096F9FFF764FF41F28830C4
:103B9800FEF7C8FFA84A1521012087E0432D16D15A
:103BA800002468468DF8004007F0C0FAA24A4C236A
:103BB8001370272393709DF800305470012041330F
:103BC800D07013710521FFF7FBFC11B030BD442DF7
:103BD800FBD1994C592323705A236370A57000F0C8
:103BE800CFFB2C228021201D10F064F900232570C2
:103BF800637001252723A370E5702571FEF710FF78
:103C08008E49FE23B0FBF3F00B6864229BB2B3FB32
:103C1800F2F3A3710B6800EB400000EB40109BB27D
:103C28006071B3FBF2F002FB1033E3714B689BB297
:103C3800B3FBF2F323724B689BB2B3FBF2F102FBC6
:103C48001133637222460A21A6E78378303BDBB240
:103C5800092BBAD87A497B4A0B700B78DBB25372BE
:103C6800754A592313704D2353700B783033937072
:103C780003210120FFF7A4FC11B0BDE83040FFF795
:103C8800F9BC8578482D16D16B4A5623137000234A
:103C980053702723937003231371172353710B2336
:103CA800012093711223D070D371082111B0BDE89F
:103CB8003040FFF785BC432D87D15F4C00213C2263
:103CC80001A8009110F0F6F86846FFF73FFD24229E
:103CD800802104F10C0010F0EDF89DF800306370BD
:103CE8009DF80130A3709DF80230E3709DF8033011
:103CF80023719DF8043063719DF80530A3719DF818
:103D08000630E3719DF8073023729DF8083025705E
:103D180063729DF80B509DF80930A3729DF80A3024
:103D2800E3722A4603A9257304F10D0010F0FBF88D
:103D380005F10D012246C9B2012044E780783928EF
:103D48000CD83038C0B2FFF73AFA3B4A23781370E0
:103D580063785370A378937003211DE711B0BDE811
:103D68003040FFF779BC80783928F7D83038C0B2AE
:103D7800FFF72AFAE9E780783928EFD83038C0B257
:103D8800FFF728FAE1E78378303BDAB2092AE5D869
:103D9800C0783038C2B2092AE0D82179A1F14802A6
:103DA800D2B20B2ADAD8284D45FA02F2D507D5D473
:103DB8000A224D2902FB030036D13C2358434FF415
:103DC8007A735843214B1860214B1860FFF75AFA51
:103DD800194A2378137063785370A3789370E37843
:103DE800D3702379137105210120FFF7E9FB154BE7
:103DF80000221A7027225A7001229A70DA70A2786B
:103E0800303A02EB8201E278303A02EB4102D2B258
:103E18001A7122795A710F4A1278D2B21A72084A64
:103E28001278D2B25A7227E74829C8D14FF4616391
:103E3800C4E700BF8B410108BD0D0020E40E00203F
:103E4800340C002078000020DEF7FFFF740000200B
:103E58000C000020520E00208278303AD3B2092B91
:103E68003FF67CAFC378303BD9B209293FF676AF2D
:103E78000079A0F14801C9B20B293FF66FAF624D36
:103E880045FA01F1C9073FF569AF0A214D2801FB41
:103E980002332DD13C2253434FF47A7253435B4A89
:103EA80013601068FFF706FA594A2378137063788D
:103EB8005370A3789370E378D37023791371052135
:103EC8000120FFF77DFB534B00221A7027225A70FE
:103ED80001229A70DA70A278303A02EB8201E27815
:103EE800303A02EB4102D2B29A712279DA7192E742
:103EF8004828D1D14FF46162CDE7502B48D102292F
:103F08007FF663AE4378303B012B3FF65EAE837895
:103F1800312B7FF45AAE0B2904D8FFF79DFB002103
:103F28003B4A39E63B4D0234002214F8013FA918F8
:103F3800303B0132DBB20C2A0B73F6D1FFF76CF978
:103F4800334B502227211A709970002201215A7090
:103F5800D97003F8041FA9180132097B0C2A01F152
:103F6800300103F8011FF6D100232B7027236B7053
:103F78000123AB70EB70284B1B78DBB22B72274BFD
:103F88001B78DBB26B72EA72FFF774FB1121C7E78B
:103F9800412B7FF41AAE4378432B7FF416AE1629D3
:103FA8007FF413AE1E4D421C002312F8011FE95482
:103FB8000133142BF9D1FFF7B3F81A4B5B7D012BB2
:103FC80019D114490023EA5CC8180133D2B2142B62
:103FD80080F82C20F7D1114B00221A701B78DBB225
:103FE8004B72FFF747FB0A4A631E1534A34206D1FA
:103FF800074A1621D0E5094B02221A70F3E713F895
:10400800011F02F8011BF1E7DEF7FFFF0C0000209B
:10401800BD0D002078000020520E0020340C002036
:104028003E0E0020A40A002038B504460D4661B3B0
:1040380016480FF07BFD2B783BB334B360682378C8
:1040480018B3032B0CD0392B17D0022B1DD1617854
:1040580001291AD00B0618D4BDE83840FFF752BD25
:104068006378012B11D10078012802D0022800D0F2
:1040780058B9BDE8384007F00FB86378012B04D170
:104088000378034A03F00103137038BD400D002084
:10409800270D0020034B0022C3E902220122C3E9B5
:1040A80000227047540E002000487047540E00202C
:1040B8004FF0B04382B0DA6C0243DA64DB6C034041
:1040C8000193019B02B070472DE9F04186B00024AE
:1040D8000220154D0594FFF7EBFF0420FFF7E8FFDA
:1040E800124F03944FF4807601230DEB0001CDE9C4
:1040F80001632846032304934FF4005803F0F2FDAC
:1041080001A93846CDF8048003F0ECFD224641466B
:10411800384603F00DFF28462246314603F008FFD3
:10412800204606B0BDE8F0810004004800080048B9
:10413800032810B50ED8012810D868B902460B48D4
:104148004FF4807103F0F4FE002209484FF4005147
:1041580003F0EEFE002010BD0122F0E70022034824
:104168004FF4807103F0E4FE0122EEE700040048FA
:10417800000800480220704700207047012070475F
:1041880000280CBF0F201620704700000D488546F8
:1041980002F0C4FD0C480D490D4A002302E0D45832
:1041A800C4500433C4188C42F9D30A4A0A4C002379
:1041B80001E013600432A242FBD30FF083FEFEF746
:1041C80065FAFEE70000012000000020BC0800207E
:1041D800B84C0108BC080020BC2C0020FEE74FF0BA
:1041E800B04382B0DA6C42F00102DA64DB6C03F0AF
:1041F80001030193019B02B07047000030B587B0FE
:10420800FFF7EDFF4FF4805101224FF0904003F08B
:104218008FFE01224FF400614FF0904003F088FEBA
:104228004FF4C0551123CDE9015301A901234FF0E3
:104238009040039303F056FD08240A2500224FF40A
:1042480080514FF0904003F073FE0120FEF76AFCA6
:1042580001224FF480514FF0904003F069FE012095
:10426800FEF760FC013DE9D14FF400614FF090404A
:1042780003F058FE08B9013CDFD14FF400614FF05C
:10428800904003F04FFE68BBFFF7A9FF0424012309
:10429800039001A92A48CDE9014303F023FD284CE6
:1042A80001220421204603F043FE2120FEF73AFCB8
:1042B80000220421204603F03BFE2120FEF732FCB9
:1042C80001220421204603F033FE2120FEF72AFCB8
:1042D80020460022042103F02BFE4FF42570FEF740
:1042E80021FCDDE7FFF77BFF4FF0B04300249A6D18
:1042F80042F480029A659B6D03F4800300934FF4A7
:10430800C052009B1223CDE901230323CDE90343C7
:1043180004230DEB03014FF09040059303F0E2FCFA
:1043280008480949094B8460C0E900130123C0E922
:104338000334C0E90744446103F06EFF07B030BDA1
:1043480000040048640E0020005800401A0910209C
:10435800FFF754BF10B1012809D0704701394A420C
:104368004A414FF090404FF4007103F0E1BD4B1EFD
:104378005A4202485A410821F7E700BF00040048A2
:1043880008B50120FEF71BFF6420FEF7CBFB00F009
:1043980023F9BDE808400120FEF716BF054B1A684F
:1043A80002805A689B684381034B028101221A707C
:1043B800704700BFE40E00203D0E002010B50446F3
:1043C80000F008F810F0FF001CBFEE232370AA23AA
:1043D800637010BD2DE9F3470024304E304D346032
:1043E80021462046FFF7B6FF21460120FFF7B2FF1E
:1043F80021460220FFF7AEFF2A4F4FF05208A14690
:10440800012195F8640185F86081C5F86891FFF786
:10441800A1FF0320FEF786FB00228821284602F030
:10442800E3FB0DF10602C021284602F02BFC80BBFD
:10443800BDF806204EF6AA639A422AD14FEA440AEA
:104448000AF1540A5FFA8AFA5146284600F032F90E
:10445800F8B90DF10602C021284685F860A102F0DE
:1044680011FCB0B9284600F0E9FA90B93268012386
:104478001A4432603A68C5F86831A34013433B6078
:104488000134032C05F5C875BAD1306802B0BDE80F
:10449800F0870021E0B2FFF75DFFF1E7DC0E0020B6
:1044A800BC000020D80E00202DE9F74F354C83467C
:1044B80004F5966A4FF00A094FF00E0848F2E8072B
:1044C8004FF490164FF48045D4F86821002A51D053
:1044D800204600F0A7FD0DF102020DF10101204672
:1044E80000F05AFB0DF1030201A9204600F09FFEDF
:1044F8000021204600F0E2F801220021204600F0C9
:10450800A1F901221146204600F09CF9BBF1020FE7
:104518000ED81D4B1D4A33F81B501D4B12F80B804B
:1045280053F82B601B4A1C4B12F80B9053F82B7056
:104538002A460121204600F0D0F9324600212046C3
:1045480000F0CBF93946204600F0D2F84246002167
:10455800204600F0CFF84A460121204600F0CAF86C
:104568000DF102020DF10101204600F015FB0122B8
:10457800C4F87C2104F5C8745445A5D103B0BDE83E
:10458800F08F00BFBC000020A0410108C041010815
:10459800A8410108C3410108B441010810B50B7EC8
:1045A8009BB9D0F87C21098912B1C0E95E1310BD0E
:1045B800084BD0F878411A68C2F580734B4304FB66
:1045C80002331B12C0F87831F1E70123C0F87C31BF
:1045D800EDE700BFB80000202DE9F84FDFF8BCA0D8
:1045E8002F4DFFF7B5FEDAF800300BB12B6813B981
:1045F800FFF7F0FE28602B682A4E0024A34234609F
:104608007460B46044DDDFF8A080284DDFF8A0B006
:104618000220FFF749FF88F80040D5F86831012BE0
:104628002CD103FA04F90A272149284600F05AFC3C
:10463800B0B959462846FFF7B1FF9BF818307BB947
:10464800D5F8783146F82430DAF8003043EA09031F
:10465800CAF8003098F8003043F0010388F80030B9
:104668000120FEF75FFA9BF818309BB1013F17F065
:10467800FF07D9D14FF47A7346F824300520013466
:10468800FEF750FA032C05F5C875C6D198F8003026
:10469800BDE8F88FD5F87831EEE700BFD80E0020D6
:1046A800E00E0020E40E00203D0E0020BC0000209B
:1046B800BC0E00204A088A2102F096BA152906D8AD
:1046C800044BCB40DB0702D50174002070476FF024
:1046D800070070470B00300010B50A460C46092148
:1046E80002F0A4FA18B9237803F00103237010BD6F
:1046F80001F06BBE01F053BD01F04DBEF7B50023CC
:104708000C46174601210DF1070206468DF80730C1
:1047180002F08CFA0546D8B9012F9DF8073026D14A
:10472800042C3AD8DFE804F003171A1D200043F0E0
:104738001004A3420CD022460121304602F054FA5C
:10474800054628B9716986F830413046FFF7D0FF31
:10475800284603B0F0BD43F02804EAE743F0040418
:10476800E7E743F04004E4E743F08004E1E7042C82
:1047780013D8DFE804F00306090C0F0003F0EF0478
:10478800D7E703F0D704D4E703F0FB04D1E703F03D
:10479800BF04CEE703F07F04CBE76FF00305D7E74C
:1047A80013B500230C460DF1070201218DF80730DF
:1047B80002F03CFA78B99DF80730C3F30012227072
:1047C800C3F3C002A270C3F380026270C3F3801205
:1047D800DB09E270237102B010BD37B50D460DF14B
:1047E8000202F821044602F04DFA70B901AA042128
:1047F800204602F067FA40B9BDF802201AB1019BC1
:10480800B3FBF2F32B602B68A36103B030BD037FC9
:104818000B700020704737B50D460DF106022021B8
:10482800044602F02FFA28B9BDF8063023B9236AE6
:104838002B60207703B030BDDB002B60236201239F
:104848002377F7E70529F8B504460E46154635D807
:1048580062B100EB810301215A6B0023701E04280A
:1048680007D8DFE800F00E171A1D240011460123AF
:10487800F4E784F828103444E5B984F82850002077
:1048880007E0C2F34F224421204602F0BDF9002878
:10489800F1D0F8BD84F82A10EDE784F82B10EAE788
:1048A8005B00FE226021204602F0D5F9EFE71B01EC
:1048B800EF22F7E7012384F82830E0E76FF00300E0
:1048C800E7E7052996BF4018002390F828301370B1
:1048D80094BF00206FF00300704770B5431804467A
:1048E80093F828000E46154618B904EB8106726342
:1048F80070BD05291BD8DFE801F00309121416164C
:10490800626304EB860400206563F1E7C2F34F227B
:104918004421204602F078F90028E9D1F1E7E26362
:10492800EFE72264EDE7C2F34F226421F1E76FF06D
:104938000300DDE737B50446154605292CD8DFE81E
:1049480001F0030717191B1B436B2B60002021E0A4
:104958000DF10602442102F095F9D8B9BDF80620F8
:1049680053029AB12B60A363012384F8293011E024
:10497800C36BEAE7036CE8E70DF10602642102F075
:1049880081F938B9BDF806305B02DEE7A36B2B600E
:1049980084F8290003B030BD6FF00300FAE737B59B
:1049A8000D460DF107020121044602F03FF938B91E
:1049B8009DF8073084F83031DB092B7084F84C30CF
:1049C80003B030BD2DE9F843037C0C4601F8083BE1
:1049D8000546FFF702FF40BB207304F1100128468B
:1049E800FFF719FF08BB04F11401284600F021FC69
:1049F800D8B904F1240705F1270904F11708064678
:104A08003A46B1B22846FFF795FF70B9013619F852
:104A1800013F08F8013F062E07F10407F0D104F121
:104A28003C012846FFF7BBFF08B1BDE8F883211D0C
:104A38002846BDE8F84301F030BD0000F0B500227B
:104A4800054693B0882102F0CFF84FF47A72A5F8A2
:104A580052214FF4C872A5F854214C4AC5F8582180
:104A680000234B4A85F8F030C5F8D4202B6202A900
:104A78002846FFF7A7FF044670B9ADF8080002AE54
:104A88000FCE05F110070FC70FCE0FC70FCE0FC7F8
:104A980096E80F0087E80F003E4BC5F834314FF415
:104AA800FA730126A5F838314FF42063A5F83C3194
:104AB8003246802185F85061284602F095F8324642
:104AC8000746FF21284602F08FF8002211460743C7
:104AD800284602F089F83C4364B204430DF107020A
:104AE8009121284602F0A2F864B29DF8073085F8B3
:104AF8003A31044332460021284602F075F864B280
:104B080004430022FF21284602F06EF864B20443F1
:104B180000228021284602F067F864B2204340B2A0
:104B2800002488BBA1B2012228460134FFF78AFE7F
:104B3800062CF6D140BB0446688502460421284667
:104B4800FFF780FE00BB024605212846FFF77AFEE4
:104B5800D0B94FF490136B634FF48042012128467B
:104B6800FFF7BBFE80B94FF40C13FF22C5E90F30E5
:104B780085F830210121284602F036F8012385F80E
:104B8800323108B985F8154113B0F0BD856B0100C5
:104B9800A470090064008403012300F079BD2DE9A5
:104BA800F0428EB00C460C2304AA1421054602F0EC
:104BB80005F8844600286CD19DF81A309DF81B60D2
:104BC8009DF817209DF81810A07506EB03269DF890
:104BD8001630206002EB03229DF81930606003EB69
:104BE80001239BB25B029DF8121023619DF81330DC
:104BF800B5F8520103EB012392B252029BB2E26074
:104C0800A382B0F57A7F9DF8101095F83171B6B28D
:104C18000AD0704300F5FA704FF47A76B0FBF6F0DC
:104C28002E7F002E39D186B2002F40D0B001C0B2FD
:104C3800B608E0750DF10F002681CDE90040284641
:104C480001F086FE844620BB9DF80FE084F818E04A
:104C580005F150060FCE07AF0FC796E80700E37DB2
:104C680087E80700D4E90301A28AADF83020D4E927
:104C78000149CDE90A01CDE9084907AC8DF833307F
:104C88008DF834E00FCC50350FC597E8070086E85B
:104C9800070060460EB0BDE8F0822E8C5E43B2EB92
:104CA800262F4FEA262C04D157B948F6E0260020D3
:104CB800BFE780B25043A2EB0C06B0FBF6F0B2E7B8
:104CC80042F2B826B2E70000F7B517460E210DF1FB
:104CD80006021D460B4C064601F0D4FFBDF806300F
:104CE80004EA43433B6050B90DF106020C213046FB
:104CF80001F0C8FFBDF8063004EA43442C6003B055
:104D0800F0BD00BF0000FE1F73B590F8DA30013B1C
:104D1800022B06460C4634D801AB6A460121FFF740
:104D2800D3FF009BB3F57F0F054603D8019BB3F56E
:104D38007F0F23D915BB34B11349304602B0BDE803
:104D4800704001F00FBC0422FF21304601F04CFFF7
:104D58002A4604467021304601F046FF2A4604439D
:104D6800FF21304601F040FF64B204432A46802107
:104D7800304601F039FF64B2044365B2284602B0F8
:104D880070BD0025FAE700BF5F06002037B504466E
:104D980001228021057C01F027FF0122FF21204606
:104DA80001F022FF00221146204601F01DFF94F871
:104DB8003A219121204601F017FF012200212046C7
:104DC80001F012FF0022FF21204601F00DFF002212
:104DD8008021204601F008FF012D29D0032D37D06E
:104DE800002D3CD101222946204601F0FDFE012379
:104DF8008DF80730A0B103B030BD01460DF10702B0
:104E0800204601F013FF9DF80730DB0705F1010587
:104E180008D538B9B5F5FA6FEFD16FF00600EAE7B3
:104E28000546F0E7B5F5FA6F08BF6FF00600E2E750
:104E380018B929462046FFF767FF022200212046BD
:104E480001F0D2FE0028D6D1042384F83231D2E70B
:104E580018B901212046FFF757FF0422EEE76FF04B
:104E68000700C8E738B5057C044625B1204600F0A0
:104E780054FD28B138BDFFF789FF0028F6D0F9E7BF
:104E8800002DF7D1032384F83231F3E773B50646D2
:104E9800002501220B21304601F0A6FE002204461F
:104EA8000B21304601F0A0FE0DF107020443132147
:104EB800304601F0BBFE9DF8073064B2044301356B
:104EC8005B0760B2EDB205D0032D08D00028E0D012
:104ED80002B070BD032D08BF6FF00B00F8E76FF04C
:104EE8000B00F5E738B50023037404460D46FFF7B9
:104EF800B9FF50B929462046FFF751FE28B90146A7
:104F08002046BDE83840FFF7C1BF38BD152970B548
:104F1800054616461C4667D10122FF2101F064FEB2
:104F2800002211460446284601F05EFE0022044392
:104F3800FF21284601F058FE64B204430122802173
:104F4800284601F051FE64B2044302228521284616
:104F580001F04AFE64B204430422FF21284601F00E
:104F680043FE64B204430022CD21284601F03CFEF2
:104F780064B204431122CC21284601F035FE64B204
:104F880004430722FF21284601F02EFE64B20443A1
:104F98000022BE21284601F027FE64B204430622FF
:104FA800FF21284601F020FE64B204430922CC21E7
:104FB800284601F019FE64B204430022FF21284666
:104FC80001F012FE64B204430122FF21284601F0D9
:104FD8000BFE64B2002204431146284601F004FE89
:104FE80064B2204340B270BD042A17D80A2101F0E8
:104FF800FBFD0028F7D1231E18BF01231B01EF2258
:105008008421284601F027FE0028ECD185F8DA60D3
:1050180001462846BDE87040FFF738BF6FF00A0028
:10502800E1E7000070B594B005464022002104A8CD
:105038000EF040FF002301212846ADF806308DF818
:1050480003308DF80430029300F0B8FC95F8142171
:1050580095F81311012A04D840F0AD80202940F2B8
:10506800AC8001AA02A9284600F02DFB04460028BE
:1050780040F09E8095F85031002B40F0A280D5F882
:105088004C11284601F06EFA0446002840F0908042
:105098002346214604222846FFF738FF0446002805
:1050A80040F086800122FF21284601F09DFD0DF188
:1050B800060206468421284601F0E4FD22460643FE
:1050C800FF21284601F090FD76B2064374B2002C09
:1050D8006ED1BDF806301B01C5F8D43004A92846A6
:1050E800FFF770FC0446002862D10DF10301284641
:1050F800FFF7F2FA044600285AD19DF8033085F8E4
:10510800313104AE0FCE05F110040FC40FCE0FC419
:105118000FCE0FC496E80F0084E80F000DF10302CC
:105128000121284601F082FD0446002840D19DF85F
:10513800033085F83031024601462846FFF7DEFA8B
:105148000446A8BB024602212846FFF7D7FA0446C0
:1051580070BB0323014685F832310DF1050228465C
:1051680001F019F9044618BB9DF8053085F8E830B8
:105178000DF105020121284601F00DF90446B8B9E0
:105188009DF8053085F8E03003AA0321284600F091
:1051980001FF044660B9039BC5F8E43003AA042163
:1051A800284600F0F7FE044610B9039BC5F8DC302A
:1051B800204614B070BD0C2951E7284600F010F9BC
:1051C80054E701495DE700BF6C05002013B50C46A4
:1051D8000DF10702132101F029FD9DF8073013F0A6
:1051E800180F03F0070218BF6FF00500226002B025
:1051F80010BD13B590F8DA30042B0C460BD101A979
:10520800FFF7E4FF019B042B01D1012300E00023F9
:10521800237002B010BD01AA142101F007FD002877
:10522800F7D19DF80430DB07EFD42070F1E700F0E8
:105238004ABA13B50C460DF10602282101F022FDE9
:1052480078B9BDF80620C2F30B0312F4006F18BF3B
:10525800A3F580534FF0FA0214BF13FB02F3534334
:10526800236002B010BDF0B54FEAD20C4FF0FF3406
:105278001C6002F00702664600278E4200D207B182
:10528800F0BD845D664503BF1441E4B215463D4652
:1052980014F0010704D005EBC6051D600136ECE7E4
:1052A8000135082D4FEA5404F2D1F7E7034B800982
:1052B80053F82000003818BF012070471808002054
:1052C80010B5B1EBD20F4FEAD20402F0070381BF49
:1052D80001229A40035D13438ABF03556FF03100E2
:1052E800002010BD0A460623B02101F049BC0A4639
:1052F8000623B02101F062BC2DE9F04F85B080464D
:10530800109E0E9D01968A4693461C464FF0000952
:10531800119B994508D10023129A1660F3B16FF0DA
:10532800310005B0BDE8F08F01AB3246294658463A
:10533800FFF799FF019F7B1C0DD00F9BF818FFF713
:10534800B5FF504507D13A462046FFF7B9FF7E1C06
:1053580009F10109DCE76FF03103DDE7214640463A
:10536800FFF7C0FF0028DCD102A94046FFF7BFFFC6
:105378002544234602AAAB42D3D013F8014B12F8B6
:10538800011B8C42F7D0CAE770B5C02288B00E4620
:10539800012190F83041054601F026FCF0B901A939
:1053A8002846FFF79FFDC8B90122FF21284601F0D2
:1053B8001BFC98B93246B621284601F063FC68B94F
:1053C8000246FF21284601F00FFC38B92246012188
:1053D800284601F009FC08B985F8304108B070BDCD
:1053E800F0B50F4689B01646FF210122044601F0A8
:1053F800FBFB0246A8B94F21204601F0F5FB80B916
:105408002C224E21204601F0EFFB024648B9FF212D
:10541800204601F0E9FB20B9B422B621204601F06C
:10542800E3FB0025C4F82451A4F82851DEB9354619
:1054380007ABB422CDE903730623CDE90032029508
:1054480004F5927304F5957231462046FFF754FF30
:1054580030B9012384F8153184F8137184F8146184
:1054680009B0F0BD013505F1B400FFF71FFF0028B2
:10547800DED12C2DF6D1DBE710B541F00102002179
:10548800044601F0B1FB78B9204600F046FA58B955
:1054980001462046FFF7FAFC30B90246014620468D
:1054A800BDE8104001F0A0BB10BD2DE9F74F4FF04B
:1054B800000B88461746FF21012205461E469DF827
:1054C80038A09DF83C908DF807B001F08DFB5A4646
:1054D80004465946284601F087FB5A460443FF21F3
:1054E800284601F081FB64B2044364B2B8F1000FAE
:1054F80032D0BAF1000F06D00C9ACB21284601F021
:1055080095FB204344B2B9F1000F07D00DF1070213
:10551800EE21284601F08AFB204344B20122FF21F4
:10552800284601F061FB012204430021284601F0CE
:105538005BFB64B204430022FF21284601F054FBC0
:1055480064B29DF807300D9A204323F0100340B24F
:10555800137003B0BDE8F08FBAF1000F06D03A46D9
:10556800CB21284601F040FB204344B2B9F1000F9B
:10557800D4D033468022EE21284601F06CFBCBE7DD
:105588002DE9F04387B091460022054688468DF8FC
:1055980017201E461BB390F8307101221146284689
:1055A80001F022FB044658BB40212846FFF764FF60
:1055B800044628BBB9F1010F13D10DF11703CDE94A
:1055C8000290CDE900830246034649462846FFF784
:1055D8006CFF40B10446204607B0BDE8F0831F4683
:1055E800DBE788F80000002EF5D03A46012128466E
:1055F80001F0FAFA04460028EDD185F83071EAE79F
:10560800002388F800302046E4E72DE9F0430546FA
:1056180087B0884691461E4623B390F8307102221F
:105628000121284601F0E0FA044660BB01462846FD
:10563800FFF722FF044630BBB9F1010F14D10DF179
:105648001703CDE90209009302460346CDF804800A
:1056580049462846FFF729FF40B10446204607B0CF
:10566800BDE8F0831F46DAE788F80000002EF5D081
:105678003A460121284601F0B7FA04460028EDD140
:1056880085F83071EAE7002388F800302046E4E71F
:10569800F8B51D46164600232A4690F83071044690
:1056A800FFF76EFF70B903462A4631462046FFF7DA
:1056B800ACFF38B93A460121204601F095FA08B9FD
:1056C80084F83071F8BD2DE9F04F002393B0CDE98F
:1056D8000A12C0F82431A0F828310122FF21CDE9AF
:1056E8000E33B0F83C818DF8343005468DF83530EE
:1056F80001F07AFA0446002840F0E38002464F2180
:10570800284601F071FA0446002840F0DA802C227D
:105718004E21284601F068FA0446002840F0D1805E
:105728000246FF21284601F05FFA0446002840F0AF
:10573800C880B422B621284601F056FA044600284B
:1057480040F0BF8002468021284601F04DFA044609
:10575800002840F0B68003460DF135020DA9284611
:10576800FFF796FF0446002840F0AB800323CDE9FD
:105778000203B421062305F5957A05F592790EAE54
:10578800CDE90031049601464B4652462846FFF7BC
:10579800B3FD0446002840F094800DF136012846F8
:1057A8000E9FFFF7F1FD0446002840F08A80BDF8FF
:1057B8003630434540F2AA80C5F82401A5F82801EF
:1057C80007F1B400FFF772FD08B92B2F7DD9062326
:1057D800B4224FF0030BCDE90032CDE9027B0496E9
:1057E8004B46524601212846FFF786FD002840F027
:1057F8008B800DF1360128460E9FFFF7C5FD064642
:1058080000287CD1BDF83630434540F2828001261D
:105818000696BDF83630434560D2A3EB080383EA09
:10582800E372A2EBE3729DF81860099205F5927392
:105838004FF0030B0793079B18689B881090ADF8EF
:1058480044303A460FAB06215046FFF70CFD0F9F38
:105858007B1C56D007F1B400FFF728FD069B984241
:105868003CD10BF101033A4648460893FFF728FD5F
:10587800002849D149462846FFF734FD002843D17E
:105888000DF136012846FFF77FFD00283CD1BDF811
:105898003620A2EB0803002BB8BF5B42424516D95D
:1058A800099A934218D910A92846FFF71BFD079AB1
:1058B8000799034610981060BDF844208A806BB1A0
:1058C8001C46204613B0BDE8F08F013778E7DDF8B5
:1058D80020B009930137AEE7DDF820B00A9BC3F882
:1058E80000B00B9B1E70012385F815310A9B1B68BD
:1058F80085F813310B9B1B7885F81431E1E70446D2
:10590800DFE76FF03104DCE70446DAE70026B34648
:105918007EE70123834606937BE737B500230446D9
:105928008DF807304FF4FA650DF107012046FFF7AF
:1059380060FC58B99DF80730012B07D0013D03D012
:10594800204601F0E5F9EFE76FF0060003B030BD3F
:1059580002464FF08043934202D8002013B97047A3
:105968009B08F8E7C11891424FEA50009CBFC01845
:10597800521A9B08F2E773B500228321054601F00D
:1059880033F9044688B94FF4FA660DF1070283210A
:10599800284601F04BF99DF807300343DBB2044673
:1059A8001BB9013EF1D16FF006040122832128467C
:1059B80001F01AF9204340B202B070BD2DE9F04F52
:1059C80090F8F06091B04FF00009072ECDE90799E3
:1059D80004460F4600F0A2820122802101F004F95A
:1059E80001228046FF21204601F0FEF84A4648EA97
:1059F80000084946204601F0F7F84FFA88F848EAC7
:105A080000080622FF21204601F0EEF84FFA88F838
:105A180048EA00080DF115028321204601F006F935
:105A28009DF815204FFA88F848EA000842F0040269
:105A38008321204601F0D8F84FFA88F848EA000890
:105A48000722FF21204601F0CFF84FFA88F80122FB
:105A5800812148EA0008204601F0C6F84FFA88F884
:105A680048EA0008204601F053F94FFA88F848EA56
:105A7800000801228021204601F0B6F84FFA88F884
:105A880048EA000517F0010B6DB200F01E82F2071C
:105A980000F11E826B229421204601F0A5F8804671
:105AA8002046FFF768FF06AA48EA0008902120462A
:105AB80001F008F945EA0805069B6DB224229421F5
:105AC80005432046C3F3062AC3F3C03901F08CF816
:105AD8006DB205432046FFF74EFF6DB2054306AA97
:105AE8009021204601F0EEF8069B6DB21BBA2522E4
:105AF800942105432046099301F076F86DB20543D9
:105B08002046FFF738FF6DB2054306AA90212046CC
:105B180001F0D8F8069B6DB21A0E05431B0C6DB246
:105B28008DF828208DF8293017F00203029300F031
:105B3800DB8016F0020840F0D7800222942120462C
:105B480001F052F801902046FFF715FF019B0DF177
:105B580016020343902120461D4301F067F86DB2F9
:105B68007B2294210543204601F03EF86DB205439F
:105B78002046FFF700FF6DB205430DF11702902193
:105B8800204601F053F86DB2772294210543204650
:105B980001F02AF86DB205432046FFF7ECFE6DB21E
:105BA800054306AA9021204601F08CF8069B5A0E60
:105BB8008DF82C20C3F386428DF82D20C3F3C6221E
:105BC8008DF82E206DB2C3F30612DB0003F07803C4
:105BD800942105438DF82F20204678228DF8153022
:105BE80001F002F86DB205432046FFF7C4FE6DB21E
:105BF800054306AA9021204601F064F8069B9DF80B
:105C0800152002EB53728DF83020C3F386528DF8BD
:105C18003120C3F3C6328DF83220C3F306228DF843
:105C280033206DB2C3F346029B0103F04003942175
:105C380005438DF83420204679228DF8153000F080
:105C4800D3FF6DB205432046FFF795FE6DB20543BD
:105C580006AA9021204601F035F8069B9DF81520EC
:105C680002EB93628DF83520C3F3C6428DF83620D7
:105C7800C3F306328DF837206DB2C3F346129B008A
:105C880003F07C03942105438DF8382020467A22BE
:105C98008DF8153000F0A8FF6DB205432046FFF7D8
:105CA8006AFE6DB2054306AA9021204601F00AF863
:105CB800069B9DF815208DF83E8002EB93728DF8B7
:105CC8003920C3F3C6526DB28DF83A20C3F30642A9
:105CD80005438DF83B20C3F34622C3F386036DB218
:105CE8008DF83C208DF83D3017F00403019300F047
:105CF800F180730700F1EE807B229421204600F0AA
:105D080073FF80462046FFF736FE07AA48EA0008D8
:105D18009021204600F0D6FF45EA08084FFA88F897
:105D280048EA00057C229421204600F05DFF6DB210
:105D380005432046FFF71FFE6DB2054308AA9021D0
:105D4800204600F0BFFF6DB2732294210543204620
:105D580000F04AFF6DB205432046FFF70CFE6DB216
:105D6800054306AA9021204600F0ACFF069B6DB2C1
:105D78001B0274229421054320461FFA83F800F081
:105D880033FF6DB205432046FFF7F5FD6DB20543BD
:105D980006AA9021204600F095FF6DB29DF81B30B1
:105DA800752294210543204643EA080800F01CFFA9
:105DB8006DB205432046FFF7DEFD6DB2054306AA26
:105DC8009021204600F07EFF069B6DB21B029BB21D
:105DD8007622942105432046039300F005FF6DB217
:105DE80005432046FFF7C7FD6DB2054306AA90217B
:105DF800204600F067FF6DB29DF81B20039B05430A
:105E08006DB21343002281212046039300F0ECFE7B
:105E180006220543FF21204600F0E6FE6DB2054349
:105E28000DF115028321204600F000FF9DF8152092
:105E38006DB2054302F0FB028321204600F0D4FE38
:105E48006DB205430122FF21204600F0CDFE6DB260
:105E5800054301220021204600F0C6FE6DB205432D
:105E68000022FF21204600F0BFFE6DB2054300224C
:105E78008021204600F0B8FE6DB205436DB2039B49
:105E8800FDB9BBF1000F29D1029AAABB019AAAB1A8
:105E9800720713D4079AC4F81821089AC4F81C2169
:105EA8004FEA4822C4F820213BB1A3F5C8534FF468
:105EB8007A7253431B095B421BB2E3603E4384F88A
:105EC800F060284611B0BDE8F08FD946DA462BE6D7
:105ED800CA4629E64FF00008434693E7F007D3D4B3
:105EE8000998BDF8282084F813A184F81491C4F8FF
:105EF8002A01A4F82E21C7E7B107C7D49DF81620B8
:105F080084F8F1209DF8172084F8F2200BA904F1F9
:105F1800F30002930DF0FAFF029BB7E74D46D0E776
:105F280050B10138002330F0FF019AB203F10103A8
:105F380003D100EB022080B270474008F3E7C3B2F8
:105F4800000A03FA00F0013070470000084B5A437A
:105F58004FF47A7302F5FA724FF4FA60B2FBF0F07C
:105F6800B2FBF3F203FB0100B0FBF2F0704700BF95
:105F7800002F3A00064B5A434FF47A7002F5FA7232
:105F8800B2FBF0F24A4302F5FA72B2FBF0F0704746
:105F9800002F3A002DE9FF4102294FF0000507467E
:105FA80016468DF80350ADF804501CD80DF10202C6
:105FB8002946FEF7A1FB044630B90DF1030246213C
:105FC800384600F033FE04469DF80300FFF7B7FF9C
:105FD80081B29DF802203846FFF7CCFF306020469A
:105FE80004B0BDE8F081032918D10DF10202294659
:105FF800FEF782FB0446002846D101460DF1020255
:106008003846FEF779FB044628B901AA51213846DB
:1060180000F038FE0446BDF80400D7E7042935D15E
:1060280002A9FEF7BDFB9DF80B30ABB10DF10202E2
:1060380029463846FEF760FB044658B901AA5121A3
:10604800384600F01FFE0446BDF80400FFF777FF4E
:1060580085B214B1002015E01D460DF102020121A0
:106068003846FEF749FB04460028F3D10DF1060235
:106078007121384600F006FE0446BDF80600FFF719
:106088005EFF80B2401BA3E72846A7E728462C46B8
:10609800A4E7F0B5022985B0054616461ED80DF1CD
:1060A80005020021FEF728FB0446A0B99DF805204B
:1060B80031462846FFF74AFF83B2B3F5807F9ABF7F
:1060C80000F1FF32D2B2FF22A5F8D8204621284697
:1060D80000F08AFD0446204605B0F0BD03291FD113
:1060E8000DF105020021FEF707FB9DF8052031465A
:1060F80004462846FFF72AFF80B2FFF711FF024641
:10610800ADF80600A5F8D800002CE4D151212846A6
:1061180000F07AFD04460028DDD1C5F8E460DAE72E
:10612800042939D102A9FEF73BFB9DF80B70B7B1E2
:106138000DF1050200212846FEF7DEFA0446002884
:10614800C9D10DF106025121284600F09BFD0446F5
:10615800BDF80600FFF7F3FE87B2002CBBD10DF1A6
:10616800050201212846FEF7C7FA04460028B2D1E5
:106178009DF8052031462846FFF7E8FE3844FFF72A
:10618800CFFE71210246284600F03EFD0446002855
:10619800A1D1C5F8DC609EE76FF003049BE7F0B57A
:1061A80085B000238DF80330D30705460F46164601
:1061B80005D439B9A2F10C03DAB2062A11D96FF065
:1061C8000300E6E0012921D1A2F10803DAB2062A88
:1061D800F5D8062B1AD8DFE803F03B1969198A1994
:1061E8009D00062B12D8DFE803F004112D112F11A2
:1061F800310018225721284600F0F6FC08225621C3
:10620800284600F0F1FC002840F0C3807408013CE7
:10621800E4B2002F00F09180012FD0D101AA04210F
:106228002846FFF7B7FE50B922467021284600F0ED
:10623800DBFC20B9019A04212846FFF72AFF85F8DC
:10624800E06099E03022D5E74022D3E75022D1E739
:106258001022482100F0C8FC08224721284600F0F7
:10626800C3FC022204463221284600F0BDFC0C2261
:1062780004433021284600F0B7FC64B204430122ED
:10628800FF21284600F0B0FC64B2044364B2302217
:106298003021284600F0A8FC00220443FF212846AC
:1062A80000F0A2FC64B2204340B2ACE728224821A7
:1062B80000F09AFC08224721284600F095FC0322AA
:1062C80004463221284600F08FFC044364B20922B8
:1062D8003021284600F088FC01220443FF2128468B
:1062E80000F082FC64B2044364B22022D0E7382272
:1062F800482100F079FC08224721284600F074FC68
:10630800032204463221284600F06EFC044364B29E
:106318000822DDE74822114600F066FC08224721E2
:10632800284600F061FC032204463221284600F08A
:106338005BFC044364B20722CAE702AA0321284689
:10634800FFF728FEB0B903AA02212846FFF722FE6C
:1063580080B922465021284600F046FC50B9029ADE
:1063680003212846FFF795FE20B9039A0221284603
:10637800FFF78FFE85F8E86058B969692846FEF787
:10638800B7F930B9024601230DF103012846FFF79A
:106398003CF905B0F0BD13B5144629B1012910D058
:1063A8006FF0030002B010BD0DF10702502100F09C
:1063B8003DFC0028F6D19DF8073001335B002370BF
:1063C800F0E70DF107027021F1E7F0B5002385B081
:1063D8004FF4FA62CDE9002344F61F63994206465A
:1063E8000F4604D86FF00305284605B0F0BD02A992
:1063F800FEF7D6F905460028F6D19DF809209DF844
:10640800083013439DF80A201343A7F636341BD0EF
:106418006A4602213046FFF7BDFD00283BD19DF8B2
:1064280008302BB1009B03F24E239C42DAD9E41AC0
:106438009DF80A3023B3009B03F2B223B4EB430F59
:106448004FEA4302CED9A41A9DF80B305BB101AADA
:1064580003213046FFF79EFD019B03F52573A342F8
:10646800C0D2C0B9E41A9DF80C30002BBCD0A4F2FD
:10647800262204213046FFF70CFE77610546B3E774
:106488009DF80930002BDFD0009B03F525739C4253
:10649800A8D9E41AD8E70546A6E770B54FF4FA621A
:1064A80086B00023CDE9022340F636330B600C4654
:1064B80004A90646FEF774F90546002836D19DF86A
:1064C80011209DF8103013439DF81220134319D062
:1064D80002AA02213046FFF75DFD002840D19DF851
:1064E80010302BB1029B03F24E2223681344236021
:1064F8009DF81230EBB1029B03F2B222236803EB42
:10650800420323609DF81330EBB99DF814305BB15A
:1065180001AA04213046FFF73DFD019B03F2262224
:10652800236813442360D8B923687361284606B0EA
:1065380070BD9DF81130002BE4D0029B03F5257245
:1065480023681344DDE703AA03213046FFF722FD41
:10655800039B03F525722368134423600028D4D0D5
:106568000546E3E72DE9F743002406460D46204695
:1065780015F80480B8F1000F00D010B103B0BDE8E1
:10658800F083671CB8F1FF0F15F8079029D1A71CF5
:10659800EB5DB9F1030F36D8DFE809F0020B131BE6
:1065A800271D2C44E27802EB0323A6F834313C463D
:1065B800DEE7271D2C44E27802EB0323A6F83631E8
:1065C800F5E7271D2C44E27802EB0323A6F83831BF
:1065D800EDE7271D2C44E27802EB0323A6F83C31B3
:1065E800E5E7B8F1040F0ED802344246291901A88C
:1065F8000DF099FC434601AA4946304604EB0807CA
:1066080000F0BEFAD3E76FF00300D0E773B50023BC
:106618000E4613600DF1070105461446FEF7F7F81C
:1066280040B99DF807302BB1B38A2A6A53438033A7
:106638001B0A236002B070BD13B5CB681360144603
:1066480001AAFFF7E3FF18B92368019A13442360EE
:1066580002B010BDF8B5B0F85451D0F858016843ED
:106668008030000A0E464543DDE90717144652B14B
:10667800B60206EB5202B2FBF4F202EB42025243BC
:1066880002F50042140C069A534301F50042120C1D
:1066980006200332B2FBF0F2C2EBC202B2F5803F31
:1066A80038BF033103F500433EBFB1FBF0F1C1EB46
:1066B800C10101F500414FEA134334BF090C1B49DE
:1066C80003FB03F338BF494303EB57030B44B3FB06
:1066D800F7F39B03FE2205F120007F33B3FBF2F3AF
:1066E8005C434FF47A7704F5FA748009B4FBF7F445
:1066F8002401FFF72DF904F5FA74BC4228BF4FF4C2
:10670800FA63064629BFB4FBF3F300205B19B4FB18
:10671800F7F428BFB3FBF4F0FFF71AF9099B864298
:1067280094BF1E6018600020F8BD00BF0000F0FF95
:106738002DE9F04F91B0CDE90723036A0E930B6959
:1067480009930546CB680B930F460FAAFFF774FF12
:106758000EAA39462846FFF759FF58BB0F9C95F8F3
:10676800E0B0D5F8DC3005934FF47A7606FB04F1F7
:1067780001F5004104910E990A910499D5F8E43085
:106788000693BBF1080F04F180040CBF0223032316
:1067980024F0FF0A090C95F8E820DFF8A081CDF86D
:1067A8003CA00C9109D1079BC3F80080089BC5F851
:1067B8004081186011B0BDE8F08F06990D93284606
:1067C800FFF7C4FB5A46059981462846FFF7BEFBEA
:1067D8000D9B5B490C9A814403FB09F94FEAC929CF
:1067E80040F2776309F5FA79240AB9FBF6F903FB55
:1067F80009F909F5FA79B9FBF6F909FB04F404F18A
:106808008003099C74430C40B4FBF2F44D4A1B0A04
:10681800944228BF1446012B38BF01230C204FF4A3
:10682800167258435443FFF793F83B7E3A894FEA70
:10683800400B002B7FD14249049B0B4003F5FA71B2
:10684800414B5A4341F25C23B2FBF3F20A9B734378
:10685800B3F5481F28BF4FF44813A1EB4303B1FB1E
:10686800F6F1B3FBF6F31B02B3FBF1F63602C6F5FD
:106878008036564306F50046360C06F5803676080F
:106888007643B60B4FF44870704304F5004300F5A7
:1068980000401B0C5B43000C00FB0030FFF758F86E
:1068A80003046422323341F28837B3FBF2F340F633
:1068B800B532B3FBFBF302FB0377244B9F429CBF2B
:1068C80042F21073B7FBF3F7DDE90532134403F521
:1068D800FA734FF47A7B4FF4FA62B3FBFBF0B3FB25
:1068E800F2F202F5C812B2FBF0F088BF4FF470471D
:1068F800FFF72EF8000200F5FA70B0FBFBF04043FA
:1069080007FB0700FFF724F80BFB00F0079B0B9A27
:10691800404528BF40461860089BC5F84001CDE9AE
:1069280002934FF448730093019433465146284626
:10693800FFF790FE3EE74FF48036A3E7AE878F025D
:106948000000FFFF666666009A9906000F279F24DD
:106958002DE9F04F8BB0002711F0780FDDE914B85E
:106968000446019299468DF80E708DF80F708DF8D7
:1069780010708DF81170ADF812700997C1F3C30A41
:1069880000F0AF80AAF10503DBB20A2B01D86B4AED
:10699800D75C0DF10E0200212046FDF792FF9DF80D
:1069A8000E500646D5B1002840F09D8009AB05AAD7
:1069B80059462046FFF7BCFE002840F09680099B08
:1069C800ABF80A30014606AA2046FDF7B3FF069D3C
:1069D80025B1059B9D422CBF0025012520B904AA9D
:1069E80002212046FDF76DFF9DF8106026B30028B0
:1069F8007DD107AA02212046FDF79CFF88B9012214
:106A0800FF21204600F0F0F858B90DF11202B62126
:106A1800204600F037F920B90246FF21204600F051
:106A2800E3F8BDF81230079E5B02C4F848311EB186
:106A38009E422CBF0026012628B90DF11102032120
:106A48002046FDF73EFF9DF8113093B1002873D121
:106A5800B9F1000F03D0019B1B02B3FBF9F908AA97
:106A680003212046FDF766FF089B4B4594BF002392
:106A7800012320B9012F3CD1FF2288F8002098F883
:106A880000200AB9ABF80A200DF10F0201212046B7
:106A98000193FDF716FF08BB9DF80E20019B002A05
:106AA80008BF0125BAF1040F18BF9DF80F2084F81C
:106AB8002E501ABFB2FA82F25209012284F82F200E
:106AC8009DF81020002A9DF8112008BF0126002AF1
:106AD80008BF012384F8306084F831300BB0BDE87A
:106AE800F08F012755E700257EE735467CE700262D
:106AF800A9E70AF1FF32092A0AD8DFE802F00505FA
:106B080005090907090B070B0522B6E70422B4E7B4
:106B1800012E01D10322B0E7BAF1040F01D0012BF5
:106B280001D10222A9E7012D1BBF002388F80030FC
:106B380088F800502B46A2E70023A0E7C6410108C9
:106B480007B502F10A03009393B20A4690F8601160
:106B5800D0F85C0101F0B2FB03B05DF804FB13B59B
:106B680002F10A0390F860410093D0F85C0193B2F7
:106B78000A4644F0010101F037FC02B010BD0000E4
:106B88003F2BF8B50E46054611461C4611D80A4F4C
:106B980038461A4600F8016B0DF0C5F9621C3946F3
:106BA8002846FFF7CDFF00280CBF00206FF0130028
:106BB800F8BD6FF00300FBE7F00E002073B5154633
:106BC8008DF8071001220DF1070104461E46FFF754
:106BD800B7FF28B9324629462046FFF7C0FF08B15B
:106BE8006FF0130002B070BD08B5064B19705A70EB
:106BF80019460222FFF7A4FF002814BF6FF0130004
:106C0800002008BDF00E002008B5074B1970110AC6
:106C180059709A7019460322FFF792FF002814BF93
:106C28006FF01300002008BDF00E002037B51546A0
:106C38008DF8071001220DF107010446FFF780FFC8
:106C480028B9012229462046FFF789FF08B16FF0CD
:106C5800130003B030BDF7B515460DF1070206461F
:106C68000F461C46FFF7E2FF50B99DF807301D405C
:106C780044EA0502394630468DF80720FFF7B4FF8D
:106C880003B0F0BD73B514468DF8071001220DF15D
:106C980007010646FFF754FF18B16FF0130002B062
:106CA80070BD074D022229463046FFF758FF0028DD
:106CB800F3D12A786B7803EB02232380EFE700BF38
:106CC800F00E002073B514468DF8071001220DF15F
:106CD80007010646FFF734FF18B16FF0130002B042
:106CE80070BD0A4D042229463046FFF738FF0028B8
:106CF800F3D16B782A781B0403EB0263EA78134418
:106D0800AA7803EB02232360E9E700BFF00E002016
:106D180008B50220FBF706FF002008BD70470000F9
:106D280010B5032000F072FC01F0AAFD064B1860B4
:106D38000F20FBF7EDFE044618B9FBF75AFD204675
:106D480010BD0124FBE700BF280800204FF0E02217
:106D5800136923F00203136170474FF0E0221369AF
:106D680043F0020313617047014BD3F89005704755
:106D78000070FF1F014BD3F8940570470070FF1F88
:106D8800014BD3F8980570470070FF1F024A5368FB
:106D980023F0010353607047002004E0024A53685F
:106DA80023F0020353607047002004E0024A53684E
:106DB80023F0040353607047002004E08068C0F3A8
:106DC80080007047F7B5002301930446002800F0BF
:106DD800E980856D25B9FBF741F8E56584F85450DD
:106DE80023689A68D00040F1A1809A68D10000F128
:106DF800B480A26D42F01002A265E26D42F0010279
:106E0800E26501251846FFF7D9FFA26D02F01002CE
:106E1800024340F0C980A26D206922F4817242F0D9
:106E28000202A2659A68D2075DD4226BA67E94F806
:106E38002CC0003A18BF01221703D4E902120A43F2
:106E4800217E42EA8132617E42EAC13242EA46321A
:106E5800002842EA4C02B4BF20F000414FF4001170
:106E68003A430A4394F82010012903D1002E76D121
:106E780042F48032616A21B1A66A01F4E0713143BB
:106E88000A43D968E66C21F4FE3121F4FF711143FD
:106E9800D96094F83C206168012A01F0404C4CEA22
:106EA800060609D1D4E910273A433243A66C324387
:106EB80042EA0C0242F001061F693E4A3A40324358
:106EC8001A6121F00042B2F1804F0CD0B1F1004FAD
:106ED80009D0394ED6F8082701F4701122F470123F
:106EE8000A43C6F808275A69666BA16B22F00702A5
:106EF80032435A615A6922F0700242EA01125A6119
:106F0800002835D19A6A62F00F029A625B6903F031
:106F180007039E423CD10023E365A36D23F00303DE
:106F280043F00103A365284603B0F0BD9A682349DE
:106F380022F0104222F0170242F080529A60204A52
:106F48001268B2FBF1F2013252000192019A002A52
:106F58003FF44BAF019A013AF7E7002552E7A16DDC
:106F680041F02001A165E16D41F00101E16581E792
:106F7800B0F5001FCAD19A6AE269013A92006FF02F
:106F88000F0102F01C0201FA02F2216E0A43BCE76B
:106F9800A36D23F0120343F01003A365E36D43F0E0
:106FA8000103E3650125BEE7A36D43F01003A36564
:106FB800F8E700BF02FCFF1F00200140400D03005E
:106FC80028080020F8B54569082D04460E460AD061
:106FD8000368DB68D80705D5A36D43F02003A365D4
:106FE8000120F8BD0425FBF795FD074623681A68BC
:106FF8002A4221D0A26D42F40072A265DA6812F426
:10700800406F14D1A27E92B91A6812070FD518469C
:10701800FFF7D4FE28BB5A6822F00C025A60A26D12
:1070280022F4807222F0010242F00102A265207E61
:1070380000BB0C221A60D4E7711CD8D0FBF76AFD9C
:10704800C01BB04201D8002ED0D123681B682B404A
:10705800CCD1A26D84F8543042F00402A26503201A
:10706800BFE7A26D42F02002A265E26D42F0010284
:10707800E265DCE70020B4E70368186C704700009D
:10708800F7B50023019390F85430012B044600F023
:10709800C58005680669012380F854302846FFF743
:1070A8008DFE002840F0B480D1E90020022826F0A7
:1070B800040300F08280B3F1004FC2F3110E13D124
:1070C800AB6A43EA0E03AB628B68686903EA022382
:1070D80023F07C4323F0FF0320EA02210B43002A1C
:1070E8006B6126DB002055E0236E00F01F074FF090
:1070F8000F0C0CFA07FC6FEA0C0623EA0C0CBEF125
:10710800000F11D1C2F38463BB4043EA0C0323662A
:107118008008E36901309842D6D8A86AC2F383632D
:10712800BB4006403343CEE792FAA2F3B3FA83F3A7
:10713800EAE73B493B48D1F80837824203F0E0755B
:1071480019D11B02CED4D1F8083723F0E0732B43B2
:1071580043F40003C1F80837334B1A68334BB2FBCA
:10716800F3F20C2302FB03330193019B002BB9D0EC
:10717800019B013BF8E72E48824210D113F0807042
:10718800B0D1D1F8083723F0E0732B4343F0807374
:10719800C1F80837002384F8543003B0F0BD2548FF
:1071A80082429FD113F480009CD1D1F8083723F094
:1071B800E0732B4343F48003EAE7B3F1004F01BFC8
:1071C800AB6AC2F311018B43AB62002A8ADA154815
:1071D80013498242D1F8083709D1D1F8082703F0BA
:1071E800A07322F0E0721343C1F808377AE7104819
:1071F800824204D1D1F8082703F44003F1E70D488F
:1072080082427FF46FAFD1F8082703F0C073E8E734
:10721800A26D42F02002A2651846BBE70220BCE737
:1072280000200140001000B028080020400D030095
:10723800004000B8002000B4026838B50446104683
:10724800FFF7BCFD08B9002038BD9368990707D43B
:10725800936823F0004323F0170343F0100393606F
:10726800FBF758FC054623689B685B07EBD5FBF7E3
:1072780051FC401B0228F6D923689B685A07F2D5AF
:10728800A36D43F01003A365E36D43F00103E365C9
:107298000120D9E773B50023026801939368DD07DD
:1072A800044602D5002002B070BD9168214B1942F6
:1072B80009D0A36D43F01003A365E36D43F0010308
:1072C800E3650120EFE7936823F0004323F01703F9
:1072D80043F001039360184BD3F8083718021CD405
:1072E800637E012BDED0FBF715FC144E05462268A1
:1072F8001368DB07D6D49368D9075FBF9368334018
:1073080043F001039360FBF705FC401B0228EED90C
:1073180023681B68DA07EAD4CBE7094B094A1B68DC
:10732800B3FBF2F301330193019B002BD8D0019BEF
:10733800013BF8E71700008000200140E8FFFF7FCD
:1073480028080020400D030038B504460068FFF700
:1073580035FD054620BB94F85430012B20D001237D
:1073680084F854302046FFF795FFB0B9A36D226822
:1073780023F4706323F0010343F48073A3651C2393
:10738800E065136084F85400936823F0004323F009
:10739800170343F00403936038BD84F85450FBE7A7
:1073A8000220F9E7026838B5936891680446C8076F
:1073B80001D4002038BD9907FBD4936803F0050376
:1073C800012B19D1936823F0004323F0170343F0EE
:1073D8000203936003231360FBF79CFB05462368B5
:1073E8009B68DB07E5D5FBF795FB401B0228F6D920
:1073F80023689B68DA07F2D5A36D43F01003A365F1
:10740800E36D43F00103E3650120D3E770B504465B
:1074180000284BD0836D43F002038365FFF70CFF10
:10742800054668B92046FFF7BDFF054608B90123A0
:10743800A3652268936823F0104323F01703936031
:1074480023685A6822F4677222F003025A6040F2F5
:107458009F321A60D968164A0A40DA601A6922F01F
:1074680040421A615A6922F007025A611A6A02F008
:10747800F0221A625A6A02F0F0225A62DA6A02F0BC
:10748800F022DA629A6A0B4A00269E62D2F808371E
:1074980023F0FE73C2F808372046FAF7F3FCE665D6
:1074A8002666A66584F85460284670BD0125FBE76A
:1074B80000023E830020014010B590F85430012BA3
:1074C800044615D0012380F85430FFF7B5FE58B9AB
:1074D8002046FFF767FF38B9A36D23F4807323F0C4
:1074E800010343F00103A365002384F8543010BD61
:1074F8000220FCE7F7B50023019390F85430012BE4
:1075080004467FD0012380F85430FFF74BFF2368EF
:107518009A6812F00102054607D0A36D43F01003E4
:10752800A365002384F854302DE0A16D364F21F473
:10753800817141F00201A165DE68D96826F4FF4631
:1075480026F07C0621F40041360421F00301360CB4
:10755800D96008209968394041F0004199609968DC
:10756800002913DA0199013101910199B1F52E3FF2
:10757800F5D3A36D23F0120343F01003A365002392
:1075880084F854300125284603B0F0BDD3F8B41070
:10759800013801F07F010A44DCD199681A4801409A
:1075A80041F001019960D3F8B41021F07F0141EA5C
:1075B800D202C3F8B4209A68024042F002029A60EC
:1075C800FBF7A8FA074623689A68D20708D4DA684E
:1075D8003243DA60A36D23F0030343F001039FE70E
:1075E800FBF798FAC01B0228EDD923689B68D907D6
:1075F800E9D5A36D43F01003A365E36D43F00103E0
:10760800E365BFE70225BEE7E8FFFF7F0749CA68D1
:1076180022F4E0620302120403F4E063120C134341
:1076280043F0BF6343F40033CB60704700ED00E0E4
:10763800164B30B5DC68C4F30224C4F10703251DDA
:10764800042B28BF0423062D4FF0FF358CBF033CC5
:10765800002405FA03F321EA0303A54022EA050200
:10766800A340002843EA0203ACBF00F16040084A87
:107678004FEA0313B8BF00F00F00DBB2AABF00F552
:107688006140135480F8003330BD00BF00ED00E0C6
:1076980014ED00E0002807DB044A4109012300F04B
:1076A8001F00834042F82130704700BF00E100E02E
:1076B80000280CDB4309064900F01F002033012293
:1076C800824041F82320BFF34F8FBFF36F8F70477D
:1076D80000E100E070B5D0E913456560446D14B170
:1076E800D0E916456560D0E9105404F01C06012461
:1076F800B4406C60046863608368102B0BBFA260A1
:10770800A160E160E26070BD0268416CD3B210B55F
:10771800083B1424B3FBF4F30B4CA24288BF0B4A7A
:1077280021F0030199BF01F1804202F5023252189B
:1077380007338264064AC26403F01F03012202FA77
:1077480003F3036510BD00BF070402401C08024094
:107758008008024038B500285ED002682F4B9A4254
:107768004FF014014CD82E4B1344B3FBF1F32D49C1
:107778009B00C0E91013022380F8253013680569BF
:1077880023F4FF4323F070031360D0E9024323433B
:107798002B43456911682B4385692B43C5692B43E6
:1077A800056A2B430B431360FFF7AEFFB4F5804F18
:1077B80004BF002343604268816C02F07F030B60C2
:1077C800D0E91314013A032A4C6020D8164A174905
:1077D80081651A44013B9200012103F0030301FA79
:1077E80003F300214265C3651160114A5364002305
:1077F8000122C36380F8243080F82520184638BD5C
:107808000C4B1344B3FBF1F30B499B00B1E7002386
:10781800C0E91533C365EAE70120F0E70704024031
:10782800F8FFFDBF000002403F82001040090240FF
:1078380000090240F8FBFDBF0004024038B50028EB
:1078480041D00268136823F0010313601F4B9A426A
:107858004FF0140130D81E4B1344B3FBF1F31D490C
:107868009B00C0E91013012403F01C0304FA03F37E
:10787800002515604B60FFF747FF836C41681D606A
:10788800D0E913325A604A1E032A06D8124B0B4419
:107898009B0094401D60114B5C640023C363C0E9E6
:1078A8001533C0E90B33C0E90D33C36580F82530C3
:1078B80080F82430184638BD094B1344B3FBF1F364
:1078C80008499B00CDE70120F5E700BF0704024007
:1078D800F8FFFDBF000002403F820010000902408F
:1078E800F8FBFDBF0004024070B590F82450012D4C
:1078F80004463BD090F825600125AE4280F824501C
:107908004FF000062CD1022580F825500568C66383
:107918002E6826F001062E60FFF7DCFE036BBBB174
:107928002B6843F00E032B60A36C1A68D20342BF86
:107938001A6842F480721A60636D1BB11A6842F4C7
:1079480080721A602B6843F001032B60002070BD21
:107958002B6823F004032B602B6843F00A03E2E74B
:107968008023C36380F824602846F0E70220EEE70E
:10797800034640B190F82520022A06D00422C263AB
:10798800002280F82420012070470268806C11686A
:1079980021F00E011160016821F480710160116805
:1079A80021F001011160D3E9100202F01C0101224B
:1079B8008A404260D3E9132151605A6D32B111688F
:1079C80021F480711160D3E9162151600122002051
:1079D80083F8252083F82400704710B590F82530E7
:1079E800022B03D00423C363012010BD03681A6867
:1079F80022F00E021A601A6822F001021A60826CE4
:107A0800136823F480731360D0E9101303F01C0289
:107A1800012393404B60D0E913325A60436D33B170
:107A28001A6822F480721A60D0E916325A6001236B
:107A380080F82530836B002480F8244013B19847E0
:107A48002046D2E71846D0E770B4426C046C03684D
:107A580026681D6802F01C020421914031420FD0B3
:107A680015F0040F0CD01A6892065EBF1A6822F04F
:107A780004021A60036B6160002B33D070BC184796
:107A880002219140314217D015F0020F14D01A6824
:107A9800940606D41A6822F00A021A60012280F8B5
:107AA8002520114A93428CBF104B114B596000237B
:107AB80080F82430C36ADFE708219140314211D0B1
:107AC80029070FD5196821F00E011960012303FA5F
:107AD80002F26260C36380F82530002380F8243006
:107AE800436BC9E770BC7047800002400004024045
:107AF800000002400A4A536943F4802330B55361B9
:107B0800EFF3108472B60023CD58C5500433B3F593
:107B1800807FF9D11369DB03FCD484F3108830BD6E
:107B280000400058064B5A69002ABFBF054A9A60B0
:107B380002F188329A60BABF5869C00F00207047B6
:107B48000040005823016745044B5A6942F000423F
:107B58005A615869C043C00F704700BF00400058C1
:107B680070B50546FAF7D6FF124E04463369D903B5
:107B780013D43369DA0744BF012232614CF2FA3276
:107B8800134011D10B4E306910F480200BD0FAF756
:107B9800C1FF001BA842F6D304E0FAF7BBFF001BA5
:107BA800A842E3D3032070BD024A1361024A0120B0
:107BB8005360F8E700400058300F00202DE9F041ED
:107BC800184D98462B78012B06460C46174626D0AA
:107BD80001232B704FF47A7000236B60FFF7C0FF0E
:107BE800A0B9012E16D1104A536943F0010353611D
:107BF8002760BFF36F8FC4F804804FF47A70FFF7E3
:107C0800AFFF094A536923EA0603536100232B7027
:107C1800BDE8F08139462046FFF76CFFEDE702200A
:107C2800F6E700BF300F002000400058054A5369AE
:107C380023F47E7343EAC00040F4803040F0020031
:107C480050617047004000582DE9F041234F3B78C0
:107C5800012B054688463FD001233B704FF47A70CC
:107C680000237B60FFF77CFF044688B92B68042B50
:107C780013D11B4A536943F4803343F0040353611F
:107C88004FF47A70FFF76CFF0446154B1A681B68AF
:107C980000233B702046BDE8F0814FF0FF33C8F861
:107CA80000306E68D5E901321344B3420AD9304630
:107CB800FFF7BCFF4FF47A70FFF752FF50B1C8F8D6
:107CC80000600446064A536923F47E7323F00203D6
:107CD8005361DAE70136E5E70224DBE7300F0020DD
:107CE800004000582DE9F04F524C00234FF00F0987
:107CF8000A6832FA03F501D1BDE8F08F012505FACB
:107D080003F818EA020200F08E804E68032706F096
:107D180003054FEA430E07FA0EFC6F1E012F6FEAA8
:107D28000C0C32D8876807EA0C0ACF6807FA0EF7F6
:107D380047EA0A078760476827EA0808C6F3001772
:107D48009F4047EA08074760C76807EA0C088F683A
:107D580007FA0EF747EA0807022DC76017D14FEA5E
:107D6800D30800EB880803F0070AD8F820704FEA18
:107D78008A0A09FA0AFB27EA0B0B0F6907FA0AF7BE
:107D880047EA0B07C8F8207001E0032DDCD107682B
:107D980005FA0EF507EA0C073D4316F4403F056067
:107DA80041D023F0030707F1804707F5803703F038
:107DB800030CBD684FEA8C0C4FF0070E0EFA0CFE50
:107DC800B0F1904F25EA0E0E2FD01B4DA8422ED0B1
:107DD80005F58065A8420CBF0225072505FA0CF5B4
:107DE80045EA0E05BD602568D74316F4801F0CBF11
:107DF8003D4015432560656816F4001F0CBF3D40E3
:107E080015436560D4F8805016F4803F0CBF3D40A0
:107E18001543C4F88050D4F88450B60354BF3D408D
:107E28001543C4F88450013362E70025D6E70125DD
:107E3800D4E700BF0008005800040048374A2DE97D
:107E4800F04F00234FF0010A4FF0070B4FF00F09D6
:107E580031FA03F401D1BDE8F08F0AFA03FC1CEAF9
:107E6800010654D023F0030404F1804404F580345F
:107E780003F00307A568BF000BFA07F8B0F1904FAD
:107E880008EA050E45D0264DA84244D005F5806580
:107E9800A8420CBF02250725BD40754517D1D2F869
:107EA800805025EA0605C2F88050D2F8845025EAA9
:107EB8000605C2F88450156825EA06051560556858
:107EC80025EA06055560A56825EA0805A560056840
:107ED80003265C0006FA04F423FA06F6254300EBB1
:107EE8008606056003F00705376AAD0009FA05F54F
:107EF80027EA05073762856825EA0405856045682D
:107F080025EA0C054560C56825EA0404C460013308
:107F18009EE70025C0E70125BEE700BF000800581E
:107F2800000400480369194214BF0120002070476B
:107F38000AB181617047816270470000044AD168C4
:107F4800014208B502D0D060FBF71CFB08BD00BF9A
:107F58000008005803689A69910744BF00229A6292
:107F68009A69D2075EBF9A6942F001029A61704726
:107F780030B5039D04682B4343EA0243064A606810
:107F8800C1F309010B4342EA555223F0004320EAAA
:107F980002000343636030BDFF63FF0303682DE9FC
:107FA800F0419C6914F0100405460F4616466FD040
:107FB80010220024DA61A0462B689A69900661D4E1
:107FC800B8F1000F35D044F0040401202E68B369DD
:107FD800D90541BF4FF48072F26144F001040120D9
:107FE8005A0541BF4FF4806244F00804F261012051
:107FF8009B054FD54FF4007344F00204F361284603
:10800800FFF7A8FF736823F0FF7323F48B3323F47F
:10801800FF7323F0010373606B6C23436B642023AD
:1080280085F84130002385F8423085F8403001203A
:1080380032E07A1CC1D0FAF76DFD801BB84201D836
:10804800002FB9D12B68596895F842209869000427
:10805800D2B20AD5490408D4202A06D05A6842F474
:1080680080425A60FAF756FD06462B689B699B06C4
:10807800A2D4FAF74FFD801B1928F6D920244FF017
:10808800010899E7B8F1000F9DD12022DA619AE73B
:1080980020469BE70028B2D1BDE8F08170B50446C0
:1080A8000D46164623689B699B0701D5002070BDC5
:1080B800324629462046FFF771FFA0B96A1CF1D065
:1080C800FAF728FD801BA84201D8002DEAD1636C7D
:1080D80043F020036364202384F84130002384F8AC
:1080E800423084F840300120E1E770B504460D467F
:1080F800164623689B695B070ED4324629462046FC
:10810800FFF74CFF38BB23689A69910625D59A6911
:10811800520703D5228D0AB1002070BD9A6912F06A
:1081280010021CBF1022DA614FF0200118BF042290
:108138006264D9615A6822F0FF7222F48B3222F409
:10814800FF7222F001025A60002384F8411084F87B
:10815800423084F840300120DFE7FAF7DBFC801B6F
:10816800A84201D8002DC4D1636C43F02003636496
:10817800202384F841300023EBE72DE9F041069FE6
:108188000446884616461D462268936938EA030362
:108198000CBF01230023B34201D0002015E06B1C63
:1081A800F3D0FAF7B7FCC01BA84201D8002DEBD1D9
:1081B800636C43F020036364202384F84130002378
:1081C80084F8423084F840300120BDE8F08170B571
:1081D80004460D46164623689B699B0601D5002078
:1081E80070BD324629462046FFF7D8FE90B9FAF707
:1081F80091FC801BA84201D8002DECD1636C43F0A0
:1082080020036364202384F84130002384F842303B
:1082180084F840300120E3E710B5044600284AD02E
:1082280090F8413003F0FF021BB980F84020FAF7BC
:108238006DF9242384F8413023681A6822F001027A
:108248001A60626822F070621A619A6822F4004229
:108258009A60D4E90221012924D142F400429A60AB
:108268005A6842F0007242F400425A60DA6822F416
:108278000042DA60D4E904210A43A16942EA0122F2
:10828800DA60D4E907210A431A601A6842F0010249
:108298001A6000202023606484F84130206384F849
:1082A800420010BD42F4044202299A6004BF4FF410
:1082B80000625A60D4E70120F3E700002DE9F34794
:1082C800984690F841300A9F202B04460E46914666
:1082D80040F0868090F84030012B00F081804FF00C
:1082E800010A80F840A0FAF715FC1923054600900A
:1082F80052464FF400412046FFF73FFF18B10120D6
:1083080002B0BDE8F087212384F84130102384F8B7
:1083180042306064A4F82A80638DC4F824909BB22C
:10832800FF2B60632F4B26D9FF22228500934FF045
:10833800807331462046FFF71BFE638D9BB22A46A9
:1083480039462046FBB9FFF742FF0028D7D12368FA
:108358002021D9615A6822F0FF7222F48B3222F46C
:10836800FF7222F001025A6084F8411084F840003C
:1083780084F84200C4E7628D009392B222854FF0E0
:108388000073D2B2D5E7FFF789FE0028B7D1636A38
:10839800226813F8011B91626362638D228D013B91
:1083A8009BB26385638D013A92B29BB22285002B02
:1083B800C3D0002AC1D100953B4680212046FFF753
:1083C800DCFE00289BD1638D9BB2FF2B03D9FF22D3
:1083D80022850090ABE7628D009092B22285CEE7AD
:1083E80002208DE7002000802DE9F347984690F899
:1083F80041300A9F202B04460E46914640F0878064
:1084080090F84030012B00F082804FF0010A80F88C
:1084180040A0FAF77FFB19230546009052464FF417
:1084280000412046FFF7A9FE18B1012002B0BDE8BF
:10843800F087222384F84130102384F842306064A6
:10844800A4F82A80638DC4F824909BB2FF2B606344
:10845800304B26D9FF22228500934FF08073314696
:108468002046FFF785FD638D9BB22A463946204694
:10847800FBB9FFF7ACFE0028D7D123682021D961CA
:108488005A6822F0FF7222F48B3222F4FF7222F033
:1084980001025A6084F8411084F8400084F84200D0
:1084A800C4E7628D009392B222854FF00073D2B276
:1084B800D5E7FFF71AFE0028B7D123685A6A636A1E
:1084C8001A70636A228D01336362638D013B9BB22C
:1084D8006385638D013A92B29BB22285002BC2D08C
:1084E800002AC0D100953B4680212046FFF745FE73
:1084F80000289AD1638D9BB2FF2B03D9FF222285D6
:108508000090AAE7628D009092B22285CDE7022002
:108518008CE700BF0024008010B590F84120202A85
:108528000346D4B21CD190F84020012A18D0242246
:1085380080F841200268106820F00100106010687F
:1085480020F4805010601068014311601168002009
:1085580041F00101116083F8414083F8400010BDEB
:108568000220FCE710B590F84120202A0346D4B237
:108578001BD190F84020012A17D0242280F84120EE
:108588000268106820F001001060106820F4706024
:1085980040EA012111601168002041F001011160D9
:1085A80083F8414083F8400010BD0220FCE700003A
:1085B800024A136843F4807313607047000400583C
:1085C8000D4B10B55B690C4628B99A0507D500F024
:1085D80027F820B110BD9B0501D400F019F8074A0F
:1085E8001369012C23F00403136101D130BFF1E7B3
:1085F80040BF20BF20BFEDE70004005800ED00E0B9
:10860800024B186800F4C060704700BF00040058AF
:10861800024A136843F4804313607047000400580B
:108628000C4A136823F4804313600B4B1B683221F8
:108638004B430A49B3FBF1F35169890500D533B9B6
:10864800536913F4007F14BF032000207047013BD7
:10865800F2E700BF000400582808002040420F003D
:108668000B4A136823F0070343F002031360094B16
:108678001A69012842F004021A6105D130BF1A694B
:1086880022F004021A61704740BF20BF20BFF6E7FE
:108698000004005800ED00E04FF0B0431868C0F344
:1086A800404070474FF0B0431868C0F3400070472F
:1086B8004FF0B042536823F47F4343EA00235360EA
:1086C80070474FF0B0431868C0F34060704700002F
:1086D8007FB54FF0B0432C4AD3F80831C0F30310EC
:1086E80003F00F0352F82040284A52F82330B4FB15
:1086F800F3F4FFF785FF264B054693E80700B5F529
:10870800007F04AB03E9070010D0224B9C4218D32A
:1087180003F5B70303F67F539C4229D903F5741375
:1087280003F510639C4225D802230BE01A4B9C42A8
:1087380007D91A4B9C421BD903F5370303F5D853C5
:10874800F0E7002304AA02EB830353F80C4C144D02
:108758002B6823F0070323432B60FAF7DBF906465F
:108768002B6803F007039C4206D1002004B070BDBB
:108778000123E7E70024EAE7FAF7CCF9801B02288F
:10878800EED90320F2E700BF34420108D4410108C2
:1087980070400108C0CF6A00BFEA21013F9334024C
:1087A800004000584FF0B04310B59A68D96812F0ED
:1087B8000C0205D00C2A4AD101F00303012B50D139
:1087C8004FF0B0412B480B6813F0080306D00B6834
:1087D80013F0080337D1D1F8941007E00C68240788
:1087E80056BFD1F894300968C3F3032350F82330F7
:1087F800002A0CBF184600204FF0B0418A6802F0EA
:108808000C020C2A1ED1CA6802F00302022A2ED0DA
:10881800032A06D10B68184A13F4801F174B18BF98
:1088280013464FF0B042D068D168D268C0F3062032
:108838005843C1F302130133B0FBF3F0530F013374
:10884800B0FBF3F010BD0B68C3F30313CEE7042AA3
:108858000AD0082A05D11B6813F4801304D10748ED
:10886800CAE700231846C7E703480023C4E7024BBA
:10887800D7E700BF344201080024F4000048E801AB
:1088880008B5FFF78FFF4FF0B043044A9B68C3F366
:10889800031352F82330B0FBF3F008BDD4410108AC
:1088A8002DE9F0410446002853D04FF0B0439D68AD
:1088B800DE6803689B0605F00C0506F0030668D51C
:1088C800026A1DB10C2D46D1012E44D1002A40D098
:1088D8004FF0B043A16A1A68170756BFD3F894300F
:1088E8001B681B0903F0F00399421FD90846FFF7DC
:1088F800EFFE00282DD14FF0B042136843F0080373
:1089080013601368A16A23F0F0030B431360606AD5
:10891800FFF7CEFEFFF7B4FFAB4B1860AB4B186800
:10892800FAF7F6F8002834D0BDE8F0814FF0B042ED
:10893800136843F008031360136823F0F0030B4334
:108948001360606AFFF7B4FE0846FFF7C1FE00280F
:10895800E0D00120E8E74FF0B043002A54D01A686D
:1089680042F001021A60FAF7D5F80746FFF79AFEB7
:10897800002842D04FF0B042136843F00803136058
:108988001368A16A23F0F0030B431360606AFFF7D2
:108998008FFE2368D80748D42368990700F18C8094
:1089A80023681E0740F1FA80A3694FF0B046002BF8
:1089B80000F0E180D6F89430E16903F010029142AA
:1089C80000F0C48003F00302022AC2D0D80740F1A5
:1089D800B380D6F8943023F00103C6F89430FAF740
:1089E80099F80746D6F89430990740F1A580FAF728
:1089F80091F8C31B112BF5D904E0FAF78BF8C01BCB
:108A08000228B3D903208FE71A6822F001021A60FE
:108A1800FAF780F80746FFF745FE0028B9D0FAF7BD
:108A280079F8C01B0228F6D9ECE7082D03D00C2DE5
:108A380005D1032E03D16368002BADD189E74FF030
:108A4800B043A1681A6822F480120A431A60626867
:108A5800B2F5803F10D11A6842F480321A60FAF7F2
:108A680059F80746FFF718FE002895D1FAF752F88B
:108A7800C01B6428F6D9C5E7B2F5041F04D11A68EB
:108A880042F400121A60E6E7196821F4803119608F
:108A9800196821F400111960002AE0D1FAF73AF8B0
:108AA8000746FFF7F9FD00283FF476AFFAF732F8EA
:108AB800C01B6428F5D9A5E7042D236903D00C2D24
:108AC8000ED1022E0CD1002B3FF443AF4FF0B04231
:108AD8006169536823F0FE4343EA016353605FE72B
:108AE8004FF0B046BBB1336843F480733360FAF794
:108AF80011F8074633685A0507D57368626923F089
:108B0800FE4343EA026373604AE7FAF703F8C31BBC
:108B1800022BEFD976E7336823F480733360F9F7D3
:108B2800F9FF074633685B057FF53AAFF9F7F2FFBF
:108B3800C31B022BF6D965E74FF0B042E169D2F8C2
:108B4800943023F010030B43C2F894304FF0B04731
:108B5800D7F8943043F00103C7F89430F9F7DAFFF7
:108B68000646D7F894309A0718D4F9F7D3FF831B31
:108B7800112BF6D946E7D6F8943023F00103C6F84E
:108B88009430F9F7C7FF0746D6F894309B0705D508
:108B9800F9F7C0FFC31B112BF6D933E72368580731
:108BA80054D50B4F3B68D90514D4FFF701FDF9F7ED
:108BB800B1FF06463B68DA050CD4F9F7ABFF831B17
:108BC800022BF7D91EE700BF280800202C08002038
:108BD80000040058E3684FF0B046002B58D023F04B
:108BE8008003052B02BFD6F8903043F00403C6F883
:108BF80090304FF0B046F9F78DFFD6F8903043F03B
:108C080001030746C6F8903041F28838D6F890300C
:108C18009B0705D4F9F77EFFC31B4345F6D9F1E658
:108C2800E36823F00403812B1BD1F9F773FFD6F80F
:108C3800903043F08003C6F8903007464FF0B046B6
:108C480041F28838D6F89030180504D5E06A002833
:108C58004AD1002068E6F9F75DFFC01B4045F1D90D
:108C6800D0E6F9F757FFD6F8903023F08003C6F81E
:108C7800903007464FF0B04641F28838D6F8903029
:108C88001905E3D5F9F746FFC01B4045F6D9B9E603
:108C9800F9F740FFD6F8903023F080030746C6F86E
:108CA800903041F28838D6F890301A0516D4F9F782
:108CB80031FFD6F8903023F00103C6F8903007460C
:108CC8004FF0B04841F28836D8F890309B07BDD5B0
:108CD800F9F720FFC31BB342F6D993E6F9F71AFF59
:108CE800C01B4045DFD98DE60C2D4ED04FF0B04368
:108CF80002281A6822F080721A6033D1F9F70AFF45
:108D08000546FFF7DEFC38BBD4E90C314FF0B04222
:108D18000B43D0682D4901400B43E16B0B43216C99
:108D28000B43616C0B43A16B43EA0123D3601368C7
:108D380043F080731360D36843F08053D360F9F72E
:108D4800E9FE0446FFF7BDFC002882D1F9F7E2FEF0
:108D5800001B0A28F6D955E6F9F7DCFE401B0A285D
:108D6800CFD94FE6F9F7D6FE0446FFF7AAFC30B98B
:108D78004FF0B042164BD1680B40D360D4E5F9F7F9
:108D8800C9FE001B0A28F0D93CE601283FF4CCAD07
:108D98004FF0B043226BDB6803F0030191427FF48C
:108DA800D8AD616B03F070028A427FF4D2ADA16B3B
:108DB80003F4FE42B2EB012F7FF4CBAD626C03F0FB
:108DC800604393423FF445AFC3E500BF8C80C111B7
:108DD800FCFFFEEE2DE9F0410D46044610B90120D6
:108DE800BDE8F081684E336803F007038B4216D361
:108DF80023689A0727D54FF0B047A268BB6823F0CD
:108E0800F0031343BB60F9F785FE0646BB68DB0336
:108E180019D4F9F77FFE831B022BF7D911E03368C9
:108E280023F007030B433360F9F774FE07463368F2
:108E380003F00703AB42DBD0F9F76CFEC01B022836
:108E4800F5D90320CCE72368580617D54FF0B0476B
:108E58006269D7F8083123F00F0343EA1213C7F801
:108E68000831F9F757FE0646D7F80831D90305D473
:108E7800F9F750FE831B022BF6D9E2E723685A075D
:108E880013D54FF0B047E268BB6823F4E06313439F
:108E9800BB60F9F73FFE0646BB689B0305D4F9F7AC
:108EA80039FE831B022BF7D9CBE72368180714D5A3
:108EB8004FF0B0472269BB6823F4605343EAC2030A
:108EC800BB60F9F727FE0646BB68590305D4F9F7D6
:108ED80021FE831B022BF7D9B3E72368DA070FD4E7
:108EE800294C236803F00703AB4239D8FFF7C8FCC5
:108EF800264B1860264BBDE8F0411868F9F708BE04
:108F08006268022A1DD1FFF7C7FB00283FF467AF4C
:108F18004FF0B04641F28838B36823F00303134397
:108F2800B360F9F7F7FD0746B368626803F00C030E
:108F3800B3EB820FD4D0F9F7EDFDC01B4045F3D950
:108F48007FE7032A02D1FFF7BCFBDEE712B9FFF780
:108F5800A9FBDAE74FF0B0431B685B05D8D43EE7BE
:108F6800236823F007032B432360F9F7D3FD064654
:108F7800236803F00703AB42B8D0F9F7CBFD801B99
:108F88000228F5D95DE700BF0040005828080020F6
:108F98002C08002008B5FFF773FC4FF0B043044AD3
:108FA8009B68C3F3022352F82330D84008BD00BFA2
:108FB8001442010808B5FFF763FC4FF0B043044AB8
:108FC8009B68C3F3C22352F82330D84008BD00BFC2
:108FD800144201084FF0B043D3F89000C0F34000AA
:108FE80070474FF0B0410209D1F8883002F47F226F
:108FF800000123EA020300F47F200343C1F888300C
:1090080070474FF0B041020CD1F88830120423EABF
:10901800020343EA0040C1F88800704770B506684B
:1090280016F48036044638D0FFF7C2FAF9F772FD15
:10903800614E05463368DB0529D54FF0B043616BB7
:10904800D3F8902002F44072914214D0D3F89010D3
:10905800D3F8902042F48032C3F89020D3F89020BF
:1090680021F4407022F480328D07C3F89020C3F8B1
:10907800900000F190804FF0B042616BD2F89030D0
:1090880023F440730B43C2F89030002605E0F9F74B
:1090980041FD401B0228CDD903262568E8070AD5DB
:1090A8004FF0B0416268D1F8883023EA124392B297
:1090B8001343C1F88830A9070AD54FF0B041A26818
:1090C800D1F8883023EA124392B21343C1F88830AA
:1090D800AA0609D54FF0B0422169D2F8883023F4A6
:1090E80040630B43C2F88830AB0502D5206AFFF70E
:1090F80088FF680502D5606AFFF783FF290502D556
:10910800A06AFFF77EFF6A0602D56069FFF769FF6C
:109118002B0602D5A069FFF764FFE80502D5E069D0
:10912800FFF75FFFE90610D54FF0B042E168D2F8CB
:10913800883023F440730B43C2F88830B1F5807F40
:1091480002BFD36843F08073D3602A040ED54FF072
:10915800B042216BD2F8883023F040430B43C2F869
:10916800883019B9D36843F08073D3606B0410D585
:109178004FF0B042E16AD2F8883023F040530B43F5
:10918800B1F1005FC2F8883003D1D36843F480336B
:10919800D360304670BDF9F7BDFC41F2883605460C
:1091A800FFF718FF01283FF466AFF9F7B3FC401B3F
:1091B800B042F5D970E700BF0004005830B590F808
:1091C8002C30012B02464FF0020022D0174B82F8B8
:1091D8002D00CA24012582F82C505C6253245C625D
:1091E800B1F5807F146B996914D121F48851996184
:1091F800596C24F0010421F0004159641463DD65C1
:109208000A4BFF2159620020012382F82D3082F891
:109218002C0030BD21F408519961D96C24F0020466
:1092280021F00041D9641463D865E9E700280040BB
:1092380070B50B4E036B756D1D40EA07044603D5E8
:109248000123F365F9F7D7FDAB0704D50223F365CE
:10925800204600F0CBF9012384F82D3070BD00BF03
:109268000028004038B50A4CE36823F02003E36087
:10927800F9F750FC0546E3689B0601D5002038BD88
:10928800F9F748FC401BB0F57A7FF4D90320F6E7DC
:10929800002800402DE9F041114DEC6814F040041D
:1092A80007461AD1EB6843F08003EB60F9F732FC0C
:1092B8004FF003080646EB685B0601D4032C02D185
:1092C8002046BDE8F081F9F725FC801BB0F57A7FD0
:1092D80084BF87F82D800324EDE70024F0E700BF62
:1092E8000028004038B50F4CE36823F08003E360A2
:1092F800A3699B06054606D4FFF7B4FF10B1032007
:1093080085F82D0038BDA36923F02003A361FFF77A
:10931800A9FF10B1032085F82D00A36943F02003AD
:10932800A361EFE70028004038B5044600284BD079
:1093380090F82D3003F0FF021BB980F82C20F9F7C4
:10934800F1F90223214D84F82D30EB68DB0632D485
:10935800CA236B6253236B622046FFF79BFF78BBDF
:10936800AB6923F08E6323F04003AB612169636826
:10937800AA690B431343A2691343AB61D4E90223DF
:1093880043EA02432B61D4E90931EA680B4322F42A
:10939800F8521343EB602046FFF7A4FF80B9D4E9E5
:1093A8000713AA690B4322F060421343626913430F
:1093B800AB61FF236B62012384F82D30002002E0AB
:1093C800024BFF225A6238BD0120FCE7002800400A
:1093D8000023092803D840EA0310C0B270470A38AE
:1093E8000133C0B2F5E700002DE9F04790F82C30C2
:1093F800012B05464FF0020069D0012385F82C3077
:109408004E4B85F82D00DE6806F44076B6F5807F71
:1094180078D04C69087891F8019091F802A091F8F9
:109428002470002A55D19B6913F0400308BFCB7004
:10943800FFF7CEFF80464846FFF7CAFF0246504670
:10944800FFF7C6FF81463846FFF7C2FF0B6ACF78A1
:10945800234343EA875343EA090343EA084343EAB9
:10946800022343EA0063354ACA20506253205062FF
:109478008C6A8869B4F5807F946945D124F488544E
:1094880094610124D465B6F5807F09BFCB69136464
:109498000343536418BF5064284B4A681A672A6B01
:1094A80042F001022A639A6942F488529A61244A76
:1094B800D2F8803043F40033C2F880301F4BFF22CB
:1094C8005A620020012385F82D3085F82C00BDE86C
:1094D800F087B4F1803F07D0B4F5000F04D09B6942
:1094E80013F0400308BFCB700B6ACA781C4344EAE8
:1094F8000A0444EA004343EA092343EA825343EA5D
:109508000763B0E70023AEE724F40854946102240B
:10951800D465B6F5807F09BFCB6993640343D364F0
:1095280018BFD064054B4A685A672A6B42F002029A
:109538002A639A6942F40852B8E700BF002800403D
:109548000008005890F82C20012A03464FF002002A
:1095580012D00A4A83F82D00CA2151625321516260
:10956800916941F020019161FF215162002001229F
:1095780083F82D2083F82C00704700BF0028004096
:1095880090F82C20012A03464FF0020019D00D4A0A
:1095980083F82D00CA2151625321516291690A480A
:1095A80041F080019161D0F8801041F48021C0F829
:1095B8008010FF2151620020012283F82D2083F8BA
:1095C8002C0070470028004000080058064B5A6DD0
:1095D800520610B5044603D54022DA65F9F70EFCA9
:1095E800012384F82D3010BD002800407047890001
:1095F80001F1804101F531410A607047890001F1AC
:10960800804101F53141086870470000034AD2F8EB
:10961800903043F40043C2F890307047000400587B
:10962800034AD2F8903023F40043C2F890307047D0
:1096380000040058074B1A6822F040021A6040F4F0
:1096480041704FF4B85218605A601A6842F04002EC
:109658001A6070470000015837B5054600284ED0FB
:10966800837903F0FF046BB1032C0BD0254B4FF427
:1096780000629A612868FFF7DDFF002401232B713F
:10968800AC602FE000236B712846F9F75BF91E4A9E
:10969800D2F8903043F48053C2F89030002CE5D1D2
:1096A80002234FF0B042AB71D2F8943023F4004358
:1096B800C2F89430154B1B681C214B43DB0C64210A
:1096C8004B430193019B93B90124AC60FFF79EFFC4
:1096D8000C4B9A6842F400629A604FF400629A61F7
:1096E800002CC7D00123AB71204603B030BD019BCD
:1096F800013B0193D2F894305B04E3D4E6E70124FC
:10970800F2E700BF000400580008005828080020AD
:1097180037B5174D2B6802461C204343DB0C6420E9
:10972800434314480193019B93B901209060114C65
:1097380021732B681C214B43DB0C64214B430193A1
:10974800019B6BB9012090600A4BDB6803B030BD08
:10975800019B013B019383689C07E4D50020E6E761
:10976800019B013B0193A368DB07E9D5ECE700BF48
:10977800280800200000015837B5184D2B6802460C
:109788001C204343DB0C6420434315480193019B91
:10979800A3B901209060124CFF2323732B681C256A
:1097A8006B43DB0C64256B430193019B73B9012068
:1097B80090600B4BDB680B7003B030BD019B013B25
:1097C800019383689C07E2D50020E4E7019B013BF5
:1097D8000193A368DB07E8D5EBE700BF2808002062
:1097E800000001580F4B13B51B680F4C1822534348
:1097F8001B0D64225343014601936269019B02F0E9
:10980800040223B902238B60012002B010BD019B22
:10981800013B0193606910F00200F6D0002AECD1F8
:109828001046F2E7280800200004005807B503791D
:10983800012B0FD10A4B1B68182253431B0C0193B1
:10984800FFF7EEFE019B013B0193019B002BF9D131
:10985800FFF7DCFE03B05DF804EBFFF7C3BF00BF02
:1098680028080020F8B51E468379012B15460446C2
:109878000F46DAB22DD14379012B2AD00223427147
:109888008371FFF7D3FF0D212046FFF7C9FEFFF7CD
:109898003FFF390A2046FFF73BFFF9B22046FFF7A2
:1098A80037FF2E44B5420ED12046FFF7AFFEFFF733
:1098B80099FFA06801230038A3714FF0000318BF77
:1098C80001206371F8BD15F8011B2046FFF720FF42
:1098D800E8E70220F6E7F8B51E468379012B15461E
:1098E80004460F46DAB22FD14379012B2CD04271AE
:1098F800FFF79CFF1D212046FFF792FEFFF708FFA8
:10990800390A2046FFF704FFF9B22046FFF700FFA7
:1099180000212046FFF7FCFE2E44B5420ED120461A
:10992800FFF774FEFFF75EFFA06801230038A371FC
:109938004FF0000318BF01206371F8BD2946204687
:10994800FFF71AFF0135E8E70220F6E7F8B51F46EA
:109958008379012B154604460E46DAB22CD1437999
:10996800012B29D04271FFF761FF06F0EF03A3F145
:10997800840253425341237131462046FFF750FE7B
:10998800FFF7C6FE2F44AF4210D1FFF73FFE842EEB
:1099980002D02046FFF726FFA06801230038A371F4
:1099A8004FF0000318BF01206371F8BD15F8011BC3
:1099B8002046FFF7ADFEE6E70220F6E7F8B51E46BB
:1099C8008379012B154604460F46DAB227D143792D
:1099D800012B24D04271FFF729FF39462046FFF7B3
:1099E8001FFEFFF795FE00212046FFF791FE2E444B
:1099F800B5420ED12046FFF709FEFFF7F3FEA06837
:109A080001230038A3714FF0000318BF01206371D0
:109A1800F8BD29462046FFF7AFFE0135E8E70220EA
:109A2800F6E737B50023ADF8043001AA0223122166
:109A38000546FFF7C3FFBDF80440022364BA01AA34
:109A4800A4B219462846FFF781FFE20702D5284647
:109A580009F088FBA30702D5284609F089FB6007AF
:109A680002D5284609F0AEFB210702D5284609F0A1
:109A7800AFFBE20602D5284609F0B0FBA30602D5E3
:109A8800284609F099FB600602D5284609F076FBBE
:109A9800210606D514F4807118BF0121284609F063
:109AA80073FBA20502D5284609F07EFB630402D5A4
:109AB800284609F099FB03B030BDF8B51E468379F6
:109AC800012B154604460F46DAB227D14379012BFC
:109AD80024D04271FFF7AAFE0E212046FFF7A0FD11
:109AE800FFF716FE39462046FFF712FE2E44B54210
:109AF8000ED12046FFF78AFDFFF774FEA068012308
:109B08000038A3714FF0000318BF01206371F8BD3E
:109B180015F8011B2046FFF7FBFDE8E70220F6E7F2
:109B2800F8B51E468379012B154604460F46DAB26E
:109B38002BD14379012B28D04271FFF777FE1E21E4
:109B48002046FFF76DFDFFF7E3FD39462046FFF796
:109B5800DFFD00212046FFF7DBFD2E44B5420ED184
:109B68002046FFF753FDFFF73DFEA06801230038AC
:109B7800A3714FF0000318BF01206371F8BD294697
:109B88002046FFF7F9FD0135E8E70220F6E702680D
:109B980052E8003F23F0C00342E800310268002980
:109BA800F5D102F1080353E8003F23F4000302F162
:109BB800080C4CE800310029F3D12023C0F8883084
:109BC8007047000010B5026852E8003F23F4907314
:109BD80042E8003102680029F5D10F4C02F1080370
:109BE80053E8003F234002F1080C4CE800310029FB
:109BF800F4D1C36E012B07D152E8003F23F01003C4
:109C080042E800310029F7D12023C0F88C30002326
:109C1800C366436710BD00BFFEFFFFEFF8B50446FB
:109C28001346D4F88850202D32D1F1B1EAB1E06F53
:109C3800A4F85620A4F8542000262122C4F89060E5
:109C48002165C4F88820226888B1124FC762124F74
:109C58000763124F2832C0E90D76FDF745FE30B193
:109C68001023C4F89030C4F8885001200FE023680E
:109C780040221A62226802F1080353E8003F43F0C9
:109C8800800302F1080141E800300028F3D1F8BD53
:109C98000220FCE7A99C0008F19C0008FD9C000834
:109CA80008B50346806A1B681B6813F0200317D1A8
:109CB800A0F85630026802F1080353E8003F23F089
:109CC8008003083242E8003102680029F2D152E8E4
:109CD800003F43F0400342E800310029F7D108BDB6
:109CE800F9F7E2F9FBE7704708B5806AFFF7FBFF71
:109CF80008BD7047806A38B50468D0F88830D0F855
:109D08008C50A268120606D5212B04D10023A0F896
:109D18005630FFF73CFFA3685B0606D5222D04D119
:109D28000023A0F85E30FFF74DFFD0F8903043F0E5
:109D38001003C0F89030FFF7DCFF38BD08B5806A23
:109D48000023A0F85E30A0F85630FFF7D2FF08BD18
:109D5800704700000368D9691A682DE9F04140F698
:109D68000F0631429D68044610D18E0640F1978057
:109D780002F0200605F080573E4300F09080436FC4
:109D8800002B00F08580BDE8F0411847AB4EAC4889
:109D98002E401040304300F08280CF0709D5D0050F
:109DA80007D501201862D4F8900040F00100C4F8EB
:109DB80090008F0709D5E80707D502201862D4F864
:109DC800900040F00400C4F890004F0709D5E80758
:109DD80007D504201862D4F8900040F00200C4F8B7
:109DE80090000F070BD502F02000304307D0082061
:109DF8001862D4F8900040F00800C4F890000E05EE
:109E08000AD5500108D54FF400601862D4F8903094
:109E180043F02003C4F89030D4F89030002B37D0AA
:109E28008B0609D502F0200205F080552A4303D09D
:109E3800636F0BB1204698472668D4F89020B36822
:109E480002F0280203F0400353EA0205204621D01D
:109E5800FFF7B8FEB3685F0617D5226802F108035A
:109E680053E8003F23F04003083242E8003100295C
:109E7800F3D1D4F8800040B1724B8363FDF7ADFD98
:109E880030B1D4F88000836B7DE72046FFF731FFBF
:109E9800BDE8F081FFF72DFFC4F89050F8E7E06EB9
:109EA800012840F08980CE0640F18680D00640F136
:109EB800838010221A629A6851064BD5D4F8802004
:109EC80011684A6892B2002AE2D0B4F85C00904265
:109ED800DED9A4F85E200A6892062FD453E8002F32
:109EE80022F4807243E800210029F7D103F1080227
:109EF80052E8002F22F0010203F1080040E8002197
:109F08000029F3D103F1080252E8002F22F04002A1
:109F180003F1080040E800210029F3D12022C4F809
:109F28008C20E16653E8002F22F0100243E800215C
:109F38000029F7D1D4F88000FDF71AFD0223236722
:109F4800B4F85E30B4F85C10C91A89B22046FFF73D
:109F5800FFFE9DE7B4F85E20B4F85E00B4F85C102C
:109F680080B292B2002893D0891A89B200298FD082
:109F780053E8002F22F4907243E800200028F7D11C
:109F8800314D03F1080252E8002F2A4003F1080678
:109F980046E800200028F4D12022C4F88C2060670D
:109FA800E06653E8002F22F0100243E80020002862
:109FB800F7D102232367C9E7CF0209D56E0207D577
:109FC8004FF4801220461A62BDE8F04100F0A0BDAF
:109FD80008060BD502F0800005F40005284305D0DB
:109FE800A36F002B3FF454AF2046CCE64F0611D5A3
:109FF80056060FD553E8002F22F0400243E800210F
:10A008000029F7D12023C4F88830A1672046F9F742
:10A018004BF83DE70D0206D5500004D52046BDE8B3
:10A02800F04100F077BDCB017FF532AF002ABFF6D3
:10A038002FAF2046BDE8F04100F06BBD01000010D5
:10A0480020010004459D0008FEFFFFEFD0F88C209A
:10A05800B0F86010222A08B5036855D15B6A826D92
:10A068000B401370836D01338365B0F85E30013B9C
:10A078009BB2A0F85E30B0F85E309BB2002B42D1A4
:10A08800026852E8003F23F4907342E80031036805
:10A098000029F5D103F1080252E8002F22F001024D
:10A0A80003F1080C4CE800210029F3D12022C0F864
:10A0B8008C20184A41679342016705D1C26E012A74
:10A0C8000ED0F8F7FFFF1EE05A681102F6D553E8E4
:10A0D800002F22F0806243E800210029F7D1EDE744
:10A0E8000022C26653E8002F22F0100243E8002144
:10A0F8000029F7D1DA69B0F85C10D20644BF102203
:10A108001A62FFF725FE08BD9A6942F008029A61B3
:10A11800F9E700BF00800040D0F88C20B0F860104C
:10A12800222A08B5036852D15A6A1140826D22F872
:10A13800021B8265B0F85E20013A92B2A0F85E2058
:10A14800B0F85E2092B2002A40D153E8002F22F4E2
:10A15800907243E800210029F7D103F1080252E880
:10A16800002F22F0010203F1080C4CE8002100291D
:10A17800F3D12022C0F88C20174A41679342016727
:10A1880005D1C26E012A0ED0F8F79CFF1EE05A686E
:10A198001102F6D553E8002F22F0806243E800212F
:10A1A8000029F7D1EDE70022C26653E8002F22F01C
:10A1B800100243E800210029F7D1DA69B0F85C10F1
:10A1C800D20644BF10221A62FFF7C2FD08BD9A6981
:10A1D80042F008029A61F9E7008000402DE9F74F44
:10A1E8000368B0F86080DF691A689D68D0F88C1041
:10A1F80001922229044640F0B480B0F86890DFF854
:10A208006CA1DFF86CB10026B9F1000F01D0BB06D4
:10A2180021D4B4F85E309BB2D3B1B4F868209A4226
:10A2280016D9226802F1080353E8003F23F080534F
:10A23800083242E8003122680029F2D14D4B6367A9
:10A2480052E8003F43F0200342E800310029F7D1EB
:10A2580003B0BDE8F08F2368A26D5B6A03EA0803C8
:10A268001370A36D0133A365B4F85E30013B9BB254
:10A27800A4F85E302368DF6978072CD0F9070AD57F
:10A28800019AD20507D501211962D4F8901041F03E
:10A298000101C4F89010B80709D5E90707D50221CC
:10A2A8001962D4F8901041F00401C4F890107A07AC
:10A2B80009D5E80707D504211962D4F8903043F08E
:10A2C8000203C4F89030D4F8903023B12046FFF749
:10A2D80010FDC4F89060B4F85E309BB2002B93D1A7
:10A2E800216851E8003F23F4807341E80030236877
:10A2F8000028F5D103F1080252E8001F01EA0A011B
:10A3080042E800100028F5D120215B45C4F88C10E4
:10A31800606720670AD05968090207D553E8001F0B
:10A3280021F0806143E800100028F7D1E16E01298F
:10A3380013D1E66653E8001F21F0100143E800102E
:10A348000028F7D1D969CA0644BF102119622046EE
:10A35800B4F85C10FFF7FCFC56E72046F8F7B2FEAD
:10A3680052E79A6942F008029A6171E7FEFFFFEF2F
:10A378000080004055A000082DE9F74F0368B0F8A9
:10A388006080DF691A689D68D0F88C1001922229D4
:10A39800044640F0B280B0F86890DFF868A1DFF8B2
:10A3A80068B10026B9F1000F01D0BB0621D4B4F87A
:10A3B8005E309BB2D3B1B4F868209A4216D92268AD
:10A3C80002F1080353E8003F23F08053083242E8C3
:10A3D800003122680029F2D14C4B636752E8003FF4
:10A3E80043F0200342E800310029F7D103B0BDE86B
:10A3F800F08F2368A26D596A08EA010122F8021B4E
:10A40800A265B4F85E20013A92B2A4F85E20DF6932
:10A4180078072CD0F9070AD5019AD20507D501216A
:10A428001962D4F8901041F00101C4F89010B807EF
:10A4380009D5E90707D502211962D4F8901041F02F
:10A448000401C4F890107A0709D5E80707D5042154
:10A458001962D4F8903043F00203C4F89030D4F86D
:10A46800903023B12046FFF744FCC4F89060B4F85C
:10A478005E309BB2002B95D1216851E8003F23F450
:10A48800807341E8003023680028F5D103F1080201
:10A4980052E8001F01EA0A0142E800100028F5D13D
:10A4A80020215B45C4F88C10606720670AD0596882
:10A4B800090207D553E8001F21F0806143E8001026
:10A4C8000028F7D1E16E012913D1E66653E8001F91
:10A4D80021F0100143E800100028F7D1D969CA0615
:10A4E80044BF102119622046B4F85C10FFF730FC15
:10A4F80058E72046F8F7E6FD54E79A6942F0080263
:10A508009A6173E7FEFFFFEF0080004021A1000879
:10A5180038B5044603682169A2681D68C0690A4302
:10A5280061690A437D49024329400A431A605A680F
:10A53800E16822F440520A435A60794AA169934279
:10A548001CBF226A11439A6822F06E4222F43062DC
:10A558000A439A60DA6A616A22F00F020A43DA62F1
:10A56800704A93421CD14FF0B043D3F8883003F0BF
:10A57800030343F44033A3F54033013B022B00F2BD
:10A58800C780694A9B5CB0F5004F40F08980082B72
:10A5980024D8DFE803F061C08323802323236500E8
:10A5A800624A934209D14FF0B043614AD3F88830E8
:10A5B80003F00C0343F44023E4E7594A93420DD1D6
:10A5C8004FF0B043D3F8883003F44063B3F5006F1D
:10A5D8001AD005D853B1B3F5806F12D0012009E025
:10A5E800B3F5406FFAD14FF400400EE0FEF7D2FC0D
:10A5F80058B900204FF00113A3660023C4E91D33A6
:10A6080038BDFEF7CFF8F3E74A4865684A4B626AF7
:10A6180005EB450133F81220B0FBF2F39942DDD87F
:10A62800B3EB053FDAD800231946F7F76DFA0902AC
:10A6380041EA10616B080002C0182A464FF0000377
:10A6480041F10001F7F760FA3C4BA0F540729A42DD
:10A65800C4D82368D860CCE7FEF79CFC0028C8D093
:10A668006168354B626A33F81220B0FBF2F24B088E
:10A6780003EB42034FF6EF72B3FBF1F3A3F11001C2
:10A688009142ABD823F00F02216892B2C3F3420380
:10A698001343CB60ADE7FEF785F8DFE72548DFE732
:10A6A800082B9BD801A252F823F000BFFDA6000892
:10A6B80009A7000815A70008E5A500080FA70008C6
:10A6C800E5A50008E5A50008E5A50008D9A6000845
:10A6D8004FF400406368616A174A32F81120B0FBF2
:10A6E800F2F000EB5300B0FBF3F04FF6EF73A0F17C
:10A6F8001002ACE7FEF74EFC00283FF47AAFE9E71A
:10A70800FEF758FCF8E7FEF74DF8F5E70948E1E7EA
:10A71800B0F5004FF4D1FEF74DFC9FE7F369FFCF8A
:10A7280000800040003801407442010800440040A5
:10A738007742F5070024F40084420108FFFC0F006B
:10A74800836ADA0710B506D50168C46A4A6822F434
:10A75800003222434A609C0706D50168046B4A68A8
:10A7680022F4803222434A60590706D50168446BB7
:10A778004A6822F4802222434A601A0706D50168F3
:10A78800846B4A6822F4004222434A60DC0606D5FC
:10A798000168C46B8A6822F4805222438A60990651
:10A7A80006D50168046C8A6822F4005222438A6044
:10A7B8005A060FD50168446C4A6822F48012224375
:10A7C800B4F5801F4A6005D14A68846C22F4C0023F
:10A7D80022434A601B0606D50268C16C536823F4FD
:10A7E80000230B43536010BD2DE9F041DDF81880BC
:10A7F80004460E4615461F462268D36936EA030307
:10A808000CBF01230023AB4201D0002027E0B8F1A0
:10A81800FF3FF2D0F8F77EF9C01B4045206802D808
:10A82800B8F1000F1DD150E8003F23F4D07340E881
:10A838000032002AF7D100F1080353E8003F23F063
:10A84800010300F1080141E80032002AF3D1202376
:10A85800C4F88830C4F88C3084F884200320BDE81C
:10A86800F08103685A07C7D5C3691B05C4D54FF4DF
:10A878000063036250E8003F23F4D07340E80032DD
:10A88800002AF7D100F1080353E8003F23F0010341
:10A8980000F1080141E80032002AF3D12023C4F86E
:10A8A8008830C4F88C30C4F89030D5E773B50446C6
:10A8B8000026C0F89060F8F72DF923681B681A077E
:10A8C800054619D423681B685B070AD56FF07E43D9
:10A8D800009300222B464FF480012046FFF784FFA7
:10A8E800B0B900202023C4F8883084F88400C4F864
:10A8F8008C30E06620670CE06FF07E4300933246B0
:10A9080003464FF400112046FFF76EFF0028D9D008
:10A91800032002B070BD10B5044650B3D0F888309B
:10A928001BB980F88430F8F7ABFA22682423C4F8FE
:10A938008830136823F0010313602046FFF7E8FD11
:10A94800012816D0A36A13B12046FFF7F9FE236841
:10A958005A6822F490425A609A6822F02A029A6051
:10A968001A6842F0010220461A60BDE81040FFF75D
:10A978009DBF012010BD000030B581658168A0F839
:10A988005C200023B1F5805FA0F85E20436735D1D5
:10A998000369002B40F2FF1318BFFF23A0F86030B3
:10A9A8000023C0F890302223C0F88C30016801F1F0
:10A9B800080353E8003F43F00103083141E800343D
:10A9C8000368002CF2D1456E84680169B5F1005F17
:10A9D80034D1B0F86850954230D8B4F5805F1DD1B5
:10A9E800254A264C002918BF22464267C1B153E8C0
:10A9F800002F42F4807243E80021F7E729B9036980
:10AA0800002B14BF7F23FF23C8E7B1F1805FC5D1B6
:10AA18000369002B0CBF7F233F23BFE7174AE4E7F6
:10AA280003F1080252E8002F42F0805203F10800B7
:10AA380040E800210029F3D1002030BDB4F5805F43
:10AA48000FD10F4A0F4C002918BF2246426751B157
:10AA580053E8002F42F4907243E800210029F7D10F
:10AA6800EAE7084AF2E753E8002F42F0200243E8F9
:10AA780000210029F7D1DFE781A30008E5A100083C
:10AA880021A1000855A00008D0F88C30202B30B444
:10AA980015D1B9B1B2B100230468C3660A4B9C4210
:10AAA8000AD063681B0207D554E8003F43F080636F
:10AAB80044E80035002DF7D130BCFFF75DBF022018
:10AAC80030BC70470120FBE700800040436E30B582
:10AAD8002BB90123A0F86A30A0F8683030BD0368AC
:10AAE800094D9A689968094C490FC2F342626B5C38
:10AAF800615CDB00B3FBF1F3A0F86A30AB5CA25CED
:10AB0800DB00B3FBF2F3E7E7A44201089C4201082B
:10AB18007047704770471FB504AB03E9060090F80B
:10AB28008430012B04463AD0012380F88430242352
:10AB3800C0F8883003681A6822F001021A609A681F
:10AB480022F440120A439A6071B95A68BDF80C00A1
:10AB58009DF80E1022F0100202435A605A6822F043
:10AB68007F4242EA01625A601A6842F001021A60A2
:10AB7800F7F7D0FF6FF07E42034600924FF4800152
:10AB880000222046FFF730FE38B92023C4F8883069
:10AB9800002384F8843004B010BD0320F8E70220B5
:10ABA800F9E790F88430012B0FD0012380F8843026
:10ABB800016851E8002F42F0020241E80023002B0F
:10ABC800F6D180F88430184670470220704710B5D7
:10ABD80090F88430012B044617D02423C0F888301D
:10ABE80003681A68196821F00101196042F00052DF
:10ABF8004FF0005141661A60FFF768FF2023C0F844
:10AC08008830002084F8840010BD0220FCE770B56D
:10AC180090F88430012B044617D005682423C0F827
:10AC280088302E682B6823F001032B60AB6823F073
:10AC380060431943A960FFF749FF20232E60C0F83D
:10AC48008830002084F8840070BD0220FCE770B5CD
:10AC580090F88430012B044617D005682423C0F8E7
:10AC680088302E682B6823F001032B60AB6823F033
:10AC780060631943A960FFF729FF20232E60C0F8FD
:10AC88008830002084F8840070BD0220FCE70000B2
:10AC980038B5084D052455F8043B2BB9013C14F090
:10ACA800FF04F8D1204638BDDB6898470028F5D066
:10ACB800F9E700BF64100020034BD870034B1B68F2
:10ACC8001B6C03B1184770477810002060100020F3
:10ACD800034B1874034B1B685B6C03B11847704730
:10ACE8007810002060100020F0B5314D314B95F9F7
:10ACF8000420314E91B00C46012795F905108DF8C6
:10AD0800047002288DF809208DF80A1010D18DF8EA
:10AD18000800D8711C7202F09FFD337803B114B19A
:10AD280001A803F003FA254B059A1A6011B0F0BD8B
:10AD380059714FF480711A71D9801C7233788DF86B
:10AD4800087053BB1F2306A88DF81C208DF81830F7
:10AD580002F064FF20238DF8183006A82B798DF8AF
:10AD68001C3002F05BFF22238DF8183006A86B799F
:10AD78008DF81C3002F052FF21238DF8183006A8F8
:10AD88006B798DF81C3002F049FF29238DF81830B3
:10AD980006A80B4B079302F041FF02F05DFD01236B
:10ADA80006A88DF818308DF81C3002F037FFB4E78C
:10ADB800781000203008002054100020581000207F
:10ADC800000400017FB5092301A88DF8043003F0C1
:10ADD800ADF90038044B059A1A6018BF01204042AB
:10ADE80007B05DF804FB00BF5810002070B504469A
:10ADF8000B46134962784A700020A2780A720870DC
:10AE08001A884A729A788A72DB780B746368CB6006
:10AE18000C4B1B68DA6A2AB1237803F0FB030A2B70
:10AE280000D09047084E052556F8043B1BB15B6AD5
:10AE38000BB120469847013D15F0FF05F4D170BDD0
:10AE48003C080020601000206410002070B5044603
:10AE580010480123037063784370A3788372E36812
:10AE6800C360E378037623694376237943720A4BF8
:10AE78001B689B6A03B19847084E052556F8043BA2
:10AE88001BB19B690BB120469847013D15F0FF05A2
:10AE9800F4D170BD5008002060100020641000201C
:10AEA800014B1868704700BF5810002000B58BB0E0
:10AEB800012368468DF8003002F088FD38B99DF806
:10AEC8000400003818BF01200BB05DF804FB002017
:10AED800FAE7000008B501F073FE48B9FFF7E6FF8E
:10AEE800012806D0054BD879197AFFF7FDFE012015
:10AEF80008BDBDE80840FFF7CBBE00BF3008002002
:10AF08002DE9F04186B005460E46174601F058FE79
:10AF180000287FD101F06CFE044640B9FFF7C6FF58
:10AF2800012807D03D4B197AD879FFF7DDFE6FF07D
:10AF3800020462E0DFF8E88088F80860003E18BF85
:10AF480001268DF80460374E687833798DF8123011
:10AF5800694602F0D9FC00283ED08DF804400394DD
:10AF6800ADF810406FF0060495E803002E4B83E817
:10AF78000300337988F80A30394601A803F0DAF972
:10AF88002A4B059A1A60112841D801A353F820F0DA
:10AF9800F7AF00081DB0000817B0000817B0000888
:10AFA80017B0000817B0000817B0000837AF00083E
:10AFB80017B0000817B0000817B0000811B0000853
:10AFC80017B0000817B000081DB000081DB0000831
:10AFD8001DB000080BB000082B788DF808306B788E
:10AFE800ADF810306B6803934FF0FF34BCE7104B9B
:10AFF80000221A70E31D18BF1446204606B0BDE8AB
:10B00800F0816FF00404F8E76FF00504F5E74FF0FE
:10B01800FF34F2E76FF00104EFE700BF30080020CB
:10B0280050080020781000206008002058100020E8
:10B038005C10002037B501F0E5FD144D052455F8E6
:10B04800043B5BB11B694BB155F8043C9B682BB1C1
:10B05800984718B155F8043C1B699847013C14F00F
:10B06800FF04ECD1FFF714FE68B9094D2B7853B1F2
:10B07800084BADF80040D978019422466846FFF79E
:10B088003FFF00B92C7003B030BD00BF6410002032
:10B098005C1000207810002030B58BB0054601F018
:10B0A8008FFD0446002839D1FFF700FF012838D169
:10B0B80068468DF8004002F089FC10B14FF0FF306F
:10B0C80004E09DF80430AB4202D100200BB030BD43
:10B0D800012DF3D0022D11D0002DF7D1002BF4D083
:10B0E80068468DF8045002F099FD0028E6D10E4B11
:10B0F8001B681B6B002BE8D09847E6E7002BDDD1D7
:10B1080068468DF8045002F089FD0028D6D1064B18
:10B118001B681B6B002BD8D02846EDE76FF00100A9
:10B12800D4E76FF00200D1E76010002010B50446A4
:10B138008AB018B94FF0FF300AB010BD0023684636
:10B148008DF8003002F042FC0028F3D19DF804305D
:10B158002370F1E77FB500220B4620498DF80720C0
:10B1680001220A7042784A700446002A33D10279D3
:10B178000A721A884A729A788A72DB780B740369A1
:10B18800CB60C378164D8DF80830037B8DF80930F5
:10B19800836803932B68DB6A0BB102A898472B6876
:10B1A8009B6B13B1227E02B198470E4E052556F8C7
:10B1B800043B1BB1DB690BB120469847013D15F0F4
:10B1C800FF05F4D10DF10700FFF7B0FF637913B164
:10B1D800054B01221A7004B070BD00BF3C08002066
:10B1E80060100020641000205C10002010B5044698
:10B1F8008AB018B94FF0FF300AB010BD2023684656
:10B208008DF8003002F0E2FB0028F3D1024A9DF9E4
:10B21800043023701371EFE77810002000B58BB06D
:10B228002323019068468DF8003002F0F7FC0038BF
:10B2380018BF012040420BB05DF804FB70B5654CA7
:10B2480001468EB01822204606F0FEF8624B002216
:10B258001A70F8F729FF23784068012202FA03F1EF
:10B26800014004D15D4B084608F0E4F8FEE75C496C
:10B278005C481A4602F032F918B14FF0FF300EB0B0
:10B2880070BD272304A88DF8103002F0C7FC564E75
:10B29800564D002870D1012333702B68DB690BB140
:10B2A80000209847272304A88DF8103002F08EFB61
:10B2B800059B93F84820227093F8182193F81A31C7
:10B2C8006270A370464BD3E9020105F0AFFF054653
:10B2D8000028D2D1464E062304A88DF8103002F07B
:10B2E80075FB059B736104A802F098FC022304A86F
:10B2F8008DF81030059602F069FB0836032304A880
:10B308008DF81030059602F061FB0F2606F052F812
:10B31800012304A88DF814308DF8106002F07EFC2B
:10B3280010230DEB03008DF810308DF8145002F047
:10B3380075FC04238DF8103004A8A3788DF8143018
:10B3480002F06CFC3A238DF8103004A86369059369
:10B3580002F064FC02A920788DF8086004F0E8F88F
:10B36800003818BF0120E0711420FFF757FFE0797B
:10B3780003F0A4F9284682E728238DF810302B68BB
:10B388001B6943B104A802F021FB2B6805981B69CF
:10B3980040F2C4519847272304A88DF8103002F0D2
:10B3A8003DFC50B9012304A88DF8103002F00EFBC3
:10B3B8009DF81430002B7FF46EAF3378002B7FF4A8
:10B3C8006CAF052204A88DF81020059302F026FC26
:10B3D80078E700BF781000205C100020AC4201081C
:10B3E800A0100020B8100020541000206010002089
:10B3F8003C10002037B500230D4601930446D0B910
:10B4080000F0A8FB0190019BD3B10F4A42F8243009
:10B418000E4A9A620E4A1268916B1963916C5963CD
:10B4280092690C49D9625A6128465B680A49F22236
:10B438009847002006E001A900F092FB0028E2D01E
:10B448004FF0FF3003B030BD64100020F1AC0008AD
:10B4580060100020CDAD0008480F0020194B07B53B
:10B468001860194B194A1A60194A5A60194A9A60A1
:10B47800194ADA60194B02681A6042685A60826891
:10B488009A60C268DA60164A1A6182695A61154B75
:10B49800C26B5A60144A019119609A601946134A9E
:10B4A800DA600020FFF7A6FF48B901A800F056FBB4
:10B4B800003818BF0120404203B05DF804FB4FF08C
:10B4C800FF30F9E760100020B810002055AE0008E2
:10B4D8005DB1000875B50008F5AD0008A0100020A2
:10B4E800E9F4000890100020C1AC0008D9AC0008AD
:10B4F80051B118B1012804D000207047044B0B60EB
:10B508007047044B0B60F7E74FF0FF30704700BF00
:10B51800000400010100010208B503F0EBF800285F
:10B5280014BF6FF00100002008BD08B502F0BCF997
:10B53800002814BF6FF00100002008BD10B50446B4
:10B548008AB018B94FF0FF300AB010BD2123684601
:10B558008DF8003002F03AFA0028F3D1024A9DF93A
:10B56800043023705371EFE7781000202DE9F04183
:10B578002E4D2F4F00232B7043786B703B689B6ACE
:10B588008AB004460BB128469847DFF8A8800526FC
:10B5980058F8043B1BB11B6A0BB120469847013E83
:10B5A80016F0FF06F4D12378052B2FD00B2B35D0BE
:10B5B800012B25D1204C062368468DF8003002F077
:10B5C80005FA0199E07905F077FE10B91B4B019A4D
:10B5D8005A611B48FFF70AFE1A48FFF7AFFF6B785E
:10B5E8008BB9A371184B5878FFF756FD3B685B6A17
:10B5F8000BB1114898476B7813B9E07905F0ECFE68
:10B608000AB0BDE8F081FF23A371EFE70F4B0122D9
:10B618005A74227A9A74627ADA74F1E76378002BA2
:10B62800EED00AB0BDE8F041FFF7CCBB50080020CF
:10B638006010002064100020300800203C1000201A
:10B648003408002035080020781000203C0800202D
:10B6580030B58BB0FFF769FF0446F0B903F048FF37
:10B66800831C1DD0F8B9134D2B685B69DBB1272308
:10B6780068468DF8003002F0A9F92B6801985B69DB
:10B688004FF4B961984703F045FF78B92CB9094BD5
:10B698001B68DB690BB10120984720460BB030BD11
:10B6A8006FF00704EFE74FF0FF34ECE74FF0FF349B
:10B6B800F3E700BF60100020014B1878704700BF07
:10B6C800CC100020014B5878704700BFCC100020E8
:10B6D80070470000044B9A7A0AB101225A70034B52
:10B6E8005B6903B118477047CC1000206C08002034
:10B6F80073B5224C6378002B33D008F085F966685F
:10B708000546FFF7CDFB0644AE4214D2A37A93B1A7
:10B71800E0228DF800208DF80130217AE36801934A
:10B7280001226846FFF7ECFB08B1073010D100236F
:10B738006370A372656094F83430EBB1002384F829
:10B7480034300F4B5B6BBBB102B0BDE8704018479B
:10B7580040F2DC510B4808F023FA0A4808F0E6F9F1
:10B76800E8E794F83520002AE5D094F8360084F804
:10B778003530FFF791FCDEE702B070BDCC10002039
:10B788006C0800200411002037B5104D104CC8B1CA
:10B79800C1B10123627200222860E16023700D4864
:10B7A8000D4B00924FF0FF3108F014F900250B48BB
:10B7B80025822022294605F05BFE6570A574A586C2
:10B7C80003B030BD00232B602370EFE7C8100020C2
:10B7D800CC10002004110020DDB60008E010002085
:10B7E8002DE9F0478E4C23788CB0002B56D0C278C8
:10B7F8000AB9837B13B1238A01332382437B002B4D
:10B808004CD0E02A4AD10023A372876897F80080B9
:10B81800B8F1220F27D8B8F1220F30D8DFE818F096
:10B828004100FB0052005A0061006E0075008E0056
:10B838009D00B400C7002F002F002F002F002F00FD
:10B848002F002F002F002F002F002F002F002F0078
:10B858002F002F002F002F002F002F002F002F0068
:10B86800C900D000D400B8F17E0F00F0CC80B8F148
:10B878007F0F00F0DF80B8F17D0F00F0AB80A57A74
:10B88800002D00F05B81674C637A3BB94FF47A7105
:10B89800204608F085F9204608F048F90CB0BDE8C4
:10B8A800F087E36801220021A2721970A37AE16887
:10B8B8009818A0720620C854A37AE1689818A07254
:10B8C800CA54DCE7584B9B6A002BD8D001210220D0
:10B8D8009847D4E77B7884F83630012384F83530EC
:10B8E800CDE704238DF804307B78003B18BF012393
:10B8F80001A88DF8083002F091F9C0E7787800388F
:10B9080018BF012002F0DAFEB9E7484E0FCE01ADAC
:10B918000FC50FCE0FC596E8070085E807007B78AE
:10B928000A2BACD8424A12685268002AA7D00CA940
:10B9380001EB830353F82C0C9047A0E77878431E5B
:10B94800012B9CD83A4B01381B6818BF0120207284
:10B958009B68002B93D0984791E7E2680123082160
:10B96800A3721170627A057BA17AAA4228BF2A467F
:10B97800934284D285685A1CEB5CE56801334E1CFF
:10B98800A6726B54D3B2EDE7E3680122A2720922D2
:10B998001A70A37AE268218A581CA072D154A27A3C
:10B9A800238AE1681B0A501CA0728B5467E7238224
:10B9B80065E705238DF8043001A802F0B7FB5EE7C0
:10B9C800194BDB6A98475AE7194B78781B686075FA
:10B9D800DB68BEE7037B072B7FF451AF06238DF8A6
:10B9E8000430B7F80130ADF808307B793A791B0498
:10B9F80043EA0223FA781343642253430393BB793F
:10BA08008DF81030D8E73B2201A88DF804208DF876
:10BA1800083002F003F9012384F834302FE700BF1F
:10BA2800CC100020041100206C0800207C40010884
:10BA3800C81000202A2301A88DF8043001F0C6FFA1
:10BA480094F80A90E6689DF808009DF809509DF85A
:10BA58000A709DF80BC09DF80D309DF80E209DF8DA
:10BA68000F109DF80CE009F1010A84F80AA006F805
:10BA78000980354E94F80A903668D4F80C8009F19C
:10BA8800010A84F80AA096F803A008F809A094F817
:10BA98000A90D4F80C8009F1010A84F80AA096F8F3
:10BAA80002A008F809A094F80A90D4F80C8009F1CB
:10BAB800010A84F80AA096F801A008F809A094F8E9
:10BAC8000A9009F1010A84F80AA096F80080E6684D
:10BAD80006F8098094F80A80E66808F1010984F8F4
:10BAE8000A9006F808C094F80AC0E6680CF1010844
:10BAF80084F80A8006F80C70A77AE66807F1010C4A
:10BB080084F80AC0F555A57AE6686F1CA7727055C7
:10BB1800A07AE568461CA6722954A17AE0684D1CF3
:10BB2800A5724254A27AE168501CA0728B54A37A81
:10BB3800E268591CA17202F803E0A0E6034807F086
:10BB4800A7FF6570AAE600BFC810002004110020F6
:10BB580070470000004870476C08002000207047BC
:10BB68004FF0FF3070470000044B054A93F8183136
:10BB7800022B18BF062382F890347047E016002085
:10BB8800A81C0020034BD3F8483313B15B6903B1F9
:10BB980018477047A81C0020034A137843F0040391
:10BBA8001370FFF7EFBF00BFA41C00201FB50A4B9E
:10BBB8008DF8090093F87C208DF80A2093F88C20E2
:10BBC80093F848000D3202A98DF8082003F0B0FC64
:10BBD800C0B205B05DF804FBE016002010B5074CB4
:10BBE80004F5806007F054FF94F81A3413B1012368
:10BBF80084F81934BDE81040FFF7C4BFA81C002022
:10BC080010B50C4CD4F8403343F08003C4F84033EB
:10BC180094F81A3413B10020FFF7E0FF94F8913438
:10BC280023F0120343F0120384F89134BDE8104066
:10BC3800FFF79ABFA81C00202DE9F041DFF8AC807F
:10BC480098F81831022B06460D4602D0284BDB6ABD
:10BC5800984702F0E9FD044628B1022002F0DAFD17
:10BC6800002002F0DCFD98F81831012B17D102F002
:10BC7800DDFD074630B1002002F0CDFD002002F0C6
:10BC8800CFFD3C4602F0D4FD48B1002002F0C4FDCF
:10BC9800002002F0C6FDBDE8F041FFF765BF002CAB
:10BCA800F9D1144C94F8902494F81A34BAB90BB119
:10BCB80084F84164304602F065FFD8F82C0007F09C
:10BCC800ADFED4F8B4339842E5D30B4807F0E0FE54
:10BCD80094F8913443F0100384F89134DBE70BB106
:10BCE80084F84154284602F04DFFF1E7E0160020A1
:10BCF800304A0108A81C00204020002073B5164CCB
:10BD0800164D04F57A76EB6C95F8502095F9781075
:10BD180095F84800009603F031FC95F8303184F826
:10BD2800FC3395F8480040F2012304F224423146DE
:10BD3800A4F8FA3303F02EFC58B194F8243484F8AC
:10BD48006A34074B00205B6B984794F8FB3384F800
:10BD5800903402B070BD00BFA81C0020E01600207F
:10BD6800304A0108074A10B5137843F002031370EC
:10BD7800FFF708FFBDE81040034B01220021022015
:10BD880007F058BBA41C0020F5420108074A10B56B
:10BD9800137843F008031370FFF7F4FEBDE8104072
:10BDA800034B01220021022007F044BBA41C002001
:10BDB800054301082DE9F0410F4616461D46804609
:10BDC80007F022FE0B4A0C4C1378278123F011034D
:10BDD80043F011031370C4E9000866812573FFF767
:10BDE800D1FEBDE8F041054B01220021022007F0F9
:10BDF80021BB00BFA41C00205422002015430108C9
:10BE080013B507F001FE0D4B6C461860204607F08D
:10BE18004FFD94E803000A4A0A4B83E803001378AD
:10BE280043F020031370FFF7ADFE074B01220021FA
:10BE3800022002B0BDE8104007F0FCBA64220020DE
:10BE4800A41C0020E01F002022430108F8B5334D50
:10BE580095F81841012C06464BD0022C51D064B9F4
:10BE680038B9D5E91B0105F1740383E803002046BE
:10BE7800F8BD01283DD0022801D00324F7E7284F58
:10BE880085F8180107F5747EBEE80F0007F57A7C7F
:10BE9800ACE80F009EE8030095F8E9308CE8030051
:10BEA80087F8FB63E3B195F80031022B18D1D5F878
:10BEB80004316B67C7F8EC3395F87D3095F80821A5
:10BEC80087F8F83395F88C3085F8782087F8F933B7
:10BED80097F81B2487F8E82340F20133A7F8FA33D0
:10BEE800002387F81A340F4BDB6A9847FFF706FFE1
:10BEF800BDE702F0A4FC04460028B8D185F8186113
:10BF0800B5E70028B9D1064B85F81801062283F851
:10BF18009024044BDB6A98473446A8E7E0160020D3
:10BF2800A81C0020304A01082DE9F04192B00646CD
:10BF380002F07AFC002840F05981AD4D95F818318F
:10BF4800012B09D02B6BAB4C93B194F80431BBB1E6
:10BF5800042B6FD0032003E002F068FC18B10F2017
:10BF680012B0BDE8F08102F063FC0028EAD0F6E7E1
:10BF7800B5F82031D4F81C24013B53432B63E4E784
:10BF88009D4803F00CFA002840F02C8194F80C31FD
:10BF980023802B6B0C930DF1180895F839308DF828
:10BFA8003830404695F81C318DF83A3007F0A6FC39
:10BFB800D5F82831009302AF98E80600D5F8243167
:10BFC800384607F032FC97E803000FAB83E803001C
:10BFD800EB6A0D9300238DF844302388ADF8463082
:10BFE80095F8303101228DF839201BB98DF844209D
:10BFF8008DF83930814B0093814B95F84800A3F1B7
:10C0080079020CA903F009FBC0B10B28A8D1D4F818
:10C01800941499B1002EA3D0D4F84033794843F052
:10C028002003C4F8403307F0BBFD764807F07EFDD7
:10C03800002095E7704803F0E6F9A4E795F8487002
:10C0480095F9693095F9392095F87D106E4E384686
:10C0580003F0F0FA009641B2EB6C95F850203846A0
:10C06800183603F08BFA0096EB6C95F8502095F98A
:10C07800701095F8480003F081FAD4F8C413AB6D3A
:10C08800D4F8DC230B44C4F8B033EB6D1344C4F884
:10C09800B43394F80431042B07D02B6E0B44C4F846
:10C0A800B0336B6E1344C4F8B4330023089395F887
:10C0B800303183B108A802F095FC00284ED195F9DB
:10C0C800390094F837629DF82070FFF76FFD3E4401
:10C0D80080B2B04240D300238DF8133095F8393040
:10C0E8008DF8213095F838308DF82230D5F8803029
:10C0F8000993D5F884300A932388ADF82C3095F845
:10C10800303194F81B648DF82E3095F848003F4B79
:10C118008DF820600DF1130208A903F043FA0123FA
:10C1280084F8413495F8393084F842349DF8133056
:10C1380084F84334D4F81C34C4F85064C4F8483440
:10C14800C4F8583402F076FB50B1D4F81C0402F05D
:10C1580083FB28B1102003E7082001E71320FFE63E
:10C1680095F81831012B01D102F078FB02F065FB3C
:10C178000023059394F8043195F9395094F81B6419
:10C188009BB1042B7FF4E6AE05A802F067FE58BB0E
:10C1980094F8183413B1059B013B0593164B059889
:10C1A8003246E9B202F0C0FE02E0134802F090FE07
:10C1B800C0B9D4F8403394F80C11218043F002033D
:10C1C800C4F8403394F8183411480133DBB284F8CA
:10C1D800183484F845340F4B00259B6AC4F89854EA
:10C1E800984725E71120BBE61220B9E60E20B7E6EE
:10C1F800E0160020A81C0020B01D00201017002009
:10C208003C2100201020002060200020C4200020B5
:10C21800AA1C0020304A0108F0B5504C504EB4F822
:10C22800DC202287D4E92D0194F8B12084F8692014
:10C2380004F16C0282E80300D4E92F0104F17402CE
:10C2480082E80300B4F8C420A4F87C2091B0D4F8A4
:10C25800CC20D4F8C810C4F884200025D4F8D02005
:10C26800C4F888200123A4F82031C4F8801084F889
:10C278003051A56284F81B5184F83A5084F81D5156
:10C2880084F81E51C4F83451C6F89854A6F81854C6
:10C2980086F81A54A4F838518DF8183004F5097343
:10C2A800039304F50A7394F84800A4F846510493DC
:10C2B80003A92C4B84F84551C4E94F55059303F065
:10C2C80045F9E36EC6F8D43394F87D3086F8E03348
:10C2D80094F88C3086F8E1334FF48073A6F8E23393
:10C2E80086F8D05394F8303186F8E43306F574773D
:10C2F8000FCF06F57A740FC497E8030040F20123C4
:10C3080084E80300A6F8FA33D6F8483386F81B54B5
:10C31800CDE901551BB15A685B6901920293124B32
:10C328000793A3F148020892A3F1140209920F4A55
:10C338000B9229330A93A2F19C030C93A2F1980360
:10C348000D93131D0E9301A902F14C0307A802F5E2
:10C3580099620F9302F05DFA11B0F0BDE01600206B
:10C36800A81C0020C421002010210020C417002090
:10C37800F8B50D4F0D4C0E4E0D4607F089FB3B6B83
:10C38800984796F8480004F22442294603F002F937
:10C3980048B194F8243484F86A34706D7B6B9847FC
:10C3A800EB7C84F89034F8BD304A0108A81C0020C2
:10C3B800E01600200F4890F81B3480F8B8330E4B75
:10C3C80093F8692080F8BB2393F87D2080F8C82370
:10C3D80093F88C2080F8C92393F8303180F8CC3357
:10C3E8000022A0F8CA2300F56E7100F56070FFF70F
:10C3F800BFBF00BFA81C0020E0160020114890F81D
:10C408009034EBB190F81B3480F8D0330E4BDA6ED1
:10C41800C0F8D42393F87D2080F8E02393F88C208B
:10C4280080F8E12393F8303180F8E4334FF48072D8
:10C43800A0F8E22300F5747100F56670FFF798BF65
:10C44800704700BFA81C0020E016002070B5344CCF
:10C458002421204605F00EF8636A984218BF6062EE
:10C468004FF01C012F4814BF0125002505F002F8E4
:10C47800636C984218BF60644FF480712A4818BFF3
:10C4880045F0020504F0F6FFD4F84831984218BF89
:10C49800C4F848014FF0D401244818BF45F00405FA
:10C4A80004F0E8FFD4F82032984218BFC4F82002FC
:10C4B8004FF000011E4818BF45F0080504F0DAFFE8
:10C4C800D4F82432984218BFC4F824024FF460719B
:10C4D800184818BF45F0100504F0CCFFD4F8A8356B
:10C4E800984218BFC4F8A8054FF01401124818BFA5
:10C4F80045F0200504F0BEFFD4F8C03598420F4B34
:10C5080018BFC4F8C005D3F8483318BF45F0400534
:10C518002BB11B691BB12846BDE87040184770BD98
:10C52800E016002008170020281700202C180020EB
:10C5380004190020081900208C1C0020A81C0020C9
:10C548002DE9F04F91B04FF00008012B05460F463A
:10C5580002928DF81580ADF8188003D8C84EC146F0
:10C56800B94502D311B0BDE8F08F15F8090002F003
:10C5780077FA4844B842F5DC15F8093009F10104A6
:10C58800023BE4B2112BEDD801A252F823F000BF10
:10C59800E1C5000813C6000813C700083DC7000816
:10C5A800C5C70008EDC700085FC8000891C80008A3
:10C5B8000DC900086DC500086DC500086BC90008E5
:10C5C8006DC500086DC5000829CA000851CA0008D1
:10C5D80095CA0008D3CA0008052002F0EDFA90B108
:10C5E8000521002002F0ACFA2A5DA64B09F10304EC
:10C5F80009F102095FFA89F983F85C2415F8092022
:10C6080083F85D24E4B2A146AAE700238DF816302A
:10C618008DF817308DF81C308DF82030B8F1000FE8
:10C628006CD14FF0050896F87C208DF83920631EF0
:10C6380096F839208DF83B202B4496F838200D9336
:10C648008DF83C2096F81A3196F868208DF83D2030
:10C65800D6F82C218DF83A300C9273B37B1C1B1B37
:10C66800DBB28DF8383008AB019307AB009396F82E
:10C6780048000DF117030DF116020CA902F09EFFF8
:10C688008DF8150000F00700072813D196F9392016
:10C698009DF9163086F839309A429DF8173086F899
:10C6A8003830B8BF01229DF81C30B8BF86F81D216C
:10C6B80086F868304FF0000909E00523D1E7012228
:10C6C8000DF11501032002F0DBF809F101095FFA09
:10C6D80089F29DF82030B3FBF8F19142EFD823445A
:10C6E800DCB2631EDBB29F420DD9EA5C032A9AD002
:10C6F800A74288BF1C464FF0010884E709F10509E5
:10C708005FFA89F4F7E71C46F5E72B5D012203F091
:10C718000F0309F1020986F81B3102FA03F35FFAE5
:10C7280089F9A6F82031002206A9042002F0A8F809
:10C738004C4668E707238DF815302B5D96F84800BE
:10C74800C3F3021203F00F038DF8303009F103032D
:10C75800DBB28DF83120EA5C09F10403DBB209F1A0
:10C768000504EB5C09F102095FFA89F91B0443EA45
:10C77800022315F809201343642253430CA90D938F
:10C7880002F02BFF00F00703072BE4B28DF8150029
:10C798000CD19DF8303086F8703086F878300D9BD3
:10C7A800F36673679DF8313086F869308DF81800A4
:10C7B800012206A9052002F063F824E7314BD3F8DB
:10C7C80048336BB11B685BB19847029B8DF8180022
:10C7D80003F03F038DF81930022206A90620EAE784
:10C7E800FF20F2E703238DF815302B5D8DF82430F8
:10C7F8000CAB089309F10303DBB209F10604EA5C08
:10C8080096F8480009F10403DBB208A9EB5C1B04A5
:10C8180043EA022309F10202D2B209F10509AA5C2E
:10C828001343642253435FFA89F90C9300230D9351
:10C8380015F809308DF8383002F0D5FEC3B200285B
:10C84800E4B28DF81530FFF6DEAE8DF8183001220F
:10C8580006A90720AFE72B5D03F00F03012B4FF468
:10C868007A7238BF0123534309F10209B3651344AF
:10C878005FFA89F9F365002206A9082056E700BF88
:10C88800E0160020A81C00202B5D96F84800C3F392
:10C8980040128DF81D2007A9C3F3001203F00F03FF
:10C8A8008DF81C208DF81E3002F0A3FE09F1020954
:10C8B80001305FFA89F93FF43BAFBDF81C30914A6B
:10C8C800A6F87C309DF81E309DF81C40D05CF5F72A
:10C8D8009DF80223C6F880000CA996F848008DF848
:10C8E80030308DF8324002F023FE96F93930089046
:10C8F80040B29842B8BF184686F83900002206A907
:10C90800092013E703238DF815302B5D8DF830309F
:10C9180009F10303DBB209F10504EA5C96F8480063
:10C9280009F10403DBB209F10209EB5C5FFA89F94A
:10C938001B0443EA022315F80920134364225343D6
:10C948000CA90D9302F05BFEC3B20028E4B28DF887
:10C958001530FFF658AE8DF81830012206A90A20C6
:10C9680029E7092002F028F9DFF89CA1002854D013
:10C978000921002002F0E4F80023ADF8263009F17F
:10C988000203DBB24FF47A71EA5C09F10303DBB20C
:10C998000DF1300BEB5C1B0443EA02232A5D1343C1
:10C9A80009F10402D2B209F1060409F10509AA5CE9
:10C9B8005FFA89F943EA026315F8092003934A43A9
:10C9C80012125846ADF8242006F072FF039B03F1BB
:10C9D800965303F5A91303F5EC530893DAF83C339F
:10C9E80000930DF1200999E80600DAF838330AA80F
:10C9F80006F01BFF0B9B00939BE806000A9B48462A
:10CA080006F0F8FE99E8030006F02AFF01F021FF7E
:10CA18000123E4B28AF83834F5E58AF83804F2E5F7
:10CA28000C2002F0C9F800283FF4EDAD0C210020DD
:10CA380002F086F8344B93F89034043B012B7FF6D0
:10CA4800E2AD01F002FFDEE509F10203DBB22A5D87
:10CA5800E95C09F10303DBB209F10504EB5C09F1B8
:10CA680004095FFA89F91B0415F8090043EA012350
:10CA780013436421594300F00F0001F0E7FEE4B2CC
:10CA88008DF81800012206A9112094E60D2002F065
:10CA980093F800283FF4B7AD0D21002002F050F8BC
:10CAA80009F10203DBB2194AE85C2B5D126809F14F
:10CAB800040409F103095FFA89F943EA002015F82B
:10CAC8000910E4B201F0C4FE9DE52A5D09F10203F4
:10CAD80009F1040409F10309DBB25FFA89F9E95C99
:10CAE80015F809301B0443EA012313436420584313
:10CAF80001F0B0FEE4B28DF81800012206A9132057
:10CB080059E600BF2F430108A81C0020542200202A
:10CB18000E4B93F89124920703D593F88F24012A9A
:10CB280008D90B4991F81A2122B18A6A501C18BFFA
:10CB380001328A620022A3F8182483F81A24D3F851
:10CB4800402322F00202C3F840237047A81C0020AB
:10CB5800E016002070B5184C184D04F55A7006F010
:10CB680097FFD4F84033D4F89804D5F8906023F0B0
:10CB78002003C4F8403338B106F050FF864203D290
:10CB8800002385F83A3070BD0120FFF7CDF9002861
:10CB9800F9D00B28F7D095F8393084F842340920B9
:10CBA80094F8183484F8453484F8410401F0EAFF15
:10CBB800BDE87040FFF7ACBFA81C0020E0160020BD
:10CBC800094BD3F84023012A0AD008490978C90734
:10CBD80008D43AB993F89204013818BF0120704775
:10CBE8000020704701207047A81C0020A41C0020CA
:10CBF800034BD3F84003431E58425841704700BFC7
:10CC0800A81C00202DE9F04FA9B0EFF3108272B6EE
:10CC1800DFF8F4820021D8F80030C8F8001082F359
:10CC28001088BA4C002B00F0E480DAB29B0603921D
:10CC380064D5B74D95F81831022B02D0B54BDB6A95
:10CC48009847EFF3108972B6B34F06F0DDFE3E68E1
:10CC5800D4F8B013361A3144B04806F0A1FFAF48F3
:10CC680006F064FFD4F8B413AD48314406F098FFD9
:10CC7800AB4806F05BFF89F3108894F81A34002B50
:10CC880000F06D81152312A995F848008DF84830F9
:10CC980002F04EFCD4F8B4130F900144A14806F0FA
:10CCA8007FFFA04806F042FF3B6894F81B24EB6224
:10CCB8000DAF38468DF870201D9306F01FFED5F88D
:10CCC8002831009306AE97E80600D5F8243130469F
:10CCD80006F0ABFD96E803001FAB83E80300D4F829
:10CCE8001C341E9395F8303195F84800003B18BF66
:10CCF80001231CA98DF8713002F023FC039BDF0689
:10CD08004BD5834DDFF820A2D5F8E420BAF90A30D4
:10CD1800059298F800200493002363F300020A9315
:10CD280088F8002084F84434049AA4F8223484F85B
:10CD38002534C4F82834A4F82C3484F82E34C4F8E4
:10CD4800303484F82034C4F8343484F83834C4F8DF
:10CD58003C34704B9AF90C90A4F88C2494F89024E5
:10CD6800DB6A84F88E9484F88F24DAF80470BAF8B1
:10CD78000860984794F88F3413B9694806F088FE1C
:10CD88003146384601F04EFD8346002800F0EA801F
:10CD9800049BA4F87E3484F88094039B19071AD561
:10CDA8005B4B93F81831022B02D05A4BDB6A984739
:10CDB8000220FEF7D9FE84F8410401F0E3FE94F85E
:10CDC8001A3413B1012384F8193494F8913443F0D8
:10CDD800100384F89134039B5A0703D506210520D4
:10CDE800FEF72AFF039B9B0703D504210320FEF7C8
:10CDF80023FF01F035FD94F89124D7065FD5002371
:10CE080084F89234D4F840331E0644BF23F08203DA
:10CE1800C4F8403312F0050F00F0FC820B2001F03B
:10CE2800CBFE002800F0F68294F89134DD0700F17B
:10CE3800F182580740F10883D4F8403323F0020305
:10CE4800C4F84033D4F8402382BB94F8915415F0C9
:10CE580001011EBF2B4662F3000384F8913494F855
:10CE680091345E0744BF6FF3820384F89134012341
:10CE780084F8923421B1D4F844332C481B6898477D
:10CE88006D070BD52A4801F0A3FE01F0D1FE28B1A9
:10CE980094F8913443F0040384F8913401F0CEFC03
:10CEA80094F891346FF3041384F89134012384F8CF
:10CEB800923494F8913443F0200384F8913494F830
:10CEC800913418070AD56FF3C3031A4984F89134CB
:10CED800D4F84433A1F12400DB68984794F89134DE
:10CEE80099070AD56FF34103124984F89134D4F8AD
:10CEF8004433A1F16C005B68984794F89034022B96
:10CF08001AD1FEF7FBFE17E0A41C0020A81C002085
:10CF1800E0160020304A0108642200202820002062
:10CF280040200020A820002054220020E8200020D3
:10CF3800FC2000203421002094F891349A0640F116
:10CF4800C6826FF3451384F89134D4F84033002B2C
:10CF580040F0BD8229B0BDE8F04FFFF777BA84F8FA
:10CF68004134A1E695F81821012A0CD101F05EFCA4
:10CF7800804668B1584601F04EFC584601F050FC16
:10CF8800042384F88F347EB9012384F8213450E1D6
:10CF980001F04EFC0028F6D0404601F03DFC40462A
:10CFA80001F03FFC0523ECE73B7804935B09013B68
:10CFB800062B00F21882DFE813F00700160295002E
:10CFC8001602920016020702102EDDD995F83031AC
:10CFD8001297F6B28DF84C60002BD5D11CA804F03E
:10CFE8005DF912AA1CA9FF2002F0B2F89DF858308A
:10CFF800C3F3030307468DF82C3095F8480095F8DD
:10D008007D308DF82D3007220BA902F0A4FA002FED
:10D018005DD100285BD09DF853309DF852201599BA
:10D02800C5F8E4101B0443EA02239DF851200220AE
:10D038001343C5F8E03004F03FF99DF8583095F8EF
:10D04800480085F82E71C3F30212C3F3030385F871
:10D05800703085F878309DF8593085F86920012BB3
:10D0680038BF01234FF47A725343AB651344EB6521
:10D078000DF15A034FF001081093113E94F81B3438
:10D088008DF83C300FA985F868808DF8446002F06F
:10D098006AFA0223404685F8303101F08DFD18B157
:10D0A8004146384601F04CFD94F88F34012B00F2CC
:10D0B800A88194F81A34002B40F09B8194F891349D
:10D0C80043F0100384F89134FEF74EFD65E6012025
:10D0D80001F072FD0028E7D001210720E2E70123D3
:10D0E80084F8203495F87D308DF82E3094F8243467
:10D0F8008DF82D3095F88C3095F848000D330BA934
:10D108008DF82C3002F014FAA6F10D031BB2099029
:10D1180023EAE37300B283423FF736AF0B2E7FF664
:10D1280033AFBB4B25931CA8FF231C978DF8746065
:10D138008DF8983002F0D8F8074600287FF424AF1D
:10D1480095F81831012B13D101F070FB002873D02A
:10D15800384601F060FB384601F062FB04239DF875
:10D168007C101E9884F88F34C1F3001101F077FB0E
:10D178009DF87C301E99C4F8341413F00F0203D0C4
:10D188009DF89000002863D19DF89800002862D08F
:10D19800002A7FF4F9AE9DF89020002A0CBF4FF0CA
:10D1A80002084FF0030800220A92D5F8EC209142B9
:10D1B80054D195F8E910002950D0D5F80C1195F8FC
:10D1C800EAB009680A9195F81811022902D10321D9
:10D1D80084F88F14B8F1030F7FF4D6AE13F0600F04
:10D1E8007FF4D2AE0592012795F82E31BBF1000FDE
:10D1F80037D0BBF1010F38D1012B34D16FF00906BC
:10D2080046FA08F606F00106C6F10206F6B2BDF8BF
:10D218007E100AAA304601F02DFE40B307280CBF45
:10D228000823012384F821340A9BC4F83034C4F855
:10D238006C34FEF7E5FCB0E501F0FAFA002897D067
:10D24800384601F0E9FA384601F0EBFA052386E79B
:10D258004FF00008A7E74FF00108A4E74FF0010BD3
:10D26800C2E70426D3E70326D1E70123DAE71CAB9C
:10D27800009305990A9B3246584601F0BBFE20B13F
:10D2880002280CBF0A230B237FE60A9BC4F830341C
:10D29800C4F86C349DF87C3084F82104C3F340133F
:10D2A80084F82E3484F8443494F88F3484F8227443
:10D2B800012B9EBF0122A86285F81E21012FC4F808
:10D2C800280484F82C0484F8410438D1022284F814
:10D2D800202495F83A20002A4AD19DF87C20D606C9
:10D2E80046D4012B94F840149DF87C2005D80129D8
:10D2F80001D1900601D501F05FFBB8F1020F94F857
:10D308008F3443D0B8F1030F0AD09DF87C10B8F1E0
:10D31800010F4A4601F00F0120A83BD0FFF710F992
:10D328009DF8903084F82334259BC4F828349DF860
:10D33800983084F82C34012384F82D3430E0049A92
:10D3480002F0E002A02A1BD195F82E11012285F8DF
:10D358003A2009B927996963012B84F8202407D951
:10D36800D5F89020C4F83C24DAF80020C4F89824B2
:10D3780095F81821002AB4D1012284F82524B0E7B1
:10D38800002285F83A2084F82024A6E79DF8981012
:10D3980025984A46FFF7D4F89DF8903084F823344E
:10D3A8009DF89020E02A08D195F81F312BB984F810
:10D3B8002324C4F82834A4F82C3494F8913443F086
:10D3C800020384F891346FE6114D013EB2B2791C24
:10D3D800284604F039F80323A4F82034C4F8285464
:10D3E80084F82C64E9E7012384F82134FEF708FC6B
:10D3F8005AE694F84434002B3FF460AE0020FEF760
:10D40800EDFB94F88F34022B3FF45EAE56E600BF76
:10D41800E01E002094F89134590715D5012001F039
:10D42800CBFB60B1012001F09DFB08B984F818041A
:10D43800D4F8403323F00203C4F8403304E0062054
:10D4480001F0BAFB0028F3D194F89134DA077FF59C
:10D45800F9AC94F840240AB1032A18D11D4A94F86B
:10D46800181492F86820914205D29B0723D594F8A6
:10D478008F34012B1FD8184806F00AFBD4F8403324
:10D4880023F02003C4F84033FFF742FBDAE4012A13
:10D4980011D194F81924002A3FF4D4AC0D4A94F819
:10D4A800181492F868209142E5D29F0703D594F8A2
:10D4B8004434002BDFD194F8913400206FF3041327
:10D4C80084F8913484F81904FFF744FBBAE429B0CE
:10D4D800BDE8F08FE0160020102000202DE9F04F65
:10D4E80089468DB090460746002800F08F810029B4
:10D4F80000F08C810368002B00F088814368002BC2
:10D5080000F084818368002B00F08081C368002BC1
:10D5180000F07C81104602F007F8002800F07881BE
:10D52800BD4CBE4D384601F0C1FA40F2C45200214C
:10D53800204603F09DFF40F21C520021284603F0CC
:10D5480097FFB74BC4F82C3104F50973089304F519
:10D558000A7300264046099308A9B24B84F848800C
:10D568000A9384F8186184F88C608DF82C6001F0B7
:10D57800EDFF0F2306A994F848008DF8183001F044
:10D58800D7FF801B18BF01204FF00A0B84F81C013D
:10D5980006A994F848008DF818B001F0C9FF4FF0BB
:10D5A800060A84F8DC0006A994F848008DF818A04B
:10D5B80001F0BEFF102384F8DD0006A994F84800A6
:10D5C8008DF8183001F0B4FF1123C4F89C0006A9A7
:10D5D80094F848008DF8183001F0AAFF1223C4F817
:10D5E800A00006A994F848008DF8183001F0A0FFB3
:10D5F8001323C4F8A40006A994F848008DF818303D
:10D6080001F096FF1423C4F8A80006A994F848006E
:10D618008DF8183001F08CFF1623C4F8AC0006A969
:10D6280094F848008DF8183001F082FF172384F829
:10D63800B10006A994F848008DF8183001F078FF79
:10D6480018230DEB0301C4F8B400C4F8BC0094F827
:10D6580048008DF8183001F06BFFC0B21D2384F824
:10D66800B80084F8C00006A994F848008DF818306E
:10D6780001F05EFF1E2384F8C40006A994F8480050
:10D688008DF8183001F054FF1F2384F8C50006A94F
:10D6980094F848008DF8183001F04AFF2023C4F8A8
:10D6A800C80006A994F848008DF8183001F040FF2A
:10D6B8000B23C4F8CC0006A994F848008DF818305C
:10D6C80001F036FF0C2306A9A4F8D00094F848000E
:10D6D8008DF8183001F02CFFD4F89C306365D4F82D
:10D6E800A030A365D4F8A430E365D4F8A830236645
:10D6F8004FF00108D4F8AC300590A4F8D200636666
:10D7080084F8B080C4F894B084F898A0C4F84CB0F9
:10D7180084F850A084F8688084F81F81C5F848937D
:10D72800FEF77AFD404B009632464FF0FF3105F583
:10D738005A70C5F84473C4E90B6684F8198185F8F2
:10D748009164C5F8408306F045F9384B0096324697
:10D758004FF0FF3105F5607006F03CF9344B009648
:10D7680032464FF0FF3105F5667006F033F902AF27
:10D77800304B009632464FF0FF3105F5806006F0D9
:10D7880029F9384606F0BAF897E8030004F59273C9
:10D7980083E80300284B294F1E60294BC5F84C33FA
:10D7A800284BC5F85433284BC5F85C33274BC5F8CC
:10D7B8005033274BC5F8583305F553703B689847E5
:10D7C80004F5A67003F088FB20B1112630460DB091
:10D7D800BDE8F08F204601F01DFB0028F5D101F0CF
:10D7E80041F8B8B91B4801F067FB06460028ECD1A0
:10D7F8007B69984703F006FEBB6D94F819019847BA
:10D80800FB6A9847012385F89234DFE70326DDE7B2
:10D818000926DBE71326D9E7E0160020A81C00201C
:10D8280000040001C42100205DCB0008BDC300082E
:10D8380005C40008E5BB0008A41C0020304A010804
:10D8480009BE0008BDBD0008A1BB000895BD0008C1
:10D858006DBD0008C817002008B5034B0020C3F8A9
:10D868004003FEF781F908BDA81C002010B5FFF79A
:10D87800A7F90A4C60B90A4B93F81831022B02D168
:10D88800084BDB6A98470123C4F84033002010BDD9
:10D89800D4F84003013818BF0120F8E7A81C00207D
:10D8A800E0160020304A010838B5134C04F55A70C8
:10D8B80006F0EEF804F5607006F0EAF804F5667014
:10D8C80006F0E6F804F5806006F0E2F800F0B5FF2F
:10D8D8000A4B0025DB6A9847C4F84053FEF7B6FDAB
:10D8E8000749084840F2C45203F0AEFD0123C4F8CA
:10D8F8004033284638BD00BFA81C0020304A010824
:10D90800E01600201C11002070B52E4B8AB0054689
:10D9180093F8DD008DF8090093F8DC008DF80A0013
:10D9280029489A6A90F81804039200268DF80B008B
:10D9380004960C46002940D00692D3F88820079216
:10D948001A8F93F81A118DF8151052BAADF82020D5
:10D9580093F87C2093F848308DF8243003AB8DF889
:10D9680022008DF8232000930DF10A020DF10B031C
:10D978000DF1090105A88DF8146000F0DDFE9DF990
:10D988000900FEF713F9607004A801F02BF8B0B98C
:10D99800049A0F2A0DD863789A420AD81544AB42E4
:10D9A800A3EB02012CBF002001202170C0000AB0A7
:10D9B80070BD002323700820F9E70320F7E7132040
:10D9C800F5E700BFE0160020A81C00201FB504469C
:10D9D800002800F012810078412800F20881DFE871
:10D9E80010F0420048004D00520056005A005F00F7
:10D9F80006010601060106010601060106010601E7
:10DA080066006A006E0079008000830086008B0043
:10DA180089008D009100940097009A009D00A00055
:10DA2800AF00B300BB00B700BF00C200C600CF0004
:10DA3800CB00CD000601D300060106010601060150
:10DA48000601060106010601060106010601060196
:10DA5800060106010601DB00DF00E300E800EC0038
:10DA6800F000F400FD00674B93F81831237104B0FF
:10DA780010BD644B93F83031237102E0606803F005
:10DA8800C7FB0020F3E7606803F008FCF9E75D4B8B
:10DA980093F81A31F0E75B4BD3F8E0306360F0E7B6
:10DAA800584B211D93F8300103F010FCE9E7554B62
:10DAB80093F81931E0E7534B93F88C30DCE71C23DB
:10DAC8008DF808304F4B02A993F8480001F030FD5B
:10DAD8006060D6E74C4B043493E8030084E8030005
:10DAE800CFE74A4B0434F7E7494B0434F4E7494B92
:10DAF8000434F1E71A23E3E71923E1E7414B93F8EC
:10DB08006830B9E73F4B5B6DC8E73E4B9B6DC5E797
:10DB18003C4BDB6DC2E73B4B1B6EBFE7394B5B6E83
:10DB2800BCE702238DF80830364B02A993F87C2015
:10DB380093F848008DF80A2001F0FAFC2071A0E75C
:10DB4800304B93F8DD3097E72E4B93F8393093E755
:10DB58002C4B93F8DC308FE72A4B93F838308BE75F
:10DB6800284BDB6C9AE7274B93F8503084E7254B1A
:10DB7800D3F88430636084E7224B8FE7264B8DE728
:10DB8800204BD3F8CC30F5E71E4BD3F82C3163602B
:10DB980001F05CFDA06074E71A4BD3F890307DE784
:10DBA800184B93F81F3167E7164BB3F88830A380FA
:10DBB80067E7144BB3F88A30F9E7124BB3F8D03063
:10DBC800F5E7104BB3F8D230F1E70E4B93F8482045
:10DBD8000AB1062A13D1B3F8A035E8E7094B93F840
:10DBE80048200AB1062A0AD1D3F8A43556E72046B8
:10DBF80004B0BDE8104000F024BE032037E7182029
:10DC080035E700BFE01600204C17002094170020CD
:10DC1800541700209C1700201C1100207FB50446D3
:10DC280010B9032004B070BDA44DD5F840339A074D
:10DC380000F171820278412A00F26A82DFE812F06C
:10DC48004200480056005C00600065006A007700EA
:10DC5800820088008E0094009A00A000A600AC0004
:10DC6800B6006802BB00DD00F000170139012A0187
:10DC780044014D015101550159015D0168026101DD
:10DC880073019B018901AD01B301BA01BF01C40150
:10DC980068022A026802680268026802680268026A
:10DCA800680268026802680268026802680268021C
:10DCB8006802680236023B02400245024A024F02ED
:10DCC80054025E020079FEF7C1F80028AAD105E0E7
:10DCD8000379022BA5D07A4A82F8303195F891342D
:10DCE80043F0200385F8913400209BE7406803F057
:10DCF80081FA0028F2D094E7406803F0BFFAF8E709
:10DD08006F4B027983F81A21E8E76D4B4268C3F834
:10DD1800E020E3E76A4E416896F8300103F0CCFA58
:10DD280000287FF47EAF6368C6F8E430D6E7416820
:10DD380000293FF476AF002001F0EEF90028CDD09D
:10DD480011206FE7416800293FF46BAF0120F3E72A
:10DD5800416800293FF465AF0820EDE741680029D4
:10DD68003FF45FAF0920E7E7416800293FF459AF66
:10DD78000C20E1E7416800293FF453AF0D20DBE7B1
:10DD8800416800293FF44DAF0E20D5E741680029CE
:10DD98003FF447AF0F20CFE74A4C494B007983F84F
:10DDA8001901A36D9847E36A984797E7444B0279AE
:10DDB80083F88C2092E7424E037A8DF8043096F867
:10DDC800480096F87D308DF80530072201A901F04A
:10DDD800C2FB00283FF425AF636896F8480001931A
:10DDE800002201A901F0B7FB00283FF41AAF6C36F6
:10DDF800D4E9010186E8030070E7314E037A8DF813
:10DE0800043096F8480096F87D308DF805300722E2
:10DE180001A901F0A0FB00283FF403AFB436E7E7FF
:10DE2800274E037A8DF8043096F8480096F87D302E
:10DE38008DF80530072201A901F08DFB00283FF479
:10DE4800F0AED4E9010106F1740383E8030096F803
:10DE58001831022B7FF442AF96F83031002B3FF493
:10DE68003DAF184BDB6A9847FDF748FF36E7144E7D
:10DE7800037A8DF8043096F8480096F87D308DF8CE
:10DE88000530072201A901F066FB00283FF4C9AE5E
:10DE9800BC36ADE74368029301238DF80C30084B7C
:10DEA80002A993F8480001F063FB00287FF416AF3D
:10DEB800B7E6436802930023EFE700BFA81C0020E1
:10DEC800E0160020304A010803795A1E0E2A3FF650
:10DED800A8AE934A82F8683000E7914B42685A65C9
:10DEE800FCE68F4B42689A65F8E68D4B4268DA6526
:10DEF800F4E68B4B42681A66F0E6894B42685A662C
:10DF0800ECE6874C037994F848008DF80430062233
:10DF180001A901F020FB00283FF483AE9DF80430EE
:10DF280084F8DD30DAE67E4C03798DF8043094F815
:10DF3800480094F87C308DF80630052201A901F0DC
:10DF48000AFB00283FF46DAE9DF8043084F83930A0
:10DF5800C4E6734C037994F848008DF804300A221B
:10DF680001A901F0F8FA00283FF45BAE9DF80430EF
:10DF780084F8DC30B2E66A4C037994F848008DF8EE
:10DF88000430092201A901F0E6FA00283FF449AE5D
:10DF98009DF8043084F83830A0E6614B4268C3F835
:10DFA8009420DA649AE65E4B027983F8982083F825
:10DFB800502093E65A4B4268C3F884208EE6584BAB
:10DFC8004268C3F8CC2089E6012B40F0A480554C68
:10DFD8002421204603F04EFA636A984201D01720A4
:10DFE80020E61C2104F1280003F044FA636C9842EF
:10DFF800F5D14FF4807104F1480003F03BFAD4F8EE
:10E0080048319842EBD1D42104F5A67003F032FAD6
:10E01800D4F820329842E2D1002104F5097003F0C7
:10E0280029FAD4F824329842D9D14FF4607104F512
:10E038000A7003F01FFAD4F8A8359842CFD11421FA
:10E0480004F2AC5003F016FAD4F8C0359842C6D1A1
:10E05800334E2146304640F2C45203F0F5F92046CB
:10E0680040F2C452002103F003FA95F81B3485F8F6
:10E07800E833736FC5F8EC3396F87D3085F8F833DC
:10E0880040F20123A5F8FA33274B96F819019B6D46
:10E09800984723E68379012B3FF6C3AD204B4268AE
:10E0A8004068C3F82C2100F0D1FE47E61C4B4268BB
:10E0B800C3F8902012E61A4B027983F81F210DE667
:10E0C800174B8288A3F8882008E6154B8288A3F8A6
:10E0D8008A2003E6124B8288A3F8D020FEE5104B75
:10E0E8008288A3F8D220F9E50D4B93F848200AB1AD
:10E0F800062A12D1A288A3F8A025EFE5084B93F8C9
:10E1080048200AB1062A08D16268C3F8A425E5E5C3
:10E1180000F099FBD9E5012084E5182082E500BFCD
:10E12800E01600201C110020304A01082DE9F043B8
:10E1380087B00023ADF800300646002800F0ED80D7
:10E148000361FEF73DFD20B10124204607B0BDE87C
:10E15800F08300F073FD0028F6D100F069FD014658
:10E1680018B96F48142203F083F96E4D95F891346D
:10E17800012243F0040385F8552485F89134337857
:10E188008DF804300021013B8DF80520ADF806100C
:10E198000C2B00F2BA80DFE803F007B8B8B8788132
:10E1A800B8B88FB8AC99A800D5F8407317F0200715
:10E1B800CAD196F80480B8F1020F45D1DFF868811A
:10E1C8005A4CFEF729F896F9051098F848003A468F
:10E1D80001F01BFA88F83900B37988F838303846E6
:10E1E80007238DF80530FDF731FEFF2304F586700F
:10E1F800A5F80C31C5F8084185F8047103F04EF80C
:10E2080004F58A7003F004F83846FDF78DFE0446DD
:10E2180040B196F9051098F84800012201F0F5F987
:10E2280088F83900D5F894343361002C71D000F0A7
:10E23800FFFC002889D195F8913485F81A0460F319
:10E24800820385F8913480E7B8F1010F4FF002049A
:10E25800E8D1DFF8D4908DF8144099F8480089F88F
:10E268001D7102A901F072F9337989F830318DF8FE
:10E2780005708DF80680FDF785FC95F8913443F01C
:10E28800100385F891340024CCE700226946022067
:10E2980000F0F6FA0028F6D01324C3E7244BB2881E
:10E2A800DB6B96F90C10B0689847D5F8403343F00B
:10E2B8000203C5F84033E6E702A90D2000F060FB31
:10E2C8000028E0D0002269460D20E1E7164B93F8BC
:10E2D8001831D3B9347904F0070000F0ADFA8DF89D
:10E2E8000040012269461020D2E700226946122028
:10E2F800CEE78DF8072000F090FA044638B900F010
:10E3080089FA204600F08BFA8CE702248AE7012478
:10E3180088E701A800F0DEFB17E7032415E700BF34
:10E32800FC200020A81C0020E0160020AA1C0020C9
:10E33800304A01082DE9F04F99B08046059118B987
:10E34800032019B0BDE8F08F00230361FEF738FC05
:10E358000646002840F0AB8045460FCD0EAC0FC4F2
:10E368005A4C98F800A0B8F80C7098F90EB014221E
:10E3780004F58860314603F07BF8012284F84124D3
:10E38800534C94F83021022A35460BD194F81821C1
:10E39800022A07D194F81E2122B9BAF1010F38BF19
:10E3A8004FF0010ABAF1010F2DD0BAF1030F2CD0AA
:10E3B800BAF1000F35D102229DF83C30DDF84090CB
:10E3C800029362F34715012694F87C108DF83210F9
:10E3D80002220CA994F848008DF8302001F0A8F822
:10E3E80094F81A3194F830C194F81D1140B2022201
:10E3F800002B6FD0BCF1010F65D1002963D1002E2D
:10E408006DD1104627E00422D6E70023DDF83C90C2
:10E41800BDF840709DF942B0029365F01F050126D2
:10E42800D2E74FF0000BD946CDF808B0CCE74FF053
:10E43800010084F81A04DDE005F29A420BA900F005
:10E44800DDFA002800F020811320049B33871F4B3E
:10E45800002283F81A241D4BD3F89434C8F81030DE
:10E468006FE705F29A452A460BA900F0C7FA00287B
:10E47800EAD10B9B84F82801C4F82C5184F8303178
:10E4880002E1B9F1000F00F0FF80002A00F0FC80E3
:10E498004946E01C02F0D8FF94F837320133238054
:10E4A800F2E01220D1E70220CFE70720CFE70120D2
:10E4B80047E7064B93F8912483F840A442F0010201
:10E4C80083F89124C7E7EEB90220C4E7A81C00200E
:10E4D800E0160020002E94D05845B8BF584694F84E
:10E4E8007C308DF82000052294F848008DF8223001
:10E4F80008A901F030F800283FF422AF9DF8203039
:10E5080084F83930694A6A4BD2F89804D3F89040B5
:10E5180038B105F083FA664B84423CBF002283F889
:10E528003A20198F1A8F93F830010491996A09914A
:10E5380052BA0028B9D093F81B0100B9186393F8B0
:10E548001801ADF85820013893F87C2093F81A4147
:10E558001491D0F1000BD3F888108DF85B204BEBA9
:10E56800000B93F8482093F83A0093F868308DF838
:10E578005A3009AB00934F4B03904FF001008DF8D0
:10E588004C0015918DF85C20A3F12F01A3F1300206
:10E5980013A88DF84D4000F0CFF8039B4FEA0B1BF2
:10E5A8004BEA431B00264BEA801B4BEAC413B145D8
:10E5B8003E4C039308BF37463A46494604F59C70DB
:10E5C800CDE90A669B46268084F81A6402F03CFF6F
:10E5D800E9B2A570C5F34215FAB2042D344E039B77
:10E5E80084F837223FF423AF072D3FF44AAF022DBA
:10E5F8007FF459AF304D84F80D110420029984F846
:10E608000401FF2084F80C0184F8281184F81431DF
:10E61800D6F8E410C4F8085105F59B730AA8C4F8A5
:10E62800101184F83021C4F82C3100F017FC0028B0
:10E638007FF437AF0A9BA4F844040BA8A4F816315A
:10E64800C4F84C3400F0CEF900287FF4FDAE0B9BE3
:10E65800D3B196F93900FDF7A9FA94F83732002BAF
:10E668003FF4FFAE0B9B0F2B3FF6E6AE05F58B7222
:10E678000BA90F2000F0C2F900287FF4E5AE0B9B30
:10E6880063F3030B84F814B10598FDF74DFC0028DB
:10E698007FF4DBAE099B86F83A00B36200F07EF99E
:10E6A80000283FF406AF1320D1E600BFA81C0020C5
:10E6B800E016002048170020AA1C002037B50B4D93
:10E6C8008DF8040004460F2295F8480001A900F0CF
:10E6D80042FF40B1064A85F81C4192F8913443F054
:10E6E800200382F8913403B030BD00BFE01600204B
:10E6F800A81C002010B5FFF7B9F8044688B90A48E5
:10E7080005F0C6F9094805F0C3F9094805F0C0F94C
:10E7180000F093F8FDF780FD064BDB6A984720462A
:10E7280010BD0124FBE700BF102000202820002096
:10E7380040200020304A01082DE9F04F8BB047787F
:10E748000093149B90F90C8090F90D6090F80E904E
:10E758008B464168196004469246002F57D0022321
:10E768008DF8103004A9C37B007C8DF8123000F0BE
:10E77800DFFEB4F808C0618943B260689845454631
:10E788006144B8BF1D46604534BF00270127884251
:10E7980009D30A218DF81010207C019304A900F0F8
:10E7A800C7FE019B46B2B4F808C0608961680CEBEB
:10E7B800400E714520D3A1EB0C01B1FBF0FC00FB2E
:10E7C8001C11C9B998450ADC237833B10223207C8F
:10E7D8008DF8243006A900F0B9FE4FF00109212375
:10E7E8008DF81030207CE37B8DF8115004A98DF84A
:10E7F800123000F09DFE45B2009B8BF80050384661
:10E808008AF8006083F800900BB0BDE8F08F4546A9
:10E81800F2E77047704770477047002070477047AD
:10E8280070477047002070470020704700207047ED
:10E8380000207047002070477047704770470220DB
:10E8480070470220704702207047704700207047C9
:10E858007047704700207047002070477047704726
:10E868007047000010B5054C4FF403722046002194
:10E8780002F0FEFD0020C4E9000010BD682200205F
:10E888002DE9F8438146174600293FD0244B00253F
:10E8980003F1010C1A462801103312F8018FB8F160
:10E8A800000F36D19A42F8D11E4E33680BB9C6F81C
:10E8B80000C073680BB1C3F800C0331800240135D9
:10E8C8009C6083F80C900D302B01BAB206EB05154D
:10E8D8003044F750C6F804C002F0B6FDB9F1110F84
:10E8E8004FF0000398BF104C6B71D6F8083298BFF0
:10E8F80024FA09F403F1010398BF04F001043B442E
:10E908002C71C6F808324046BDE8F8834FF001087C
:10E91800F9E70135202DBBD14FF00208F3E700BF1E
:10E928006F220020682200202007020010B510B3D3
:10E93800124A1368984204D103681360002304E064
:10E948000B4613B119688842FAD15168884208BF4A
:10E9580053600BB101681960D2F808328168013B35
:10E9680000245B1A04602146C2F80832102202F023
:10E978007FFD204610BD0120FCE700BF6822002073
:10E98800054B1B6813B11A798242FAD1002B0B6030
:10E998000CBF0320002070476822002010B5054BEB
:10E9A800186800B910BD037B04680BB9FFF7BEFFF8
:10E9B8002046F6E76822002038B5084B084C18684E
:10E9C80000B938BD03790568112B05D824FA03F37B
:10E9D800DB0701D5FFF7AAFF2846F1E768220020E8
:10E9E8002007020028B1044BD3F808320360002046
:10E9F80070470120704700BF682200202DE9F041D0
:10EA080007460E4615463AB331B3144B1C6800232B
:10EA18002CB93046FFF7E6FF0020BDE8F081A26878
:10EA2800F91A0132914210D32279EA54581C2289EA
:10EA38005FFA80F8611D55FA80F002F005FDA368C1
:10EA4800246898445FFA88F3E2E720462468FFF7D1
:10EA58006DFF002CF9D1DCE70120DEE768220020F9
:10EA68000238C0B211289ABF014B185C00207047C9
:10EA78003F43010830B50B4B93F820200446084665
:10EA880072B100211C330578A54208D001319842A3
:10EA9800CDB20CBF04480430AA42F4D8002030BDDF
:10EAA8001046FCE7742400208024002010B5084C90
:10EAB80000232060142204F10C00FF2184F8203088
:10EAC800C4E9010002F0D4FC012384F8213010BD10
:10EAD8007424002010B50E4A92F82010042915D885
:10EAE800936804781C7044785C70C4788078987057
:10EAF8000131DC7082F8201002F11C018B4214BF36
:10EB0800043302F10C039360012010BD0020FCE7E0
:10EB180074240020094B93F8200068B15A6803F167
:10EB28001C018A4200F1FF3014BF043203F10C02C9
:10EB380083F820005A600120704700BF7424002029
:10EB480010B5074B93F820200446084632B159689F
:10EB5800FFF790FF10B101234470837010BD00BF10
:10EB68007424002008B5064B93F820202AB1596870
:10EB7800FFF780FF08B1407808BD0120FCE700BF1F
:10EB88007424002030B50A4A92F82010536882F89D
:10EB9800210061B1916801241C32DD78587005B9F3
:10EBA8009C7093420CBF034B04339942F5D130BD9E
:10EBB800742400208024002008B5044B5968FFF70E
:10EBC80059FF003818BF012008BD00BF7424002079
:10EBD8002DE9F3410422154E044600210DEB0200F5
:10EBE80096F8208002F044FC0025EBB2984502D844
:10EBF80002B0BDE8F0817368197821705A786270A4
:10EC08009F785FB1336820469B689847FFF782FF7B
:10EC180017B901A8FFF75EFF0135E6E7DB788DF845
:10EC280004108DF805208DF80730EFE774240020D4
:10EC3800014B93F82000704774240020034B93F88D
:10EC48002000042894BF002001207047742400206D
:10EC58001FB50024CDE90244C41F8DF800408DF88B
:10EC680001100C0AADF80420090C120C8DF80310E1
:10EC78008DF806208DF8073002461B0A01216846E8
:10EC88008DF802408DF8083002F04FFA002818BFBE
:10EC98000E2004B010BD2DE9F04188B017460D468E
:10ECA8000F9A064600284DD000240121CDE90444DE
:10ECB8008DF810109DF838108DF81510ADF8163035
:10ECC800190CCDE900441B0ECDE902448DF819302A
:10ECD800ADF81A20130C120E07948DF818108DF841
:10ECE8001C308DF81D20E3B24FEA0318002D5FFA9F
:10ECF80088F803DC002008B0BDE8F081013310215A
:10ED08008DF81F303A466B460DEB010002F0A3F96F
:10ED18000346C8B9102DAC46A8BF4FF0100CDAB2A4
:10ED2800624503F1010303DB103D2DB20134DAE73C
:10ED380008EB020020326A44315C12F8202C4A4069
:10ED48003254ECE70920D6E70E20D4E7013803282F
:10ED580015D8DFE800F002080C100A4B1B681B6985
:10ED68000B6000207047074B1B685B69F8E7054B91
:10ED78001B689B69F4E7034B1B68DB69F0E7052018
:10ED8800704700BF982400202DE9F041C4B00C461C
:10ED98004A9E17461D468046B8B3B1F5807F36D8DF
:10EDA8004FF488720021684602F062FB4923009301
:10EDB8004FF48073ADF804302B0C8DF80830330C09
:10EDC800ADF80650ADF80A608DF80C3022460023E5
:10EDD800414604A82D0E360E8DF80E308DF80950D8
:10EDE8008DF80D608DF80F4002F02EFB04F1100134
:10EDF8004B9A3B4689B2684602F017F910B10128D0
:10EE080018BF0E2044B0BDE8F0810920FAE70D20B4
:10EE1800F8E7000010B590B10A4C282200212060C4
:10EE280002F026FB2368084A1A6000204FF0FF32E0
:10EE3800C3E90302C3E90522C3E9072210BD08207C
:10EE4800FCE700BF9824002000010101024B1B6869
:10EE580018600020704700BF9824002030B1044B90
:10EE68001B68DB6801330360002070470920704786
:10EE78009824002013B500230C460193D2B101A9B0
:10EE8800FFF764FF18B9019B591C02D1146002B046
:10EE980010BD99B2611A002902DD0B441360F6E730
:10EEA80002D113600720F2E71B0C1B0403F5803323
:10EEB8002344F3E70920EAE728B1044B1B681C3315
:10EEC8004362002070470920704700BF9824002043
:10EED8001FB5044600B3002303A8039302F07CF98E
:10EEE800104ABDF80C30126820469380E38200F087
:10EEF80056FA98B904F118030093216801231322E4
:10EF080002F08AF860B9204600F049FA003818BFC4
:10EF18000120000104B010BD0920FBE71020F9E72B
:10EF28000E20F7E798240020F0B5054687B01C4668
:10EF38003BB32F4E3368DB68834257D894F82020C0
:10EF4800002A14BF09220822834205D3204600F074
:10EF58005AFA70B110200AE0002301900093A368C8
:10EF680094F82810606AFFF796FE0028EED007B0E4
:10EF7800F0BD23792168B4F808C0A768043B9AB2A9
:10EF880009B90920F3E7B2F5807F2DD8ADF80EC096
:10EF98008DF817304FEA174C04F12C033F0E8DF80B
:10EFA800117000932F0C08234FF0490EADF80C0098
:10EFB8008DF814708DF816002F0E0DEB0300CDF8A8
:10EFC80008E08DF810C0ADF812508DF8157002F0F9
:10EFD80023F808B10E20CAE7204600F014FA0028EA
:10EFE800B8D13368DD60C2E70D20C0E70620BEE770
:10EFF800982400202DE9FF410A9D80460F461646B9
:10F008001C46002D5AD0002303A910460393FFF78E
:10F018009DFE18B1062004B0BDE8F081039B9C4218
:10F0280001D80133F6D1284600F05EF9002847D10F
:10F03800264B1A78424503D01A79424542D101201D
:10F04800AA68BA4240D103EB8002EB6A92F80180C9
:10F058002979CDE900430439927828683B4689B27A
:10F06800FFF792FE0028D6D195F820300194002BA6
:10F078004FF00103009314BF4246082295F8281068
:10F08800686A3B46FFF707FE0028C4D1013E032EFD
:10F09800C1D8DFE806F002070B0F0D4B1B681C6197
:10F0A8001C62B8E70A4B1B685C61F9E7084B1B68F0
:10F0B8009C61F5E7064B1B68DC61ACE70920AAE711
:10F0C8000F20A8E70B20A6E70220A4E7A408002049
:10F0D800982400201FB50A460B2A4FF00001CDE9FD
:10F0E8000011CDE9021107D00C2A13D00A2A0FD03B
:10F0F8000A2005B05DF804FB012802D120238DF811
:10F108000030684602F011F8002818BF0E20F0E71A
:10F118003023F4E70B21F4E738B5054602F000F890
:10F12800044678B97DB9094B1B680B219878FFF71D
:10F13800D1FF38B90C21FFF7CDFF18B90A21FFF725
:10F14800C9FF00B10E24204638BD00BF9824002016
:10F158002DE9F04380468FB00C461746002A6BD045
:10F16800002969D0002529461D2206A8059504F026
:10F17800A1FE8DF81350344D2B680DF114099E88AB
:10F18800CDF804900DF1130302933B7900933B688B
:10F1980032462146404601F0E4FF00284ED1386847
:10F1A8003A79494602F050F9384600F04FF80028FD
:10F1B80046D13C7AFA79BB79240444EA02241C43F8
:10F1C8002B689A6894423DD99C609DF813000B21E6
:10F1D800FFF780FF034658BB0C21FFF77BFF034670
:10F1E80030BB0A21FFF776FF034608BB7B7ABA7A61
:10F1F800FF7A3F0447EA02271F433A46334621462F
:10F208000920FFF725FD034690B933463A462146C3
:10F218000820FFF71DFD034650B92A689DF8131012
:10F2280091700021D1604FF0FF31C2E90411916162
:10F2380018460FB0BDE8F0830923F9E70E23F7E776
:10F248000F23F5E70323F3E79824002010B50446BD
:10F25800002845D00168002942D011F8013B4371CC
:10F268000322063002F0F0F82046032250F8091B6A
:10F27800043102F0E9F82168CB79E3600A7A43EABD
:10F288000223E3604A7A43EA0243E3608A7A43EA64
:10F298000263E360CB7A23740B7B63742379212B9D
:10F2A8001AD110220D3104F1120002F0CDF81D22FE
:10F2B8002168501C8B5C6362085C43EA0023901C45
:10F2C8006362085C033243EA004363628A5C43EA90
:10F2D80002636362002010BD112B03DC0D22E7E7F7
:10F2E8000220F8E70120F6E710B50446002854D0BC
:10F2F8000168002951D00B7843714B7883608A7874
:10F3080043EA02238360CA7843EA024383600A79A6
:10F3180043EA026383604B7903738B79C381CA79AB
:10F3280043EA0223027BC38102F00F020831103046
:10F3380002F08AF8237B002203F00F0384F82020D0
:10F3480084F82820227903F10800111A04290DDD18
:10F3580021680933043AD21A085C84F82000D2B232
:10F36800606A84F82820194402F06EF8237922682C
:10F378001A44002012F8043CE36212F8031C43EA22
:10F388000123E36212F8021C43EA0143E36212F824
:10F39800012C43EA0263E36210BD0220FCE710B5CA
:10F3A800044660B3036853B30279162A29D942790F
:10F3B8001A700146082251F8060B013002F04EF887
:10F3C8002146082251F80E0B093002F047F823684D
:10F3D800E28A5A74E38A22681B0A93742368A26932
:10F3E800DA74A36922681B0A13752368628B5A753D
:10F3F8002368E27E9A7517232371002010BD01202F
:10F40800FCE70220FAE738B50446002863D0016813
:10F41800002960D0037B90F8282003F00F03002A0E
:10F4280057D10833207904321344984255D363796D
:10F438000B702368A2685A70A36822681B0A93702D
:10F4480023686289DA702368E27A1A712368227B5A
:10F458005A712368E2899A71E38922681B0A214656
:10F46800D371227B51F8100B02F00F02083001F023
:10F47800EBFF237B94F8282003F00F0303F1080522
:10F488002AB1226894F82010515503F10905206823
:10F4980094F82820616A284401F0D6FF94F82830AF
:10F4A8002268E16A2B44D1545A1CE16A206892B25E
:10F4B800090A81549A1C2168E08D92B28854DA1C9A
:10F4C800216894F82F0092B20433885423710020E5
:10F4D80038BD0933A6E70120FAE70220F8E7000063
:10F4E800024B1A8810431880704700BF9C240020E4
:10F4F80008B5074B1B883BB1FEF7B8F900280CBFCD
:10F5080000206FF0020008BD6FF00100FBE700BFAC
:10F518009C24002010B5034B00241C80FEF79CF9A6
:10F52800204610BD9C240020B0FA80F040097047A6
:10F5380082B018B9084602B000F0CAB8002002B07C
:10F54800704710B9084600F077B9704710B90846F7
:10F5580000F08EB970470346084611460BB900F013
:10F56800E5B90020704710B9084600F071BD704732
:10F5780010B9084600F006BA0020704710B40446D7
:10F58800084611461A46019B14B910BC00F018BA77
:10F5980010BC70470346084611460BB900F042BA42
:10F5A8000020704710B40446084611461A4614B99C
:10F5B80010BC00F0AFBA002010BC704730B405464C
:10F5C800084611461A46DDE902341DB9029430BCDA
:10F5D80000F02EBB002030BC704710B9084600F080
:10F5E800DFBB0020704710B9084600F06FBD00204F
:10F5F800704710B9084600F0EEBB0020704710B9FC
:10F60800084600F0EBBB0020704703460846114649
:10F618000BB900F005BC0020704710B4044608463A
:10F6280011461A46019B14B910BC00F0FBBB092017
:10F6380010BC704710B40446084611461A4614B95F
:10F6480010BC00F063BDC8B210BC704700487047DA
:10F6580001000102064B10B51B6A0446984730B1F9
:10F668000448054B204498428CBF0020012010BD5F
:10F67800304A010840C220C980B92A00F0B5114BB0
:10F6880085B00C4610491F56054601F049F80F4B46
:10F69800E4B25E6A072D4FF00103CDE9024301464B
:10F6A8000AD105220023CDE900234FF47A727A4368
:10F6B8001846B04705B0F0BD08220020CDE900206B
:10F6C8003A46F5E77B43010854430108304A0108EC
:10F6D8001FB5002300930378013B372B21D8DFE8BF
:10F6E80003F01C242020201E202020204143454ECA
:10F6F8002055585B5E6164206C1E6E73787A2020FA
:10F708007D8126202020202020202020202020202D
:10F7180083858A2020838A208C90C3780BB10223AA
:10F728000093009805B05DF804FB8378F6E743780A
:10F738008DF8043005238DF805308378003B18BF19
:10F7480001235B008DF8063010238DF80730304B0D
:10F758001B6801A803F55872CDE9022300F0C0FF29
:10F768000090DEE74023DBE72023D9E7827890F991
:10F77800013012B9274AD35CD2E7274AFBE78278DF
:10F7880090F90130002AF8D1244AF4E740F6B8335A
:10F79800C6E74FF47A73C3E74FF4FA63C0E741F260
:10F7A8008833BDE741F27073BAE71D484FF47A71A8
:10F7B80001F02EFE00F5FA60D2E71A4BB0E7144BC1
:10F7C8001B6803F55873ABE7114B1B6803F55B73B4
:10F7D800A6E71023A4E70E4B1B68A1E74FF083436D
:10F7E80000939EE7104BFBE7104B99E740F211138B
:10F7F800ADF8003095E7032392E790F901300C4A01
:10F80800B9E70C4990F9010000F08AFFA8E700BFAA
:10F81800A4240020034401080B44010813440108F0
:10F8280018FCFFFF00EA06379A99094040F70937A4
:10F838007B4301085443010837B50B4B02781B681A
:10F848000C2101FB02335B7A03EB4304074B1D6871
:10F8580003690093C3684278816805EBC40000F02F
:10F86800DFFC03B030BD00BFA4240020A02400208A
:10F8780070B586B0027B6423ADF80030012A4FF0E2
:10F888000003CDE90133CDE903338DF802308DF85B
:10F89800143030D0022A39D05ABB03684BB34368BE
:10F8A8003BB31F4D80682B601E4B182269461860B9
:10F8B80001F0CAFD1C4B2C6893E807000C3384E860
:10F8C800070093E8070004F10C06032386E8070005
:10F8D800A4F86C33012204F55B7104F5587000F04C
:10F8E80090FC2B684FF6B072A3F878230522C3F872
:10F8F8007C2306B070BD0A4908684360036100F5BF
:10F908005B7100F5587000F07CFCF2E7044B1B6853
:10F91800B3F86023B3F86C130A43A3F86023E8E74D
:10F92800A4240020A0240020A840010808B503460C
:10F938000A2924D8DFE801F006232323230B161B0A
:10F9480023212100BDE808400068FFF783BE90F935
:10F9580000009978052271B900F013FC003818BF2F
:10F96800012008BD052293F900000021F4E790F971
:10F9780000005978EEE70221EEE70722F3E70020BE
:10F98800EFE7000010B504791CB1012C0BD0002062
:10F9980010BD0A4B01681B68012203F5587000F07E
:10F9A80030FC0120F4E7054B01681B68224603F58B
:10F9B8005B7000F026FC2046EAE700BFA424002084
:10F9C800F7B50528144D1C46A8BF052058700E46EB
:10F9D8002946174600F0A4FE94F90130A070072BC1
:10F9E80013D1322000F09CFD0C4BDB6D0546984787
:10F9F80004F10C0208340346019200943A46314659
:10FA0800284600F092FD03B0F0BD054A55F82310D2
:10FA1800D05C00F07DFDE7E754430108304A010857
:10FA28007B4301082DE9F04F344F90F901607B6862
:10FA3800D0F804908BB004468846984705460028BD
:10FA480059D1E37C73B92E4A2378126803EB430338
:10FA5800990002EB8303D3F80490B9F1000F01D1A8
:10FA680052F80190274B484613F906B0FB689847AF
:10FA7800A37CD7F818A022890993072E28D1002340
:10FA88000121CDE90223204A0693CDE90431CDE9CD
:10FA980007330521CDE900214FF47A7202FB0BF2FE
:10FAA8004CF250311846D047637C13B3174B995D1D
:10FAB8007B6D0D31C9B228469847E07C32464946ED
:10FAC80000F040FE88F8006001200BB0BDE8F08F20
:10FAD800002101250823CDE90013CDE90715CDE95B
:10FAE8000511CDE903110292A1782B465A46284602
:10FAF800D9E7074BDBE70020E7E700BF304A0108FA
:10FB0800A42400207B430108854501001344010813
:10FB1800034401082DE9F04F8DB090F90130DFF86A
:10FB2800FCA0DFF8FC90CDE90A123E4A12F903B0B6
:10FB38000278DAF800300C2505FB02333A4A5B7A82
:10FB4800126803EB430302EBC303044693F9021064
:10FB580090F9020000F0DFFD3449064694F90100EF
:10FB680000F0DEFDA26861688046304600F005FDC1
:10FB78002178DAF80020D9F80C3069430746505844
:10FB88009847D9F81C309C4694F901300025072B7A
:10FB98004FF47A63CDE90753CDE905552DD10123FB
:10FBA800CDE903530523CDE901534FF47A7303FBE1
:10FBB8000BF300933946434646F2A8122846674697
:10FBC800B8472378DAF800200C214B4394F9011048
:10FBD800D05800F0D9FDA18994F90100FFF74EFD36
:10FBE8000B9B217B1860D9F85430284698470A9B0C
:10FBF80001201E700DB0BDE8F08F01200823CDE96B
:10FC08000350CDE901032A46CDF800B065464346C6
:10FC18003946A84701200546D3E700BFA4240020A1
:10FC2800304A01087B430108A024002054430108FE
:10FC38002DE9F04F8FB0002405468A469146984634
:10FC48000494ADF81440ADF8024007264FF0010BBC
:10FC58002B7AA34206D9686804A9204400F0F2FB75
:10FC680000285ED102238DF8083002A86B7A8DF83F
:10FC78000A30FFF72DFDAB7A8DF81D309DF8113055
:10FC88008DF81E309DF812308DF81F309DF8103019
:10FC98008DF82030EB7A8DF821302B7B8DF82230CF
:10FCA8006B7B8DF8233010238DF81C608DF8243081
:10FCB8003A4E8DF82C000DF102030A9305238DF8B6
:10FCC8002D3033680C930723ADF834302B68069336
:10FCD8000DF1120204AB0DF1110106A800F0CCFBE6
:10FCE800072805460BD130680C22002100F5587012
:10FCF80001F0BEFB3368BDF80220A3F860239DF82D
:10FD080011308AF800309DF8123089F800309DF8DB
:10FD1800103088F80030189B28461C700FB0BDE8DA
:10FD2800F08F9DF81330BDF81470ADF802702044C0
:10FD3800C4B2F3B917B3194A00201168072602465E
:10FD48004FF00C0C062B1BD10CFB00FE51F80EE0FB
:10FD5800BEF1000F04D00BFA00F23A4397B2012229
:10FD680001301028EED1002A3FF472AFADF80270CE
:10FD78006EE75A1E042A01D9062BDCD0062667E74F
:10FD880047FA00FE1EF0010FEAD00CFB00FE51F806
:10FD98000EE0BEF1000F08BF0626E1E7A42400200C
:10FDA80038B505464068FFF755FC0522841D00213B
:10FDB80095F90000E4B200F0E4F908B904F0FD0494
:10FDC80095F901000722002100F0DBF908B904F0D9
:10FDD800FB04204638BD00207047000010B50378AA
:10FDE8000F2B044618D84068FFF734FC22780B49DB
:10FDF80002EB42020968831C01EB820051F82220C1
:10FE0800DBB21AB903F0FD0358B210BD032B06BFCD
:10FE1800626842600223F7E70020F6E7A424002086
:10FE2800022070472DE9F04FDFF838810446D8F8F2
:10FE3800000099B08946174600211E460122032377
:10FE480000F55870CDE90611CDE908118DF81410A8
:10FE58008DF81510ADF8163000F0B5F938B9D8F8A6
:10FE68000020B2F8603343F00303A2F86033D8F8F7
:10FE78000020637A8DF8283002F55871CDE90B120D
:10FE8800394A94F9083012680D920DF116020F9252
:10FE98002268109262681192D4E90301A27A8DF85F
:10FEA800482001228DF8492013AA82E80300102572
:10FEB800227DE18A8DF8293018468DF85420ADF856
:10FEC8003850FFF7DBFB0AAB17930DF115031690BB
:10FED80000933146019705AB06AA10A800F0BCFBB9
:10FEE800064698BB9DF81410204F013901F090FA8E
:10FEF8001F4B1B690393C4B24FF00C0B04F1600352
:10FF08006B44D8F8000013F848AC9DF814300BFB8C
:10FF18000AFC01343946B4FBF3F203FB1244D0F86F
:10FF28007C33B0F9782350F80C00DDF80CC0E4B24B
:10FF3800E04728B189F800A0304619B0BDE8F08F35
:10FF4800013D15F0FF05D9D10D26F5E70C2801BFB5
:10FF5800D8F80020B2F8603343F00303A2F8603306
:10FF6800EAE700BFA4240020A0240020400D0300DD
:10FF7800304A0108F8B50679012E054601D8062051
:10FF8800F8BD0F2E2BD80368187A40F3030005221A
:10FF9800002140B200F0F5F82B680446187A40F3C7
:10FFA80003100522002140B200F0EBF8A8B1B4FA22
:10FFB80084F4640929680B7A086843F3030243F35D
:10FFC800031352B25BB29A42C8BF0124FFF742FB47
:10FFD80048B9002CD3D10420D2E70124EAE7032052
:10FFE800CEE70520CCE7002CFBD10C4F29683B68F5
:08FFF80006EB460003EB80005C
:020000040801F1
:100000000C2201F025FA3A680C2303FB0623204654
:100010005C72B2F860130123B3400B43A2F8603363
:10002000B2E700BFA424002010B4017801290ED942
:10003000084B18680C234B43C4180022C250C4E973
:10004000012200F5587010BC102200F0A7B8002063
:1000500010BC7047A42400202DE9F04186B0502345
:100060008DF81430037A102B074630D14368DD7BBE
:100070006DBB0224A8466426062C14D87A68535D0A
:1000800003932A44517843EA01230393927843EA85
:1000900002437343CDE9033863B968468DF80040E5
:1000A000FFF7C2FF0DE0CDF80C808DF81480CDF87D
:1000B0001080F2E703AB01A801938DF80840FFF729
:1000C0005DFF0134E4B2102C05F10305D4D106B074
:1000D000BDE8F0811FB502680379116851B901A824
:1000E0008DF80430FFF7A0FF78B9002040B205B0CA
:1000F0005DF804FB02A802928DF80C30FFF73EFF7A
:100100000628F2D8024B185CF0E70320EEE700BFA8
:1001100074430108C90020B9034B0B449856C0B280
:100120007047024BF9E700BF83430108C34301084E
:10013000F0B59A42069D03DB9DF914309A4220DD0A
:100140000020F0BD03EB430331F814C005EB83033B
:1001500000264CFA06F7FF0707D51F7A07F00F0EA7
:10016000724502DBB2EB171F0DDD0136102E03F1D5
:100170000C03EED10134E4B22301DBB29842E1D8A2
:10018000DEE70024F8E70120DBE7884204DB904249
:10019000CCBF0020012070470020704710B5140923
:1001A000B4EB111F03464FEA11100ED391420CD24B
:1001B00002B201F00F0133F81240012000FA01F100
:1001C00024EA010123F8121010BD0020FCE7F0B56D
:1001D00028B100EB410501270020914200D3F0BD7A
:1001E000002435F802CB234607FA04F636EA0C065B
:1001F00008BF013304F1010408BFDBB2102CF3D1B6
:1002000018440131C0B2C9B2E7E710B500B149B92D
:1002100010BD31F8134020F813400133DCB2A24284
:10022000F7D8F5E70023F9E782B030B504880493E6
:100230006AB9B3F5616F18D349F6AF2542F210726F
:10024000AB4298BF4FF47A72944238BF1446012CE7
:1002500038BF01246143BDE83040C3688B428CBF86
:100260005B1A0023C36002B070476422ECE7000011
:100270002DE9F04F91B01546DDF86C8004939DF8A0
:10028000683009930C46064603F0C2FB684ADFF863
:10029000A4B10590A8F5F633303BB3FBF2F353431A
:1002A00003F5F63203F5A83303F5C073039318235F
:1002B00013FB054330320692089300254FF0FF3AB6
:1002C000089BA34207D1002D14BF50464FF0FF30CA
:1002D00011B0BDE8F08FBDF97030ADF82C300B993E
:1002E000CDF86C804046CDF8288003F021FBB4F8AF
:1002F00000906EB9B8F5616F5BD349F6AF2242F258
:100300001073904598BF4FF47A73994538BF99465A
:100310004B46012B38BF01230793002E52D1B9F170
:10032000640F48D1A0605F46A1680EA803F022FBCD
:100330000F9B0093DDE90A120E9B0CA803F079FADB
:10034000049B0C9A0BB9099B2BB12369BB4202D1C8
:10035000394B9A420DD9394BE760984509D90023AA
:10036000ADF83430069B0D990C93184603F0E0FA73
:10037000A060606800B9E760276126B103F052FB16
:10038000E3680344E360D4E903329342059B1D997B
:100390006360079B88BFE2604B43E168994202D2E9
:1003A0000498A8B9A6B101231D442375EDB21834F1
:1003B00086E76423A9E7B9F57A7F0ABF204F214F6A
:1003C000A060B1E7049B0BB9C4F80CB05F46D0E75E
:1003D00000209342207506D85B1A9A4505F1010565
:1003E00028BF9A46EDB2002EE1D1B9F1640F164A4A
:1003F000ADF8346019D049F6B023B9F57A7F18BF4B
:100400001346904584BF039A9B180C931C9B009342
:100410000CAF97E806001B9B384603F00AFA97E8F2
:10042000030003F085FA8246C1E74FF46163E8E711
:100430008051010040771B007F5101002FEC01002B
:1004400080A81201002E930230EC01000378032BE8
:1004500014D1437803F00F021B098A704B70837824
:100460008B80C27843EA02238B800379C3F30212A4
:1004700003F00F03CA700B7005207047002070470F
:100480002DE9F34798464379057990F9076091463D
:10049000044690F906208A4683B190F9087075B336
:1004A0000F2A12D194F909200F2E1ED194F90A6057
:1004B000072D24D1002F08BF012720E090F90B70F1
:1004C00090F9092090F90A60E9E7A369019394F98A
:1004D00015300093216994F91430207BFFF728FE32
:1004E0000028E1D105F0FD05DEE794F91D30B342A7
:1004F0000FDC94F91C30B342DADA05F0FB0528462C
:100500008AF8002089F8006088F8007002B0BDE821
:10051000F0871E46CCE70000024B03FA00F0B0FB68
:10052000F1F0704740420F004FF4FA53B3FBF0F084
:10053000704730B54FF47A750C1F6A4300FB0422F4
:1005400052001EBF00F1FF341219B2FBF0F29142CB
:1005500038BF1146039A1160820048431CBF013026
:1005600040084FF47A71121A01FB1323002BCABF03
:1005700003F2E73393FBF1F1B3FBF1F1049B196054
:1005800030BD38B5400014460D46F1F743FA014638
:100590002846F1F78DF92146F1F78AF9F1F77CF851
:1005A00003F0DAFCF1F758F940B238BD2DE9F74F06
:1005B000019300231F469C461C01058A5FFA84FEB6
:1005C00004F0F004A54206D8019B82F800C01F7019
:1005D00003B0BDE8F08F0EEB4E054FEA4309AD00C6
:1005E0000024466836F809602641F60727D5866854
:1005F00006EB050A765916B3067836B9466926B170
:1006000036F809602641F60719D59AF8086090F97E
:1006100001B046F303084FFA88F8D8450FDC46F3DB
:10062000031676B25E450ADB9AF8096006EB4608C7
:10063000C66806EBC806367D4EB90137FFB20134F5
:10064000102C05F10C05CCD10133DBB2B4E70CF171
:1006500001060EEB040801F80C805FFA86FCEEE759
:100660002DE9FF4704464068DDE90C671D468A46D0
:10067000914603F0D7F923681B1A3B604FF000083E
:100680000123337085F80080636813B123688342C7
:1006900024D8CAF80080D4F81CC0A3699CF800E0F4
:1006A0000393D4E9030101AB83E80300237D0093A6
:1006B000DCF80C10237A627A7046FFF7D9FD3346D6
:1006C00038602A46E0694946FFF770FF2B782BB166
:1006D000C7F80080002004B0BDE8F0873378002B15
:1006E00014BF0B200C20F6E737B590F9002090F9E5
:1006F0000250954204460FD0013A52B295420BD0B7
:10070000A368019394F9013000936168E0782B4667
:10071000FFF70EFD0028EFD0104603B030BD884231
:10072000B8BF08467047000051F82000054B9842BA
:1007300005D0054BC31A584258414000704701206C
:10074000704700BF90D0030020A1070005281FB507
:100750000ED80C4B53F820300093CDE901120A4B10
:1007600001220021022002F069FE05B05DF804FBC1
:10077000CDE90012054B01220021022002F05EFEAD
:10078000F3E700BF884401081B4401083A4401080C
:1007900007B5054BCDE9000101220021022002F03E
:1007A0004DFE03B05DF804FB5644010810B510225D
:1007B00004460021F13000F05FFE0021C4F814115E
:1007C0002046F022BDE8104000F056BE0246084622
:1007D000102100F0A5B92DE9F0430446D0F814012A
:1007E00085B00E46154604F2011988B3C0F1100811
:1007F0009045474628BF1746BAB2484400F028FE45
:10080000D4F814313B440F2BC4F814312DD9A8452A
:100810002BD204F1F00304F5807113F8012F187C3A
:100820008B4282EA00021A70F7D104F1F10810221B
:100830004146684600F00CFE22466946684600F0D4
:10084000E9F910226946404600F002FE3E44ED1BE5
:1008500004F5807804F1F107102D09D8AAB23146C9
:10086000484600F0F5FDC4F8145105B0BDE8F0832A
:1008700004F1F003711E13F8012F11F8010F434525
:1008800082EA00021A70F6D110223946684600F05A
:10089000DFFD22466946684600F0BCF91022694631
:1008A000384600F0D5FD1036103DD5E7F0B589B0DB
:1008B0000C46102200210546684600F0DDFD224668
:1008C0006946684600F0A6F99DF90030002B6A469B
:1008D0004FF0000143DA137812F8010F01315B0089
:1008E00043EAD0130F2902F8013CF4D19DF80F30F0
:1008F0005B0083F08703D4F81401DBB210288DF875
:100900000F303BD104F58073694604F5887013F805
:10091000016F11F8012B984282EA06021A70F6D193
:1009200004F1F00304F5807113F8012F187C8B4259
:1009300082EA00021A70F7D110220DEB020004F1D6
:10094000F10100F085FD2246294604A800F062F975
:1009500010220021684600F08FFD09B0F0BD137829
:1009600012F8010F01315B0043EAD0130F2902F89E
:10097000013CF4D19DF80F305B00BCE79DF90030DD
:10098000002B6A464FF0000137DA137812F8016F36
:1009900001315B0043EAD6130F2902F8013CF4D180
:1009A0009DF80F305B0083F08703471CDBB28DF8A6
:1009B0000F30102F04EB0003C0F10F064FF0800240
:1009C00088BF002600F5817083F80121002132469E
:1009D00020443E4403F072FAC4F8146104F58073B5
:1009E000694604F5887013F8016F11F8012B9842DD
:1009F00082EA06021A70F6D192E7137812F8016FB4
:100A000001315B0043EAD6130F2902F8013CF4D10F
:100A10009DF80F305B00C8E70A78037853400370F5
:100A20004A784378534043708A7883785340837080
:100A3000CA78C3785340C3700A790379534003716D
:100A40004A794379534043718A798379534083715A
:100A5000CA79C3795340C3710A7A037A5340037247
:100A60004A7A437A534043728A7A837A5340837234
:100A7000CA7AC37A5340C3720A7B037B5340037321
:100A80004A7B437B534043738A7B837B534083730E
:100A9000CA7BC37B5340C373704710B50B7814787F
:100AA0006340037054784B786340437094788B783C
:100AB00063408370D478CB786340C37014790B792A
:100AC0006340037154794B796340437194798B7916
:100AD00063408371D479CB796340C371147A0B7A04
:100AE00063400372547A4B7A634043728B7A947AF0
:100AF00063408372D47ACB7A6340C372147B0B7BDE
:100B000063400373547B4B7B63404373947B8B7BC9
:100B100063408373CB7BD27B5340C37310BD000013
:100B2000A1F11003DBB2102B2DE9F04704D8374CAC
:100B300024FA03F3DB0705D4002382F8F030FF200A
:100B4000BDE8F087531E4418A0424ED101F11C03AA
:100B50009B005FFA83F9C3F30313013B2C4D82F82A
:100B6000F03001240B46D618B3FBF1F001FB103036
:100B700010F0FF0016F804AC16F803EC16F802CCDF
:100B800016F8017C36D115F80E8015F80CE015F832
:100B900007C015F80A70E00900EB400084EA080875
:100BA00000EBC0006400C0B2E4B24440C246581A30
:100BB000C0B212F800808AEA080A02F803A01044C2
:100BC000043390F801808EEA080E86F801E090F870
:100BD00002E08CEA0E0C86F802C0C078DBB2474017
:100BE0009945F770BFD80020AAE710F8015B03F819
:100BF000015FA9E71829DAD9102801BF15F80AA062
:100C000015F80EE015F80CC0EF5DD0E7010101000A
:100C1000A04601082DE9F04FA3B092F8F0301D91E5
:100C20001B920193002B00F0538101461EA8FFF791
:100C300034FF1B9BA74CA84DA84E103302930023F2
:100C400003939DF87C0004909DF886000590205C3D
:100C500006909DF87B000790205C089004989DF812
:100C600081C0205C099014F80C000A909DF8800067
:100C70000B909DF885009DF878809DF87DE09DF8AB
:100C800082A09DF887900C909DF87A00029B1C939F
:100C900014F80A2014F8093014F8081014F80E702B
:100CA0000D90205C0E909DF87F000F90205C1090BE
:100CB0000B98205C11900C98205C12909DF8840099
:100CC00013909DF8790014909DF87E001590205C9B
:100CD00016909DF883001790205C18901398205C64
:100CE00019901498205C1A90039801300390029890
:100CF000DDF804B0103002909DF80C00834536D822
:100D00008DF878108DF87A2009990E9A8DF87C105C
:100D10008DF882201199069A8DF880108DF87E202A
:100D20001999169A8DF884108DF886200A99189AC8
:100D30008DF87D108DF887201299109A8DF87B30F0
:100D40001B9B8DF881108DF883201A99089A1D98A5
:100D50008DF885108DF87F201EA903EB0B128DF8FE
:100D60007970FFF79AFE002023B0BDE8F08F15F8E8
:100D700008B082EA03008BEA000016F80EB080EAA1
:100D80000B008DF8780015F80E004B40434016F824
:100D90000A0043408DF8793081EA070315F80A10FC
:100DA000594016F80930594016F808308DF87A1075
:100DB0007A40534015F8092053408DF87B30089A4B
:100DC000069B5340049AAA5C534016F80C205340EB
:100DD0008DF87C30DDE908325A4015F80C3053406C
:100DE000059AB25C53408DF87D30DDE909325A40F6
:100DF000059BEB5C5340079AB25C53408DF87E3004
:100E0000069B0A9A5340049AB25C5A40079BEB5CDB
:100E10005A408DF87F200E9B109A53400B9AAA5C83
:100E200053400C9AB25C53408DF88030DDE91032AB
:100E30005A400C9BEB5C53400D9AB25C53408DF8CA
:100E40008130DDE911325A400D9BEB5C53400F9A23
:100E5000B25C53408DF88230129A0E9B53400B9A2D
:100E6000B25C5A400F9BEB5C1C995A408DF8832072
:100E7000169B189A5340139AAA5C5340149AB25C7A
:100E800053408DF88430DDE918325A40149BEB5CF6
:100E90005340159AB25C53408DF88530DDE9193224
:100EA0005A40159BEB5C5340179AB25C53408DF847
:100EB00086301A9A169B5340139AB25C5340179A85
:100EC000AA5C1EA853408DF88730FFF7A5FDB8E651
:100ED000FF2049E7A0460108A0440108A0450108F9
:100EE00008B538B1044A05491060D82200F0B0FABC
:100EF000002008BD0220FCE7A8240020D04B0108F8
:100F00000A4B1A6870B5002302F1180503EB0314AD
:100F10002E5D864204D1183422440A60002070BD40
:100F200001330B2BF2D10320F9E700BFA8240020E6
:100F30002DE9F041CCB00646DDF8488117461C4645
:100F40000D4631B3B8F1000F23D006A8FFF72EFCF1
:100F5000204601A9FFF7D4FF0446B0B9019906A8BD
:100F60000131FFF733FC26B11022314606A8FFF706
:100F700032FC3A46294606A8FFF72DFC06A902A82E
:100F8000FFF794FC029BC8F8003020464CB0BDE847
:100F9000F0810224F9E7000030B595B013A90446AA
:100FA000FFF7AEFF002830D11B490C2303FB00F2F2
:100FB000555CA5422BD1139B187C1090D87B0F90C9
:100FC000987B0E90587B0D90187B0C90D87A0B90E4
:100FD000987A0A90587A0990187A0890D8790790E8
:100FE000987906905879059018790490D8780390EC
:100FF000987802900A445B780193936800930022EA
:10100000064B1146022002F019FA15B030BD01302E
:101010000B28CBD1F9E700BF18490108A047010808
:101020000B2B10B402D810BCFFF782BF032010BCFA
:10103000704730B50D4685B01446014668B103AA25
:10104000002000922A460390FFF772FF18B9039818
:10105000001B18BF012005B030BD0220FBE72DE9C1
:10106000F0430D46BFB014469946804620B31BB3EB
:1010700011F00F0122D1F02201A800F0FDF9204665
:101080006946FFF73DFF044648B9009801AA1021C0
:101090000130FFF745FD2E46AF1BFFB21EB92046BB
:1010A0003FB0BDE8F08301AA09EB070108EB070098
:1010B000FFF7B0FD103EEFE70224F0E70524EEE76E
:1010C000F0B5184E3468024685B00846002304F196
:1010D000180103EB03154F5D97421ED10D2A05F150
:1010E000190513D10023CDE90033CDE902330C22D9
:1010F00010216B46FFF7B3FF0446306810226946A3
:10110000284400F0A5F9204605B0F0BD01461022A4
:10111000601900F09DF90024F5E701330B2BD8D1BD
:101120000324F0E7A824002009B1FFF7C9BF02207B
:1011300070471FB51446A0B10C2A01D10B2912D15A
:101140000023CDE90033CDE902330A466B46102176
:10115000FFF785FF18B969462046FFF7B1FF04B0D5
:1011600010BD0220FBE70320F9E7F8B51E46DDE9D4
:1011700007479DF818505BB354B34FB3212D29D8BE
:1011800019462A46204600F063F90122631C691EB5
:10119000B018FFF764FFF8B9E37ADB093B70EBB9ED
:1011A0006319204613F8012C13F8021C120642EAB8
:1011B000014213F8041C0A4313F8031C012342EAFA
:1011C0000122291FFFF735FF003818BF0120F8BDA5
:1011D0000220FCE70520FAE70720F8E70420F6E7FD
:1011E00010B5044628B1044B5B6998472060002085
:1011F00010BD0220FCE700BF304A010808B50146D7
:1012000030B1044B0822186800F022F9002008BD14
:101210000220FCE7A824002008B530B1044B0822C6
:10122000196800F015F9002008BD0220FCE700BF96
:10123000A82400207FB5124E0023044602A8019383
:101240000D46FFF7E9FF33685B6901936CB102AAB1
:10125000082312F8011B41B9013B13F0FF03F8D139
:1012600002A8A04702A8FFF7C9FF35B1019B23B927
:1012700001A8A8473368019A5A61002004B070BDE4
:10128000A824002008B5014638B1054B186808228B
:10129000104400F0DDF8002008BD0220FCE700BF8C
:1012A000A824002008B538B1044B1968082211445D
:1012B00000F0CEF8002008BD0220FCE7A8240020A2
:1012C000034B1B6802280CBF19615961002070474D
:1012D000A824002041B1054B1B6802280CBF1B69E4
:1012E0005B690B600020704702207047A824002033
:1012F00030B58FB0002405460CA80994FFF78CFF89
:101300009DF8373007939DF8363006939DF83530B9
:1013100005939DF8343004939DF8333003939DF882
:10132000323002939DF8313001939DF830300093B4
:10133000224621461E4B022002F080F80AA8FFF741
:10134000B1FF9DF82F3007939DF82E3006939DF83E
:101350002D3005939DF82C3004939DF82B3003938A
:101360009DF82A3002939DF8293001939DF828308A
:10137000009322460F4B2146022002F05FF809A994
:101380002846FFF7A7FF9DF8243003939DF82530EA
:1013900002939DF8263001939DF827300093224652
:1013A000054B2146022002F049F80FB030BD00BFC6
:1013B000FC4701083A4801087848010808B50020B0
:1013C000FFF7EAFD0120FFF7E7FD0920FFF7E4FD45
:1013D0000820FFF7E1FD0020FFF78AFF002008BD8D
:1013E00010B504460B20FFF7D7FD0C20FFF7D4FD06
:1013F0000920FFF7D1FD0820FFF7CEFD0A20FFF7F7
:10140000CBFD2046FFF774FF002010BD014B186094
:10141000704700BFAC0800200B4A30B514680B4D74
:1014200043F2390305FB04331360091A6FF00042DD
:10143000B3FBF2F2C2EBC27201319B1A93FBF1F2E1
:1014400001FB1233184430BDAC0800206D4EC6417C
:1014500001380A44914200D1704711F8013B00F86D
:10146000013FF7E710440A44914200D1704711F858
:10147000013B00F8013DF7E702F020BD30B530B187
:101480000A4D01444FF0FF33814201D1D84330BDB2
:1014900010F8012B5340082243F30004013A2C407A
:1014A00092B284EA5303002AF6D1EDE72083B8ED27
:1014B00001207047054B4FF400529A62044B1B68A1
:1014C00013B15B6803B11847704700BF00040048C0
:1014D000AC250020054B4FF480529A62044B1B68E8
:1014E00013B1DB6803B11847704700BF0004004820
:1014F000AC250020012070470120704701F048B959
:1015000001F036B910B501F019FE0E21044640F67F
:101510001F1001F02DF92046012101F0F9FDBDE871
:10152000104001F0D7BA000070B50C4E01EB40033B
:101530000D46B3654FF6FF71002304461A46084670
:1015400001F05EFB96F85600002101F0E1FD29460E
:101550002046BDE8704001F095BA00BFC8250020C4
:1015600010B5044601F0AAFE01281CD101F0AEFE20
:1015700034B11248214602F017FB104802F0DAFAA3
:101580000F4C104B00214FF48052A1659A6194F8E2
:10159000560001F0BDFD63786BB16FF07F40BDE890
:1015A000104001F053BA002340F262211A46084667
:1015B00001F026FBDCE7A0688001F0E7B025002001
:1015C000C825002000040048002001F0BFB9000039
:1015D00008B501F0C7F80438C0B2032896BF024B23
:1015E0000020185C08BD00BF2C4A010808B501F0B6
:1015F000BAFD033008BD01F049B901F009B908B5D9
:1016000001F000FD00B208BD38B50D46144601F0EA
:101610005DFB284601F092FD0E21054640F61F10A5
:1016200001F0A6F828460121074D01F071FD01F0F7
:1016300051FA4FF47A716143284602F0B5FA284610
:10164000BDE8384002F076BA2426002001F03EBB07
:1016500008B5084B002193F8560001F059FD00230E
:101660004FF4C0711A46084601F0CAFABDE80840B6
:1016700001F024BAC825002010B5044601F01EFE72
:1016800001281CD101F022FE34B11248214602F09B
:101690008BFA104802F04EFA0F4C104B00214FF419
:1016A0008052A1659A6194F8560001F031FD63788B
:1016B0006BB16FF07F40BDE8104001F07DB90023B1
:1016C00040F262211A46084601F09AFADCE7A06867
:1016D0008001F0E7B0250020C82500200004004864
:1016E00008B54FF0040001F017F9BDE808400220EA
:1016F000F1F71CBA08B500231A461946184601F03E
:101700007FFABDE8084001F06DB900001D4B73B5CC
:101710001D4D186000241D486C70C5E90144AC657E
:1017200001F098FAAC8101F003FA2146204601F05D
:101730004BFC21460422012001F0FCFA144E154D09
:101740004FF6FF7123462246084601F059FAFFF78B
:10175000C7FF2246104B00944FF0FF31304602F095
:101760003DF90E4B009422464FF0FF31284602F01F
:1017700035F9304602F090F9284602B0BDE87040D5
:1017800002F08AB9AC250020C825002055270108A1
:1017900024260020B0250020B5140108D514010826
:1017A0000128084805D1084BC17719700E3001F0A7
:1017B000A7BB437D012B03D1034B81751970F5E75E
:1017C000704700BFC8250020B00800200D4B10B5A1
:1017D000044618735873012000F016F85CB13421E8
:1017E0004FF4E86000F0C4FF4421BDE8104040F22F
:1017F000417000F0BDBF14214FF4E86000F0B8FF65
:101800002421F2E7C825002038B5114C0546207088
:1018100001F061FD052D04D8DFE805F0090B031781
:101820001709032001F070FA0023637338BD00200C
:10183000F8E7012001F068FA207B637B8342F5D052
:101840006073BDE83840FFF7C1BF0220EAE700BF80
:10185000C82500202DE9F0431E4687B00023054629
:10186000CDE901330C46174601F027FD032D61D861
:10187000DFE815F07B00C3000E010400A27C082AFB
:1018800004D94FF0FF3007B0BDE8F083A16801A88C
:1018900001F0DCFE21680029F3D042F2107291427F
:1018A000E37C864D51D80322AA7385F83820E9637A
:1018B00085F844304FF002086368A17DDB002B827D
:1018C0000423AB74A37CDB00EB7402294FF000030C
:1018D0002B75637D02D0227D022A42D103F10F02D3
:1018E000D2B2012A01D9012BCBD1754B754A1968A7
:1018F00003944FF0010903A88DF8149001F0DAFC6D
:101900000028BED1287685F817906875FFF75CFE31
:101910004046FFF779FF6C4801F086FA6B4801F00A
:10192000EFFA01A800F084FF208A00F055FFA0899B
:1019300000F09AFF384601F001FC604C84F8560034
:1019400001F0C0FC666000209DE74FF00008E963ED
:10195000890885F80E8085F8388085F84430296438
:10196000AAE7EB7529766A75D0E72368002B88D043
:10197000A27C082A85D8514DA16801A801F066FE15
:10198000002385F838302268EA63E27C85F8442039
:10199000A269AB732A646268A17DD2002A82042204
:1019A000AA74A27C2B75D2000229637DEA7402D04E
:1019B000227D022A1DD103F10F02D2B2012A02D9DF
:1019C000012B7FF45EAF3E4B3E4A196803944FF003
:1019D000010803A88DF8148001F06CFC00287FF446
:1019E00050AF287685F817806875FFF7EDFD002069
:1019F0008FE7EB7529766A75F7E7304D012185F899
:101A00003810227885F85020637885F85130A37813
:101A100085F85230E3788B4202D0022B03D03BB9D9
:101A200085F8533004E00B3A012A29D885F8531081
:101A30004FF0010885F80E80A388AB83A379AB77BC
:101A4000E37985F82030237A85F82130FFF7BCFD53
:101A50004046FFF7D9FE1C4801F0E6F91B4801F0AB
:101A60004FFA95F85130062B40F689000AD100F064
:101A70008FFE00F0FB0140F6890000F079FE59E787
:101A80000023CDE700F084FE40F00401C9B2F2E784
:101A90002368013BB3F57A7FBFF4F3AE0320FFF771
:101AA000B3FE0648022380F8383023688364162387
:101AB00080F84C30383001F0B7F93BE7C8250020FA
:101AC000AC2500202426002000260020D62500205A
:101AD0002DE9F041002686B01F461446CDE9016687
:101AE00080460D4601F0E9FBB442764C16BF012357
:101AF000334637466370B8F1000F06D0B8F1010FD6
:101B00007CD0002006B0BDE8F081AB68002B00F06F
:101B1000D680EB68002B00F0D280AA7F082A00F262
:101B2000CE80296901A801F091FD2868003818BF0E
:101B3000012000F0D9FF84F83880AB68E36395F8A2
:101B4000203084F84430686801F05AFB84F80E8035
:101B500084F84500EB68DB002382EB7FA374AB7F46
:101B6000DB00E37495F82130237595F82230002BC3
:101B70003ED12A7D95F82410A275022995F82320DC
:101B800001D0022B36D102F10F03DBB2012B02D9B7
:101B9000012A40F0948000238DF814304A4B4B4AC0
:101BA0001968049503A801F085FB002840F08780A0
:101BB00001232076E3756075FFF706FD0020FFF72F
:101BC00023FE434801F030F9424801F099F901A899
:101BD00000F02EFEA88B00F0FFFD288B00F044FEE5
:101BE0004FF4FA53AA687B43B3FBF2F3A36088E790
:101BF000FF22BFE7E27521766375DDE72B8E002BB0
